:020000040800F2
:10000000000004208D730408E9DA0308EBDA030822
:10001000EDDA0308EFDA0308F1DA03080000000064
:10002000000000000000000000000000F3DA0308F8
:10003000F5DA030800000000F7DA0308F9DA03082C
:10004000DD730408DD730408DD730408DD73040840
:10005000DD730408DD73040821B7030839B703080A
:1000600051B7030869B7030881B70308DD730408B3
:10007000DD730408DD730408DD730408DD73040810
:10008000DD7304080DBE0308DD730408DD73040886
:1000900081920308DD730408DD73040899B703082F
:1000A000DD730408ADE00308DD730408DD730408A4
:1000B000FDE003084DE10308A5E10308EDBD0308D9
:1000C000F9BD0308DD730408DD730408DD7304085B
:1000D000DD730408DD73040835D80308BDD70308B1
:1000E000CDB70308DD730408DD730408DD7304086D
:1000F000DD730408DD730408DD730408DD73040890
:1001000000000000DD730408F1B50308DD73040886
:100110000000000000000000DD73040805E2030891
:10012000DD730408DD73040895DA0308A1DA030817
:10013000DD730408DD730408DD730408DD7304084F
:10014000DD730408DD730408DD73040819DB03089C
:10015000DD730408DD73040879CD0308DD7304083A
:10016000DD730408DD7304080000000000000000D7
:10017000000000000000000000000000000000007F
:10018000DD730408DD7304080000000000000000B7
:10019000DD730408DD7304080000000000000000A7
:1001A000000000000000000000000000000000004F
:1001B000DD7304080000000000000000DD73040887
:0401C000DD730408DF
:1001D00010B5054C237833B9044B13B10448AFF381
:1001E00000800123237010BDA81D00200000000026
:1001F000EC73040808B5034B1BB103490348AFF384
:10020000008008BD00000000AC1D0020EC73040855
:1002100010F8012B11F8013B012A28BF9A42F7D0B0
:10022000D01A7047034613F8012B002AFBD1181A85
:1002300001387047000000000000000000000000CE
:1002400001F0FF01102A2BDB10F0070F08D010F887
:10025000013B013A8B422DD010F0070F42B3F6D18B
:10026000F0B441EA012141EA014122F007047FF0A4
:1002700000070023F0E80256083C85EA010586EAFB
:10028000010685FA47F5A3FA87F586FA47F6A5FA37
:1002900087F68EB9EED1F0BC01F0FF0102F0070243
:1002A00032B110F8013B013A83EA010313B1F8D1EE
:1002B0000020704701387047002D06BF35460338CF
:1002C000073815F0010F07D1013015F4807F02BF08
:1002D000013015F4C03F0130F0BC0138704700BF59
:1002E00081F0004102E000BF83F0004330B54FEAE7
:1002F00041044FEA430594EA050F08BF90EA020F54
:100300001FBF54EA000C55EA020C7FEA645C7FEAE6
:10031000655C00F0E2804FEA5454D4EB5555B8BF09
:100320006D420CDD2C4480EA020281EA030382EA7A
:10033000000083EA010180EA020281EA0303362D0C
:1003400088BF30BD11F0004F4FEA01314FF4801CDF
:100350004CEA113102D0404261EB410113F0004FF1
:100360004FEA03334CEA133302D0524263EB4303A8
:1003700094EA050F00F0A780A4F10104D5F1200E46
:100380000DDB02FA0EFC22FA05F2801841F10001A1
:1003900003FA0EF2801843FA05F359410EE0A5F175
:1003A00020050EF1200E012A03FA0EFC28BF4CF0A6
:1003B000020C43FA05F3C01851EBE37101F000455C
:1003C00007D54FF0000EDCF1000C7EEB00006EEB69
:1003D0000101B1F5801F1BD3B1F5001F0CD34908F3
:1003E0005FEA30004FEA3C0C04F101044FEA44524A
:1003F00012F5800F80F09A80BCF1004F08BF5FEAD1
:10040000500C50F1000041EB045141EA050130BDB0
:100410005FEA4C0C404141EB010111F4801FA4F153
:100420000104E9D191F0000F04BF01460020B1FAA8
:1004300081F308BF2033A3F10B03B3F120020CDAE0
:100440000C3208DD02F1140CC2F10C0201FA0CF0BE
:1004500021FA02F10CE002F11402D8BFC2F1200C23
:1004600001FA02F120FA0CFCDCBF41EA0C019040D9
:10047000E41AA2BF01EB0451294330BD6FEA040422
:100480001F3C1CDA0C340EDC04F11404C4F120020D
:1004900020FA04F001FA02F340EA030021FA04F31F
:1004A00045EA030130BDC4F10C04C4F1200220FA76
:1004B00002F001FA04F340EA0300294630BD21FAB4
:1004C00004F0294630BD94F0000F83F4801306BF7A
:1004D00081F480110134013D4EE77FEA645C18BF6E
:1004E0007FEA655C29D094EA050F08BF90EA020F05
:1004F00005D054EA000C04BF1946104630BD91EAFD
:10050000030F1EBF0021002030BD5FEA545C05D1FF
:100510004000494128BF41F0004130BD14F580043E
:100520003CBF01F5801130BD01F0004545F0FE41B2
:1005300041F470014FF0000030BD7FEA645C1ABFE7
:10054000194610467FEA655C1CBF0B46024650EA1E
:10055000013406BF52EA033591EA030F41F400214A
:1005600030BD00BF90F0000F04BF0021704730B5D0
:100570004FF4806404F132044FF000054FF00001A5
:1005800050E700BF90F0000F04BF0021704730B566
:100590004FF4806404F1320410F0004548BF40423B
:1005A0004FF000013EE700BF42004FEAE2014FEA90
:1005B00031014FEA02701FBF12F07F4393F07F4F6B
:1005C00081F06051704732F07F4208BF704793F06E
:1005D0007F4F04BF41F40021704730B54FF4607481
:1005E00001F0004521F000411CE700BF50EA010284
:1005F00008BF704730B54FF000050AE050EA01022D
:1006000008BF704730B511F0004502D5404261EB9C
:1006100041014FF4806404F132045FEA915C3FF4DD
:10062000D8AE4FF003025FEADC0C18BF03325FEA7A
:10063000DC0C18BF033202EBDC02C2F1200300FA2B
:1006400003FC20FA02F001FA03FE40EA0E0021FA50
:1006500002F11444BDE600BF70B54FF0FF0C4CF43E
:10066000E06C1CEA11541DBF1CEA135594EA0C0FF0
:1006700095EA0C0F00F0DEF82C4481EA030621EA2B
:100680004C5123EA4C5350EA013518BF52EA033566
:1006900041F4801143F4801338D0A0FB02CE4FF018
:1006A0000005E1FB02E506F00042E0FB03E54FF048
:1006B0000006E1FB03569CF0000F18BF4EF0010E40
:1006C000A4F1FF04B6F5007F64F5407404D25FEA3C
:1006D0004E0E6D4146EB060642EAC62141EA5551EF
:1006E0004FEAC52040EA5E504FEACE2EB4F1FD0C31
:1006F00088BFBCF5E06F1ED8BEF1004F08BF5FEAAF
:10070000500E50F1000041EB045170BD06F0004660
:1007100046EA010140EA020081EA0301B4EB5C040D
:10072000C2BFD4EB0C0541EA045170BD41F4801105
:100730004FF0000E013C00F3AB8014F1360FDEBF2A
:10074000002001F0004170BDC4F10004203C35DA06
:100750000C341BDC04F11404C4F1200500FA05F389
:1007600020FA04F001FA05F240EA020001F000422A
:1007700021F0004110EBD37021FA04F642EB0601A0
:100780005EEA430E08BF20EAD37070BDC4F10C04CA
:10079000C4F1200500FA04F320FA05F001FA04F28E
:1007A00040EA020001F0004110EBD37041F100017A
:1007B0005EEA430E08BF20EAD37070BDC4F1200585
:1007C00000FA05F24EEA020E20FA04F301FA05F2ED
:1007D00043EA020321FA04F001F0004121FA04F295
:1007E00020EA020000EBD3705EEA430E08BF20EA65
:1007F000D37070BD94F0000F0FD101F0004640009F
:1008000041EB010111F4801F08BF013CF7D041EA20
:10081000060195F0000F18BF704703F00046520024
:1008200043EB030313F4801F08BF013DF7D043EAF5
:100830000603704794EA0C0F0CEA135518BF95EAAB
:100840000C0F0CD050EA410618BF52EA4306D1D132
:1008500081EA030101F000414FF0000070BD50EA51
:10086000410606BF1046194652EA430619D094EADB
:100870000C0F02D150EA013613D195EA0C0F05D1C5
:1008800052EA03361CBF104619460AD181EA030119
:1008900001F0004141F0FE4141F470014FF00000D1
:1008A00070BD41F0FE4141F4780170BD70B54FF06C
:1008B000FF0C4CF4E06C1CEA11541DBF1CEA1355EC
:1008C00094EA0C0F95EA0C0F00F0A7F8A4EB0504CE
:1008D00081EA030E52EA03354FEA013100F08880C5
:1008E0004FEA03334FF0805545EA131343EA12638E
:1008F0004FEA022245EA111545EA10654FEA002643
:100900000EF000419D4208BF964244F1FD0404F5FB
:10091000407402D25B084FEA3202B61A65EB030557
:100920005B084FEA32024FF480104FF4002CB6EB14
:10093000020E75EB030E22BFB61A754640EA0C0094
:100940005B084FEA3202B6EB020E75EB030E22BFD4
:10095000B61A754640EA5C005B084FEA3202B6EB15
:10096000020E75EB030E22BFB61A754640EA9C00D4
:100970005B084FEA3202B6EB020E75EB030E22BFA4
:10098000B61A754640EADC0055EA060E18D04FEA62
:10099000051545EA16754FEA06164FEAC30343EA02
:1009A00052734FEAC2025FEA1C1CC0D111F4801FCF
:1009B0000BD141EA00014FF000004FF0004CB6E7C8
:1009C00011F4801F04BF01430020B4F1FD0C88BF67
:1009D000BCF5E06F3FF6AFAEB5EB030C04BFB6EB72
:1009E000020C5FEA500C50F1000041EB045170BD65
:1009F0000EF0004E4EEA113114EB5C04C2BFD4EB92
:100A00000C0541EA045170BD41F480114FF0000E15
:100A1000013C90E645EA060E8DE60CEA135594EA91
:100A20000C0F08BF95EA0C0F3FF43BAF94EA0C0F94
:100A30000AD150EA01347FF434AF95EA0C0F7FF409
:100A400025AF104619462CE795EA0C0F06D152EA5D
:100A500003353FF4FDAE1046194622E750EA410641
:100A600018BF52EA43067FF4C5AE50EA41047FF452
:100A70000DAF52EA43057FF4EBAE12E74FF0FF3CB7
:100A800006E000BF4FF0010C02E000BF4FF0010C88
:100A90004DF804CD4FEA410C7FEA6C5C4FEA430C01
:100AA00018BF7FEA6C5C1BD001B050EA410C0CBF50
:100AB00052EA430C91EA030F02BF90EA020F0020B2
:100AC000704710F1000F91EA030F58BF994208BF19
:100AD00090422CBFD8176FEAE37040F001007047D6
:100AE0004FEA410C7FEA6C5C02D150EA013C07D12D
:100AF0004FEA430C7FEA6C5CD6D152EA033CD3D078
:100B00005DF8040B704700BF8446104662468C4671
:100B10001946634600E000BF01B5FFF7B7FF0028A4
:100B200048BF10F1000F01BD4DF808EDFFF7F4FFCD
:100B30000CBF012000205DF808FB00BF4DF808ED58
:100B4000FFF7EAFF34BF012000205DF808FB00BF7B
:100B50004DF808EDFFF7E0FF94BF012000205DF89D
:100B600008FB00BF4DF808EDFFF7CEFF94BF012052
:100B700000205DF808FB00BF4DF808EDFFF7C4FF4B
:100B800034BF012000205DF808FB00BF4FEA410C94
:100B90007FEA6C5C02D150EA013C0AD14FEA430C77
:100BA0007FEA6C5C02D152EA033C02D14FF00000B4
:100BB00070474FF0010070474FEA410212F50012F2
:100BC00015D211D56FF47873B3EB625212D94FEA94
:100BD000C12343F0004343EA505311F0004F23FA7E
:100BE00002F018BF404270474FF00000704750EAD3
:100BF000013005D111F0004008BF6FF00040704790
:100C00004FF00000704700BF4A0011D212F50012E9
:100C100011D20DD56FF47873B3EB62520ED44FEA54
:100C2000C12343F0004343EA505323FA02F07047D4
:100C30004FF00000704750EA013002D14FF0FF3012
:100C400070474FF0000070474FEA4102B2F1E043B5
:100C500024BFB3F5001CDCF1FE5C0DD901F0004CA3
:100C60004FEAC0024CEA5070B2F1004F40EB8300F3
:100C700008BF20F00100704711F0804F21D113F11F
:100C80003872BCBF01F00040704741F480114FEA58
:100C90005252C2F11802C2F1200C10FA0CF320FAE1
:100CA00002F018BF40F001004FEAC1234FEAD323FE
:100CB00003FA0CFC40EA0C0023FA02F34FEA430368
:100CC000CCE77FEA625307D150EA01331EBF4FF0F1
:100CD000FE4040F44000704701F0004040F0FE400C
:100CE00040F40000704700BF80F0004002E000BF09
:100CF00081F0004142001FBF5FEA410392EA030F07
:100D00007FEA226C7FEA236C6AD04FEA1262D2EB50
:100D10001363C1BFD218414048404140B8BF5B4255
:100D2000192B88BF704710F0004F40F4000020F0EE
:100D30007F4018BF404211F0004F41F4000121F004
:100D40007F4118BF494292EA030F3FD0A2F101024E
:100D500041FA03FC10EB0C00C3F1200301FA03F18C
:100D600000F0004302D5494260EB4000B0F5000FAF
:100D700013D3B0F1807F06D340084FEA310102F16E
:100D80000102FE2A51D2B1F1004F40EBC25008BF20
:100D900020F0010040EA03007047490040EB0000EA
:100DA00010F4000FA2F10102EDD1B0FA80FCACF119
:100DB000080CB2EB0C0200FA0CF0AABF00EBC25018
:100DC00052421843BCBFD0401843704792F0000F06
:100DD00081F4000106BF80F400000132013BB5E759
:100DE0004FEA41037FEA226C18BF7FEA236C21D0CF
:100DF00092EA030F04D092F0000F08BF0846704734
:100E000090EA010F1CBF0020704712F07F4F04D101
:100E1000400028BF40F00040704712F100723CBF14
:100E200000F50000704700F0004343F0FE4040F43E
:100E3000000070477FEA226216BF08467FEA2363FC
:100E40000146420206BF5FEA412390EA010F40F4E7
:100E5000800070474FF0000304E000BF10F0004333
:100E600048BF40425FEA000C08BF704743F096431A
:100E700001464FF000001CE050EA010208BF704735
:100E80004FF000030AE000BF50EA010208BF7047BC
:100E900011F0004302D5404261EB41015FEA010CD1
:100EA00002BF84460146002043F0B64308BFA3F1C9
:100EB0008053A3F50003BCFA8CF2083AA3EBC253AB
:100EC00010DB01FA02FC634400FA02FCC2F12002CA
:100ED000BCF1004F20FA02F243EB020008BF20F001
:100EE0000100704702F1200201FA02FCC2F1200267
:100EF00050EA4C0021FA02F243EB020008BF20EA5C
:100F0000DC7070474FF0FF0C1CEAD0521EBF1CEA89
:100F1000D15392EA0C0F93EA0C0F6FD01A4480EA77
:100F2000010C400218BF5FEA41211ED04FF0006360
:100F300043EA501043EA5111A0FB01310CF000408C
:100F4000B1F5000F3EBF490041EAD3715B0040EAB2
:100F5000010062F17F02FD2A1DD8B3F1004F40EB82
:100F6000C25008BF20F00100704790F0000F0CF055
:100F7000004C08BF49024CEA502040EA51207F3A19
:100F8000C2BFD2F1FF0340EAC250704740F40000F4
:100F90004FF00003013A5DDC12F1190FDCBF00F0E5
:100FA00000407047C2F10002410021FA02F1C2F193
:100FB000200200FA02FC5FEA310040F1000053EA2F
:100FC0004C0308BF20EADC70704792F0000F00F07D
:100FD000004C02BF400010F4000F013AF9D040EA83
:100FE0000C0093F0000F01F0004C02BF490011F417
:100FF000000F013BF9D041EA0C018FE70CEAD15315
:1010000092EA0C0F18BF93EA0C0F0AD030F0004C94
:1010100018BF31F0004CD8D180EA010000F0004048
:10102000704790F0000F17BF90F0004F084691F006
:10103000000F91F0004F14D092EA0C0F01D1420240
:101040000FD193EA0C0F03D14B0218BF084608D109
:1010500080EA010000F0004040F0FE4040F4000053
:10106000704740F0FE4040F4400070474FF0FF0CE6
:101070001CEAD0521EBF1CEAD15392EA0C0F93EA2D
:101080000C0F69D0A2EB030280EA010C49024FEA7F
:10109000402037D04FF0805343EA111143EA101338
:1010A0000CF000408B4238BF5B0042F17D024FF4F0
:1010B000000C8B4224BF5B1A40EA0C00B3EB510FCB
:1010C00024BFA3EB510340EA5C00B3EB910F24BFB4
:1010D000A3EB910340EA9C00B3EBD10F24BFA3EB39
:1010E000D10340EADC001B0118BF5FEA1C1CE0D101
:1010F000FD2A3FF650AF8B4240EBC25008BF20F0B4
:10110000010070470CF0004C4CEA50207F32C2BF07
:10111000D2F1FF0340EAC250704740F400004FF0A4
:101120000003013A37E792F0000F00F0004C02BFD5
:10113000400010F4000F013AF9D040EA0C0093F09F
:10114000000F01F0004C02BF490011F4000F013BF9
:10115000F9D041EA0C0195E70CEAD15392EA0C0F61
:1011600008D142027FF47DAF93EA0C0F7FF470AF99
:10117000084676E793EA0C0F04D14B023FF44CAFDC
:1011800008466EE730F0004C18BF31F0004CCAD171
:1011900030F000427FF45CAF31F000437FF43CAFAD
:1011A0005FE700BF4FF0FF3C06E000BF4FF0010CCF
:1011B00002E000BF4FF0010C4DF804CD4FEA4002B1
:1011C0004FEA41037FEA226C18BF7FEA236C11D0FB
:1011D00001B052EA530C18BF90EA010F58BFB2EBAE
:1011E000030088BFC81738BF6FEAE17018BF40F02E
:1011F000010070477FEA226C02D15FEA402C05D1E2
:101200007FEA236CE4D15FEA412CE1D05DF8040B66
:10121000704700BF844608466146FFE70FB5FFF7F9
:10122000C9FF002848BF10F1000F0FBD4DF808EDB1
:10123000FFF7F4FF0CBF012000205DF808FB00BFA2
:101240004DF808EDFFF7EAFF34BF012000205DF8FC
:1012500008FB00BF4DF808EDFFF7E0FF94BF012049
:1012600000205DF808FB00BF4DF808EDFFF7D2FF46
:1012700094BF012000205DF808FB00BF4DF808ED89
:10128000FFF7C8FF34BF012000205DF808FB00BF56
:101290004FEA40024FEA41037FEA226C02D15FEA43
:1012A000402C08D17FEA236C02D15FEA412C02D1A5
:1012B0004FF0000070474FF0010070474FEA4002C6
:1012C000B2F1FE4F0FD34FF09E03B3EB12620DD974
:1012D0004FEA002343F0004310F0004F23FA02F0DE
:1012E00018BF404270474FF00000704712F1610F85
:1012F00001D1420205D110F0004008BF6FF000405C
:1013000070474FF00000704742000ED2B2F1FE4F1E
:101310000BD34FF09E03B3EB126209D44FEA0023C4
:1013200043F0004323FA02F070474FF0000070478B
:1013300012F1610F01D1420202D14FF0FF3070472C
:101340004FF00000704700BF7BB972B90029BEBFE3
:1013500000204FF0004106E008BF00281CBF6FF0DE
:1013600000414FF0FF3000F0BDB9ADF1080C6DE960
:1013700004CE002909DB002B1ADB00F04DF8DDF864
:1013800004E0DDE9022304B07047404261EB410113
:10139000002B1BDB00F040F8DDF804E0DDE9022360
:1013A00004B0404261EB4101524263EB430370479A
:1013B000524263EB430300F02FF8DDF804E0DDE96F
:1013C000022304B0404261EB41017047524263EB9B
:1013D000430300F021F8DDF804E0DDE9022304B066
:1013E000524263EB4303704753B94AB9002908BF1F
:1013F00000281CBF4FF0FF314FF0FF3000F072B9F2
:10140000ADF1080C6DE904CE00F006F8DDF804E05B
:10141000DDE9022304B070472DE9F047089E044639
:101420008846002B4BD18A42154667D9B2FA82F220
:101430004AB1C2F1200701FA02F320FA07F79540FA
:1014400047EA030894404FEA154E230CB8FBFEF719
:101450001FFA85FC0EFB178843EA084307FB0CF1D3
:10146000994209D9EB1807F1FF3080F01B819942AE
:1014700040F21881023F2B445B1AA4B2B3FBFEF08A
:101480000EFB103344EA034400FB0CFCA44509D9CD
:101490002C1900F1FF3380F00781A44540F204814C
:1014A00002382C4440EA0740A4EB0C0400271EB18C
:1014B000D4400023C6E900433946BDE8F0878B429B
:1014C00009D9002E00F0EB800027C6E9000138465C
:1014D0003946BDE8F087B3FA83F7002F47D18B4236
:1014E00002D3824200F2FA80841A61EB03030120E6
:1014F0009846002EE0D0C6E90048DDE702B9FFDEDD
:10150000B2FA82F2002A40F08F80491B4FEA154E52
:101510001FFA85F80127B1FBFEFC230C0EFB1C1102
:1015200043EA014308FB0CF1994207D9EB180CF18F
:10153000FF3002D2994200F2CD808446591AA3B2FC
:10154000B1FBFEF00EFB101443EA044408FB00F864
:10155000A04507D92C1900F1FF3302D2A04500F2B3
:10156000B6801846A4EB080440EA0C409FE7C7F198
:10157000200CBB4022FA0CFE4EEA030E01FA07F4DF
:1015800020FA0CF521FA0CF34FEA1E482543B3FB71
:10159000F8F92C0C08FB19331FFA8EFA44EA0343BE
:1015A00009FB0AF49C4202FA07F200FA07F10BD990
:1015B0001EEB030309F1FF3080F087809C4240F26C
:1015C0008480A9F1020973441B1BADB2B3FBF8F090
:1015D00008FB103345EA034400FB0AFAA24508D988
:1015E0001EEB040400F1FF336BD2A24569D9023827
:1015F000744440EA0940A0FB0289A4EB0A044C456C
:10160000C2464B4654D351D0002E69D0B1EB0A05E7
:1016100064EB030404FA0CFCFD40FC404CEA0505B5
:10162000C6E90054002747E7C2F1200320FA03F778
:10163000954001FA02F021FA03F34FEA154E3843C0
:10164000010CB3FBFEF71FFA85F80EFB173341EAD6
:10165000034107FB08F38B4204FA02F407D9691827
:1016600007F1FF3C2FD28B422DD9023F2944CB1AE0
:1016700081B2B3FBFEF00EFB103341EA034100FBE5
:1016800008F38B4207D9691800F1FF3C17D28B424F
:1016900015D902382944C91A40EA07473BE73746BB
:1016A000304609E70746E7E61846FBE64145ABD278
:1016B000B8EB020A69EB0E0201381346A4E7604654
:1016C000E9E7184695E76746D1E781467CE70238A7
:1016D0002C4447E7ACF1020C2B442FE7384608E7CF
:1016E0003746E9E6704700BF704700000A4B0B4AD7
:1016F00010B51A6200240A4A1C625A62094A5C62E6
:101700001A61C0221C615A6103225C619A619C616A
:10171000FFF7EAFF204610BD00380240FFC9E61778
:10172000337917019F10600038B50E4A0E4B0546FD
:1017300018784FF47A73B3FBF0F31068B0FBF3F052
:1017400000F066FC044658B90F2D09D80246294618
:101750004FF0FF3000F006FC044B20461D6038BD02
:101760000120FCE780180020000000200400002079
:1017700008B50B4B1A6842F400721A601A6842F4FA
:1017800080621A601A6842F480721A60032000F0C6
:10179000D7FB0F20FFF7C8FF3CF088F9002008BDF9
:1017A000003C0240034A044B11681B780B44136051
:1017B000704700BF3C98002000000020014B1868D3
:1017C000704700BF3C98002038B50446FFF7F6FF8D
:1017D000631C1CBF054B1B78054618BFE418FFF7B8
:1017E000EDFF401BA042FAD338BD00BF000000202F
:1017F000014B1868704700BF107AFF1F014B186833
:10180000704700BF147AFF1F014B1868704700BF74
:10181000187AFF1F7047000038B50446002800F012
:101820009B80056C25B9FFF7F5FF656484F83C5093
:10183000236CDB0600F18E80236C23F4885323F0A5
:10184000020343F002032364444B5A6822F44032FB
:101850005A605A6861680A435A60236821695A6865
:1018600022F480725A605A6842EA01225A605A6829
:10187000A16822F040725A605A680A435A609A6816
:10188000E16822F400629A609A680A439A603449D7
:10189000A26A8A4252D0996821F070619960996871
:1018A0000A439A609A68E16A22F040529A609A6804
:1018B0000A439A609A68217E22F002029A609A682E
:1018C00042EA41029A6094F82020002A3ED05A68E9
:1018D000616A42F400625A605A6822F460425A60B7
:1018E0005A68013942EA41325A60DA6AE16922F4FF
:1018F0007002DA62DA6A013942EA0152DA629A68FF
:1019000094F8301022F400729A609A6842EA4122F8
:101910009A609A68616922F480629A609A680020ED
:1019200042EA81229A606064236C23F0030343F04F
:1019300001032364002384F83C3038BD9A6822F008
:1019400070629A609A6822F04052B2E75A6822F4B4
:101950000062C9E70120EDE70120EEE70023014026
:101960000100000F82B00023019390F83C30012B5E
:101970005CD00268012380F83C309368D9070CD50D
:10198000936813F001031AD1026C42F01002026452
:10199000426C42F00102426446E09368254943F0FC
:1019A00001039360244B1B68B3FBF1F303EB430388
:1019B0000193019B002BE3D0019B013BF8E7036CF3
:1019C00023F4E06323F0010343F48073036453685A
:1019D0005B0541BF036C23F4405343F4805303641D
:1019E000036C13F480531CBF436C23F00603436461
:1019F0006FF02201002380F83C3011600F494968E4
:101A000011F01F0109D1906810F0405010D1936877
:101A100043F08043936002B0704709498A4203D182
:101A2000906810F04050F2D01846F4E70220F2E738
:101A30000846F0E740420F008018002000230140D4
:101A40000020014003689A6870B5560504460D46AB
:101A50000BD59B68D80508D5236C43F0200323647D
:101A6000002384F83C30012070BDFFF7A7FE064636
:101A700023681A6892070CD56FF012021A60226C64
:101A800042F4007222649A6812F0405F17D000207E
:101A9000EAE7691CEDD065B923681B6813F00203FF
:101AA000E6D1226C84F83C3042F004022264032028
:101AB000DAE7FFF783FE801BA842EDD8D8E7227E45
:101AC000002AE4D1DA6A12F4700F02D09B685B0539
:101AD000DDD4236C23F480732364206C10F48050D5
:101AE000D5D1236C43F001032364BDE70368D86CB0
:101AF00070470000F7B50023019390F83C30012BAC
:101B00007ED00D688E680123092D80F83C30ACB280
:101B1000036829D904EB4402DF681E3A4FF0070C32
:101B20000CFA02FC27EA0C07DF60DF6806FA02F213
:101B30003A43DA604968062901EB810224D8596BDF
:101B4000053A1F26964021EA06015963596B04FAAB
:101B500002F20A435A632B4A934231D0002380F8A1
:101B60003C30184603B0F0BD1F6905EB45024FF04D
:101B7000070C0CFA02FC27EA0C071F611F6906FA22
:101B800002F23A431A61D5E70C294FF01F010BD836
:101B90001E6B233A914026EA01011963196B04FA7E
:101BA00002F20A431A63D6E7DE6A413A914026EA16
:101BB0000101D962D96A04FA02F20A43DA62CAE779
:101BC000122D04D1104A536843F480035360A5F1E9
:101BD0001003012BC2D80C4A5368102D43F40003A4
:101BE0005360BBD1094B0A4A1B68B3FBF2F20A23CC
:101BF00053430193019B002BB0D0019B013BF8E7BD
:101C00000220AFE70020014000230140801800209F
:101C100040420F00F0B590F82040013C012C72D8F2
:101C2000066841B9F468A40707D1436A43F4001376
:101C3000436201205CE03469F5E70C013519D5F801
:101C4000B07107F004079760002F52D1D5F8B0713A
:101C50007F0D1760D5F8B07107F00207D760D5F88F
:101C6000B47107F00F07072F96BFD5F8B471082796
:101C700007F00F071761D5F8B471D5F8B4512644B1
:101C8000C7F307272D0C97615561D6F8B8211A7054
:101C900002682244D2F8B821120A5A70026822441B
:101CA000D2F8B821120C9A7002682244D2F8B821F6
:101CB000120EDA7002682244D2F8BC211A7102684E
:101CC0002244D2F8BC21120A5A7102682244D2F886
:101CD000BC21120C9A7102681444D4F8BC21120E73
:101CE000DA71036851B9DA6842F02002DA60002044
:101CF000F0BDD5F8B071FF085760ABE71A6942F044
:101D000020021A61F3E7436A43F4802390E790F8D6
:101D10002030013B012B07D8036819B9D86800F0BF
:101D2000030070471869FAE7002070477047704752
:101D300070477047704770477047704770477047EB
:101D4000704770472DE9F84F03685E69D3F8049037
:101D50009F68D3F80CB0D3F810A0D3F8188016F011
:101D60000104054622D017F0010407D00122B9076B
:101D70009A6040F1A380FFF7D9FF0024FB0509D545
:101D80002B684FF48072B8059A6040F1A580284610
:101D9000FFF7CDFFFB0309D52B684FF48032B80362
:101DA0009A6040F1A7802846FFF7C2FF330707D5A6
:101DB0001BF0100F1FBF2B68102244F40074DA6070
:101DC000770708D51BF0080F05D02B680822DA60CA
:101DD0002846FFF7B1FFB00706D52B68DB689907E7
:101DE00002D0284637F052FA720607D51AF0100FC3
:101DF0001FBF2B68102244F480641A61B30608D513
:101E00001AF0080F05D02B6808221A612846FFF740
:101E100095FFF70606D52B681B69980702D0284660
:101E2000FFF78BFFB10308D519F0100F05D02B6811
:101E300010225A602846FFF782FFF20308D519F0F6
:101E4000080F05D02B6808225A602846FFF778FF54
:101E500033042AD519F0040F2A6824D0F70504D5D5
:101E600018F0010F18BF44F00104B00504D518F0B4
:101E7000020F18BF44F00204710504D518F0040FD6
:101E800018BF44F0040433050DD518F070030AD0D0
:101E9000302B4CD03CD8102B43D0202B44D093690E
:101EA00023F070039361042353602CB16B6A1C43CD
:101EB0006C622846FFF745FFBDE8F88F7A0705D426
:101EC00017F0080405D1FFF734FF57E74FF400641B
:101ED00054E74FF4805451E7790502D544F4005497
:101EE00058E73A0502D544F4804453E72846FFF703
:101EF00021FF4FE7790302D544F4004456E73A0343
:101F000002D544F4803451E72846FFF714FF4DE72B
:101F1000502B0FD0602B10D0402BC0D144F0400488
:101F2000BDE744F00804BAE744F01004B7E744F012
:101F30002004B4E744F08004B1E744F48074AEE7D1
:101F4000074AD36823F4E0631B041B0C43F0BF6310
:101F5000000243F4003300F4E0600343D3607047B1
:101F600000ED00E0174B70B5DC68C4F30224C4F147
:101F70000705042D04F1040328BF04254FF0FF36A4
:101F8000062B06FA05F38CBF033C002421EA030369
:101F9000A34006FA04F422EA0404002843EA0403F6
:101FA000A8BF00F160404FEA0313BCBF00F00F0070
:101FB000054ADBB2AABF00F56140135480F8003334
:101FC00070BD00BF00ED00E014ED00E0002808DB6C
:101FD0000123420900F01F0003FA00F0014B43F80F
:101FE0002200704700E100E000280DDB43090122D8
:101FF00000F01F0002FA00F02033044A42F82300E8
:10200000BFF34F8FBFF36F8F704700BF00E100E059
:102010000138B0F1807F0AD2064B074A5860F021A0
:1020200082F823100020072298601A607047012070
:10203000704700BF10E000E000ED00E00368DAB296
:1020400023F47F7323F003031821103AB2FBF1F25B
:102050000449032A88BF0433895C8365C165806DA8
:10206000704700BFFC74040870B50446FFF7A6FB78
:102070000546002C71D00223226884F835300023F5
:1020800084F83430136823F00103136021680B686F
:10209000D8073CD40B68324DA0691D40D4E9012318
:1020A0001343E26813432269134362691343E269ED
:1020B00003431343226A1343626A042A43EA050373
:1020C00002BFD4E90B5635432B430B604B69042AFE
:1020D00023F0070343EA02030BD1A26AE56A134324
:1020E0003DB1F8B9012A2DD001D3022A01D1EA016C
:1020F0002BD44B612046FFF7A1FFE26D3F239340B5
:10210000836000200123606584F8353009E0FFF723
:1021100055FB401B0528B9D920236365032084F8AB
:10212000350070BDB0F5005F13D1032AE1D801A0DE
:1021300050F822F04B210008EF2000084B21000846
:1021400045210008B5F1C07FD3D14023636501204C
:10215000E5E7022AF9D9032AC8E70120E1E700BF31
:102160003F8010F070B590F83440012C32D001243B
:1021700080F8344090F83540866D012C4FF0000512
:102180004FF0020424D180F8354004684565256885
:1021900025F48025256063608368402B0EBFA26014
:1021A000A160E260C26D08BFE1603F239340B3606D
:1021B000236843F016032360036C1BB1236843F0CC
:1021C00008032360236843F001032360002070BDEF
:1021D00080F834500220FAE790F83530022B03D013
:1021E00080234365012070470268052380F835305D
:1021F000136823F00103136000207047F7B5002334
:1022000001935C4B856D1F68C36D2E6808229A4050
:10221000324204460CD001680868400708D50868B7
:1022200020F004000860AA60626D42F0010262655D
:1022300001229A40324208D021684969090641BF0B
:10224000AA60626D42F00202626504229A40324244
:1022500008D021680968880741BFAA60626D42F012
:102260000402626510229A40324210D02368196835
:1022700009070CD5AA601A68500337D51B681903E3
:1022800001D4236C00E0A36C0BB120469847E16DAC
:1022900020228A4032423AD023681868C60636D5D2
:1022A000AA6094F83520052A1A6827D122F0160270
:1022B0001A605A6922F080025A61226C0AB9A26C33
:1022C0001AB11A6822F008021A603F238B40AB60F3
:1022D000012384F83530002384F83430236D002B3B
:1022E00045D0204603B0BDE8F04018471A68D20533
:1022F0005EBF1A6822F008021A60C2E7500327D5B1
:102300001B68190331D4636C0BB120469847636D89
:102310006BB3636DDA0719D50523226884F835306D
:10232000136823F0010313604FF41653B7FBF3F760
:10233000019B0133BB42019302D81368DB07F7D43A
:10234000012384F83530002384F83430E36CC6E789
:102350001A6812F4807208D1196821F0100119600E
:10236000012384F8353084F83420E36BCCE703B0E4
:10237000F0BD00BF8018002090F835007047406D18
:10238000704700002DE9F04F85B00B68DFF8A4819D
:10239000664A01934FF0010B0023019D0BFA03F4F1
:1023A0002540AC4240F0B2804E684FEA430E06F042
:1023B0000304032707FA0EF704F1FF3CFF43BCF1C7
:1023C000010F00973CD8D0F808C00CEA070CCF6882
:1023D00007FA0EF949EA0C0CC0F808C0D0F80490CE
:1023E000C6F3001C29EA05090CFA03FC4CEA090CA7
:1023F000C0F804C0D0F80CC0009F0CEA070C8F682E
:1024000007FA0EF949EA0C0C022CC0F80CC019D1DD
:102410004FEAD30900EB890903F0070AD9F82070C5
:102420004FEA8A0A4FF00F0C0CFA0AFC27EA0C0C50
:102430000F6907FA0AFA4AEA0C0AC9F820A001E073
:10244000032CD7D1D0F800C0009F04FA0EF40CEA98
:102450000707274316F4403F076057D04FF0000AA4
:10246000CDF80CA0D8F84470314C47F48047C8F838
:102470004470D8F8447007F480470397039F23F013
:10248000030707F1804707F59C3703F0030ED7F8E1
:1024900008904FEA8E0E4FF00F0C0CFA0EFCA04283
:1024A00029EA0C0C39D004F58064A04237D004F539
:1024B0008064A04235D004F58064A04233D004F596
:1024C0008064A04214BF0724042404FA0EF444EAF2
:1024D0000C04BC609468EF4316F4801F0CBF3C40B2
:1024E0002C439460D46816F4001F0CBF3C402C436E
:1024F000D460546816F4003F0CBF3C402C43546039
:102500001468F60354BF3C402C4314600133102B75
:102510007FF443AF05B0BDE8F08F5446D5E7012402
:10252000D3E70224D1E70324CFE700BF003C0140FA
:10253000000002400038024001684B6913F48063D8
:102540004FF0000210D06FF480634B6120230263D0
:1025500080F83D3080F83E20036C80F83C2043F04A
:102560000403036401207047184670472DE9F843BF
:10257000089E044690461F464FEA11498DB22068D6
:10258000B9F1010F0CBF4369836935EA03030CBF3E
:1025900001210021884501D0002023E07B1CEFD0E1
:1025A000FFF70CF9801BB84201D8002FE7D1216852
:1025B000B9F1010F0CBF4B698B6935EA03030CBFFE
:1025C000012100218845DAD100232022236384F8E9
:1025D0003D2084F83E30226C84F83C3042F02002EA
:1025E00022640120BDE8F8832DE9F0410446174636
:1025F00098468EB22568686936EA000017D06B6984
:102600005A0516D52B6843F400732B606FF4806372
:102610006B6120220023236384F83D2084F83E3040
:10262000226C42F00402226484F83C300120BDE8B0
:10263000F0817B1CDFD0FFF7C1F8A0EB0800B842A7
:1026400001D8002FD6D123685B6936EA0303D1D0C5
:1026500000232022236384F83D2084F83E30226C3E
:1026600042F02002DFE770B504460D4616462368A7
:102670005B695B0701D5002070BD2046FFF75CFF5A
:10268000C8B96A1CF3D0FFF799F8801BA84201D89B
:10269000002DECD123685B6913F00403E7D12022FD
:1026A000236384F83D2084F83E30226C84F83C306B
:1026B00042F0200222640120DEE770B504460D4698
:1026C00016462068436913F0400301D0002010E053
:1026D0004269D2060ED56FF01002426120222363B8
:1026E00084F83D2084F83E30226C226484F83C302B
:1026F000012070BDFFF762F8801BA84201D8002DB1
:10270000DFD123685B6913F04003DAD12022236311
:1027100084F83D2084F83E30226C42F02002E4E749
:1027200070B504460D46164623685B691B0601D545
:10273000002070BD2046FFF7FFFEC8B96A1CF3D029
:10274000FFF73CF8801BA84201D8002DECD123688C
:102750005B6913F08003E7D12022236384F83D20D6
:1027600084F83E30226C84F83C3042F0200222642F
:102770000120DEE72DE9FF41154602680B9E9846D1
:10278000136843F4807313600F460A9B009600227F
:102790004FF001110446FFF7E9FE236838B11B68CA
:1027A000DB0502D54FF40073236403200AE007F031
:1027B000FE071F610A9A194933462046FFF714FFA6
:1027C00018B1012004B0BDE8F081236803905A6974
:1027D00003929B69039332460A99039B2046FFF7B5
:1027E0009FFF40B1236C042B01BF2268136843F4A0
:1027F00000731360E5E7B8F1010F236802D1EDB271
:102800001D61DFE72A0A1A610A9932462046FFF75E
:1028100087FF0028E6D12368F1E700BF020001002E
:102820002DE9FF41984603680B9D16461A6842F44D
:1028300080621A601A6842F480721A600F460A9B1E
:10284000009500224FF001110446FFF78FFE236828
:1028500048B11B68DB0502D54FF4007323640320E5
:1028600004B0BDE8F081FFB207F0FE021A612A4908
:102870000A9A2B462046FFF7B7FE08B10120EFE782
:10288000236803905A6903929B6903932A460A9925
:10289000039B2046FFF744FF40B1236C042B01BF8C
:1028A0002268136843F400731360E7E7B8F1010F7F
:1028B000236825D1F6B21E612A460A992046FFF701
:1028C0002FFF02460028E8D121680B6843F480738B
:1028D0000B6020460A9B00954FF00111FFF746FE62
:1028E00023680028B5D147F001071F610A9A0A49F9
:1028F0002B462046FFF778FE003018BF0120AFE7D7
:10290000320A1A610A992A462046FFF709FF002871
:10291000C3D12368CEE700BF02000100704700006A
:1029200070B5044608B9012070BD90F83D3003F041
:10293000FF021BB980F83C20FFF7F0FF242384F846
:102940003D3023681A6822F001021A601A6842F4C6
:1029500000421A601A6822F400421A6002F0FAF883
:102960006368414A93424DD8404A9042DBD922687D
:102970003F495568B0FBF1F125F03F050D43556027
:10298000156A25F03F05013129431162D169364DA1
:1029900021F44F41AB4221F0FF0100F1FF3048D854
:1029A0005B00B0FBF3F0431CC3F30B03042B38BFF5
:1029B00004230B43D361D4E907301168034321F0AA
:1029C000C0010B4313609168D4E9030321F4034170
:1029D000034321F0FF010B439360D4E90530D16834
:1029E000034321F0FF010B43D360136843F001035D
:1029F000136000202023206484F83D30206384F895
:102A00003E0091E71B4A90428DD92268184E5568C6
:102A1000B0FBF6F625F03F0535435560156A4FF4D7
:102A20009671714325F03F054FF47A76B1FBF6F1CC
:102A3000A9E7A56855B903EB4303B0FBF3F0431CCA
:102A4000C3F30B036BB143F40043B2E719256B43A7
:102A5000B0FBF3F0431CC3F30B0313B143F4404347
:102A6000A7E70123A5E700BFA08601007F841E0021
:102A700040420F00FF083D002DE9F7430446994608
:102A80000F4690460C9EFEF799FE94F83D30202BA1
:102A9000054603D0022003B0BDE8F083009019235F
:102AA00001223B492046FFF761FD0028F2D194F84E
:102AB0003C30012BEED0012384F83C3023681A68A7
:102AC000D1075EBF1A6842F001021A601A6822F448
:102AD00000621A60212384F83D30402384F83E30A0
:102AE000002323640A9B6362BDF82C306385638DE9
:102AF0002385284BE362CDE900654B4642463946C3
:102B00002046FFF737FE00282AD00120C3E7FFF751
:102B100007FE40B1236C042B01BF2268136843F405
:102B200000731360F1E7636A27681A4612F8011B05
:102B300039616262628D218D013A92B262857A6951
:102B4000481E80B2520720850AD548B15A783A61AA
:102B500002336362638D013B02399BB22185638539
:102B6000238D2A4631462046002BD0D1FFF77BFD2E
:102B70000028CFD12268136843F400731360202328
:102B800084F83D3084F83C0084F83E0083E700BFC1
:102B9000020010000000FFFF2DE9F043044687B05B
:102BA00099460D469046109FFEF708FE94F83D307A
:102BB000202B064604D00225284607B0BDE8F08346
:102BC0000090192301227B492046FFF7CFFC002803
:102BD000F1D194F83C30012BEDD0012384F83C3046
:102BE00023681A68D2075EBF1A6842F001021A60B1
:102BF0001A6822F400621A60222384F83D304023D0
:102C000084F83E30002323640E9B6362BDF83C30A1
:102C10006385638D2385684BE3622946CDE90076A1
:102C20004B4642462046FFF7FBFD054608B101250D
:102C3000C2E7228D236892B902905A6902929A697A
:102C40000292029A1A6842F400721A60202384F8F1
:102C50003D30002384F83E3084F83C30ACE7012A54
:102C60002CD11A6822F480621A6003905A69039288
:102C70009A690392039A1A6842F400721A60DFF8A4
:102C80003C81238D002BE1D0032B6ED8012B2DD15D
:102C9000324639462046FFF710FD0028C7D1236889
:102CA0001A69636A1A70636A01336362238D013B98
:102CB0002385638D013B9BB26385E2E7022A0ED137
:102CC0001A6822F480621A601A6842F400621A607C
:102CD00004905A6904929B690493049BCFE7059082
:102CE0005A6905929B690593059BC8E7022B0096DC
:102CF0003B464FF000024146204619D1FFF736FC13
:102D0000002894D123681A6842F400721A601A6984
:102D1000636A1A70626A531C6362238D013B2385C8
:102D2000638D013B9BB2638523681B695370BAE7CF
:102D3000FFF71CFC024600287FF479AF236819686E
:102D400021F4806119601969636A1970636A0096D9
:102D500001336362238D013B2385638D013B9BB26D
:102D6000638541463B462046C8E732463946204601
:102D7000FFF7A3FC00287FF45AAF23681A69636A3F
:102D80001A70628D616A013A92B24B1C62852268A8
:102D90006362238D5069013B9BB2400723857FF519
:102DA00070AF032B02BF136823F4806313601369B1
:102DB0004B7078E7020010000000FFFF04000100E4
:102DC0002DE9FF4704469846002302930E46174616
:102DD000DDF83090FEF7F2FC94F83D30202B82466F
:102DE00003D0022004B0BDE8F087574B46F2A8128A
:102DF0001B68B3FBF2F2192353430293029B013B7E
:102E00000293029B4BB92022236384F83D2084F86F
:102E10003E30236C13432364E3E7226893699907E8
:102E2000ECD494F83C30012BDBD0012384F83C3007
:102E300013684649DB075EBF136843F00103136064
:102E4000136823F400631360212384F83D3040238A
:102E500084F83E300025BDF8343025646385638DE9
:102E6000C4F824909BB2E16223856664A764C4F829
:102E70004C802565002B5AD0606B68B33449C16320
:102E80003449C164C0E9105549468564056510326E
:102E9000FFF768F9814600283DD123230093CDF840
:102EA00004A043463A4631462046FFF763FC00B390
:102EB000606BFFF791F9636BC3F83C9023681A6865
:102EC00022F480621A60A4F82A901A68A4F8289064
:102ED00022F001021A600AE0202384F83D3084F8D1
:102EE0003E00236C84F83C0043F0800323640120FF
:102EF00078E7236803905A6903929A690392039AC8
:102F00005A6884F83C0042F480725A605A6842F46D
:102F100000625A6066E7202384F83D3084F83E5012
:102F2000236C84F83C5043F010032364DFE7202235
:102F300084F83D2084F83E30226C84F83C3042F026
:102F400040022264D3E700BF801800200000FFFF8A
:102F5000BD310008793100082DE9F04F044685B0F5
:102F6000984689469246FEF729FC94F83D30202B7E
:102F7000064603D0022005B0BDE8F08F009019236B
:102F800001224B492046FFF7F1FA0028F2D194F8CC
:102F90003C30012BEED0012384F83C302368DFF86D
:102FA00010B11A68D2075EBF1A6842F001021A60B7
:102FB0001A6822F400621A60242384F83D30002548
:102FC0003C4B256409F0FE09E3622268136843F470
:102FD000807313604FF00111434600960022204693
:102FE000FFF7C4FA236838B11B68DB0502D54FF43C
:102FF000007323640320BEE7C3F81090FEF7DEFBE6
:1030000023685A695B690646C2F34002C3F3802312
:10301000A02794F83D10A02901D002B9E3B123689C
:10302000202784F83D705A6912F0020F1A6842F4A2
:1030300000721A6027D0002203925A6903929B699A
:103040000393039B00961923012219492046FFF799
:103050008DFA98B101208EE7FEF7B0FB801B40454A
:1030600002D8B8F1000F01D184F83D7023685A6985
:103070005B69C2F34002C3F38023CAE784F83D7062
:1030800084F83C0077E76FF480625A6159460096F5
:10309000192301222046FFF769FA0028DAD1013509
:1030A000554592D384F83D7084F83C00D2E700BFC8
:1030B000020010000000FFFF704770477047704724
:1030C0007047704790F83D2008B5036DD2B283B9C0
:1030D000C36C0268012B836C05D1DBB21361036DF5
:1030E0000233036508BDC3F307231361036D013386
:1030F000F7E7036D012B03D1836C0268DBB2F4E7C1
:10310000036D022B2FD1222A05D10268136843F4E4
:1031100080731360EAE7438D9BB263B1212A0AD121
:10312000436A026813F8011B11614362438D013B3E
:103130009BB24385D6E7438D9BB2002BD2D1212A87
:10314000D0D10268516821F4E0615160116841F406
:10315000007111602022036380F83D2080F83E302A
:10316000FFF7AFFFBEE703685A69120644BF0022AB
:103170001A61B7E77047704710B5846B636B0BB18A
:103180000022DA63A36B0BB10022DA63FFF7F7F8D2
:10319000022812D02268136823F48063136000238E
:1031A0002022638584F83D2084F83E30236C43F070
:1031B000100323642046FFF7DEFF10BD70B5846B5B
:1031C000236894F83D1094F83E00E26A5D6825F4A7
:1031D00040755D60656BC9B2C0B20DB10026EE638B
:1031E000A56B0DB10026EE6301F02105212D05D060
:1031F00001F02205222D23D1202821D15A6822F462
:1032000000625A6029294FF0000363850DD1212304
:103210002363282384F83D302046FFF74EFF2268C1
:10322000536843F44073536070BD2A29F7D12223B9
:103230002363282384F83D302046FFF73FFFEEE765
:1032400094F83E100029EFD0618D89B2012902BFA8
:10325000196821F480611960596812F5803F21F4E2
:103260004071596006D0082A04D0B2F12A4F01D02B
:10327000202A03D1196841F400711960596821F4BA
:1032800080515960596821F40061596000236385B9
:10329000236C1BB12046FFF76EFFC5E7202184F8A1
:1032A0003D1094F83E1084F83E30402904D1236349
:1032B0002046FFF75FFFB7E7082A01D0202A05D193
:1032C00000232363204638F07DFDADE71223F8E7A5
:1032D0007047000037B50023806B019390F83D20C4
:1032E0002B4BD1B21B6846F2A812B3FBF2F2232398
:1032F000534301930368019A42BB026C42F02002DF
:103300000264456B0DB10022EA63846B0CB10022AC
:10331000E2631A6822F480621A600022428505B1D5
:103320002A6504B122651A6822F001021A6090F839
:103330003D20602A11D1202380F83D30002380F801
:103340003E300364FFF7C4FF03B030BD019A013A79
:1033500001921A689205CED4D3E701F02802282AF8
:103360000ED1196841F001011960196841F48061BA
:1033700019600023036380F83D20FFF7FCFEE3E7BC
:10338000202380F83D30002380F83E30F5E700BF71
:103390008018002090F83D2090F83E100368C9B2D4
:1033A000102910B5D2B2044601D0402905D1222AF5
:1033B00002BF196821F40061196002F02801282970
:1033C0003DD10022226384F83D105A6812F4006255
:1033D0005DD05A68606B22F400625A6090F8353014
:1033E000012B3E4B39D00365FEF7F6FE50B1226843
:1033F000606B136823F001031360202384F83D30D1
:10340000036D9847236C19071FBF2268536823F484
:10341000E063536094F83D30226C5207DBB20DD567
:10342000282B0BD12E4BE36220220023236320465E
:1034300084F83D2084F83E30FFF742FE10BD596805
:1034400011F4006106D1602A1EBF202284F83D20BD
:1034500084F83E1000222263B7E7A06B0365FEF7F5
:10346000BBFE0028CED023685A69510605D51A69DB
:10347000636A1A70636A013363622268A06B13681F
:1034800023F001031360202384F83D30B8E794F85B
:103490003D10602915D1202184F83D1022645A691D
:1034A000520605D51A69636A1A70636A013363624A
:1034B0002268136823F0010313602046FFF708FF1A
:1034C000A0E75A69500605D51A69636A1A70636ADB
:1034D000013363622046FFF74EFE93E7D5320008C2
:1034E0000000FFFF0368F0B55A68C66A90F83E50C6
:1034F00090F83D10EDB2102D8FB00446C9B202D045
:10350000402D40F0CC829F69586910F0010F07D11F
:10351000B6F52A0F02D0B6F12A4F51D10FB0F0BD47
:1035200096054DD5E26AB2F52A0F0CD10122E2626E
:1035300094F83E20402A11D1226D52B9626C02F0FB
:10354000FE021A61EAE7E26AB2F12A4FF0D10822DC
:10355000EDE7626C42F00102D2B2F2E72269B2F505
:10356000804F1AD194F83D20212A626C11D102F0CB
:10357000FE021A61626B0AB1D26B2AB9A26B002AF1
:10358000CCD0D26B002AC9D05A6842F400625A608B
:10359000C4E742F00102D2B2EBE7226D32B9626CAD
:1035A000D21102F0060242F0F002CAE7226D012AAF
:1035B000B4D1626CD21102F0060242F0F102C0E70F
:1035C000060703D5960501D5626CE4E7860740F14E
:1035D000DD80960540F1DA8094F83E10E26A256BB2
:1035E00094F83D002228C9B240F0C880206D40B94F
:1035F000402906D101905A6901929B690193019B70
:103600008CE7216D89B92069B0F5404F0DD1029149
:103610005A6902929A690292029A1A6842F4807276
:103620001A60236D0133236578E7618D89B251B942
:1036300003915A6903929A690392039A1A6842F4B1
:1036400000721A6019E0618D89B2012949D112F521
:10365000803F1BD11A6822F480621A605A6812F403
:1036600000620CD01A6822F480621A600022049270
:103670005A6904929B690493049B0023D3E7059243
:103680005A6905929A690592059AD7E7082A1CD0CB
:10369000202A1AD0122D0DD1012A16D11A6822F42F
:1036A00080621A60002206925A6906929B6906930C
:1036B000069BE2E7102AF1D8934921FA02F2D707D4
:1036C000ECD51A6842F48062EBE71A6822F4806253
:1036D0001A60002207925A6907929A690792079A1C
:1036E000ACE7618D89B202292AD1102A03D8864914
:1036F000D140CE0720D4196821F48061196019687F
:1037000041F40061196059680D050DD512F5803F2F
:1037100006D0511E1F2907D87C4ACA40D00703D5BE
:103720005A6842F480525A60002208925A690892FC
:103730009B690893089BA0E7196841F48061E1E761
:10374000196841F480611960596809050ED512F5B0
:10375000803F07D0013A1F2A08D86C4921FA02F2AB
:10376000D20703D55A6842F480525A600022099267
:103770005A6909929B690993099B7EE700220A9284
:103780005A690A929B690A930A9BC7E67F0740F130
:103790008D805E6836053FF5C1AE0706C0F3800632
:1037A0003ED550053CD5002E3DD194F83D20258DC9
:1037B00094F83E10E06AD2B2C9B2C5B9212A18D134
:1037C000082858D0202856D010F5803F53D05A688A
:1037D00022F4E0625A6011232363002384F83E3010
:1037E000202384F83D302046FFF766FC96E6212A28
:1037F00005D040297FF492AE222A7FF48FAE628DED
:1038000092B21AB95A6822F48062C0E694F83E2057
:10381000402A16D120460FB0BDE8F040FFF752BC59
:10382000002E3FF47BAE97057FF578AE212939D184
:10383000E16A94F83D20212A7FF470AE628D92B245
:103840004AB1626A12F8011B19616262638D013B21
:103850009BB2638562E608290DD020290BD011F5B3
:10386000803F08D0596821F4E06159601123236337
:1038700084F83E20B4E75A6822F4E0625A601A687D
:1038800042F400721A6000232022236384F83D2052
:1038900094F83E2084F83E30402A2046A4D1FFF719
:1038A00010FC3BE6402D7FF439AEB3E759680E05B6
:1038B0003FF534AE4506C0F3800140F18A805005E3
:1038C00040F18780002940F0878094F83D20222A2B
:1038D0007FF424AEE06A628D92B2032A18D91A6985
:1038E000636A1A70636A01336362638D013B9BB242
:1038F0006385638D9BB2032B7FF410AE22685368FF
:1039000023F48063536009E6140001008180008085
:10391000E56A022D3FF476AF012A3FF673AF794A8C
:103920000B91126846F2A811B2FBF1F202EB82028F
:103930000B920B9A013A0B920B99D1B9226C42F07F
:10394000200222645A6822F4E0625A601A69636AAB
:103950001A70636A01336362638D013B9BB26385B6
:10396000202384F83D30204684F83E10FFF703FC06
:10397000D4E51A6812F40072DBD1196821F4806171
:103980001960596821F4E06159601969636A197016
:10399000636A01336362638D013B9BB263852023BD
:1039A00084F83D3094F83E3084F83E20402B04D11A
:1039B00022632046FFF7DEFBB0E5082801D020286F
:1039C00001D1002300E012232363204638F0FAF9E6
:1039D000A4E500293FF4A2AD92057FF59FADE26A10
:1039E000608D616A80B2042809D15A6822F480622D
:1039F0005A601B690B70636A0133636226E7608D4E
:103A000080B203280CD15868042A20F480605860E2
:103A1000EFD0022AEDD01A6822F480621A60E8E73B
:103A2000608D80B20228E4D1012A186801D0102AE2
:103A300027D120F4806018601B690B70616A4B1CF1
:103A40006362638D013B9BB2638523681B694B7086
:103A5000636A216801336362638D013B9BB26385B6
:103A60004B6823F440734B60202384F83D3094F876
:103A70003E30402B4FF0000384F83E300BD12363DF
:103A800097E7042A01D0022A02D140F48060D2E7ED
:103A900040F40070CFE7082A93D0202A90E7006C0A
:103AA00010B35869002587072ED596052CD5226CB2
:103AB00002B19D6994F83D2002F02802282A16D10F
:103AC0005A6822F480625A602F066FEA95014FF01F
:103AD000000301F0010154BFA289228B84F83C301D
:103AE0002046FFF7ECFA19E59D695869DBE70022EB
:103AF0000C9259690C919B690C930C9B84F83C20A7
:103B00000CE500BF80180020C60640F1B180950585
:103B100040F1AE8094F83D505A6822F4E0625A6059
:103B200000220D925A690D921A6842F001021A6041
:103B30000D9A1A6822F480621A605A681005EDB274
:103B400020D505F0F702222A4AD1A06B02685268FC
:103B500092B26285628D92B21AB1226C42F0040276
:103B600022645A6822F400625A60FEF705FC0128BC
:103B700008D0A06B794B0365FEF72EFB10B1A06B4C
:103B8000036D9847638D9BB213B323685A6951073D
:103B900009D51A69636A1A70636A01336362638DB7
:103BA000013B9BB2638523685A69520609D51A699D
:103BB000636A1A70636A01336362638D013B9BB26F
:103BC0006385638D9BB21BB1236C43F004032364B4
:103BD000236C13B320460FB0BDE8F040FFF7DABB0B
:103BE000606B0268526892B26285628D92B21AB1BD
:103BF000226C42F0040222645A6822F400625A6085
:103C0000FEF7BAFB0128BDD0606B544B0365FEF78D
:103C1000E3FA0028B6D0606BB2E72A2D06D1236301
:103C2000282384F83D302046FFF748FA94F83D30C9
:103C3000282B0CD14A4BE362202200232363204629
:103C400084F83D2084F83E30FFF73AFA66E4236BAF
:103C5000222B02D0222D7FF461AC0023202223638B
:103C600084F83D2084F83E302046FFF727FA55E4DB
:103C700001F0F7012129C0F3800535D1070627D5CA
:103C8000560525D53DBB94F83D00628D92B2C0B279
:103C9000002A3FF443AC626A12F8015B1D61626264
:103CA000628D013A92B26285628D92B2002A7FF4EF
:103CB00035AC29287FF432AC5A6822F480625A600D
:103CC00028232163204684F83D30FFF7F6F925E4E8
:103CD000002D3FF423AC95057FF520AC628D92B2A8
:103CE000002A7FF4AEAD19E4400627D5510525D54D
:103CF0003DBB94F83D20618D89B2D2B200293FF4DA
:103D00000DAC1969636A1970636A01336362638D6C
:103D1000013B9BB26385638D9BB2002B7FF4FEABAE
:103D20002A2A7FF4FBAB2268536823F48063536034
:103D300022232363282384F83D3095E7002D3FF4A8
:103D4000EDAB92057FF5EAAB628D92B2002A3FF4AB
:103D5000E5AB1A69636A1A704DE600BFD5320008F8
:103D60000000FFFFF8B503685F695E6890F83E20C9
:103D7000C7F300250446D2B235B1C6F300251DB104
:103D80006FF4807159610125B80506D5F10542BF70
:103D90006FF4007145F002055961780536D5F105DB
:103DA00034D5608D94F83D10D4F830C0202A80B20C
:103DB000C9B25FD100285DD101F0F700212804D0FD
:103DC000282957D1BCF1210F54D194F83D20E16A44
:103DD0000829D2B201D020292AD1282A28D12E4A56
:103DE000E2625A6822F4E0625A606FF480625A61BB
:103DF0001A6822F480621A6000232022236320467E
:103E000084F83D2084F83E30FFF75AF93A053FD553
:103E1000F3053DD523686FF4006245F008055A614B
:103E2000236C1D4325642046BDE8F840FFF7B2BA75
:103E3000212A1BD11849E16222630021202284F843
:103E40003D2084F83E105A6822F4E0625A606FF414
:103E500080625A611A6822F480621A605A691006F8
:103E600048BF19612046FFF728F9CFE76FF4806259
:103E70005A61CBE76FF48061102A596145F004055F
:103E800001D0402AC2D11A6842F400721A60BDE71C
:103E9000002DC5D1F8BD00BF0000FFFFF7B50446F7
:103EA00010B390F89534056803F0FF021BB980F851
:103EB000942428F079FE0323B5F1A04F84F89534BB
:103EC00004BF0023A371206802F0B8FC237C8DF8A6
:103ED0000030251D95E80E00206802F0F0FB014639
:103EE00020B1022384F8953401254CE0206802F0CB
:103EF000ABFC0028F5D1267904F114030127024612
:103F0000C1B28E4203F1240317D8002104F51573C2
:103F10000A46C8B2864203F124031CD8237C8DF8DC
:103F2000003095E80E00206802F00AFD01230546E6
:103F3000E8B1022284F89524D6E723F80A0C03F8A6
:103F4000237C03F8241C03F8202C43E9072243F8C0
:103F5000142C0130D4E703F8232C03F8240C03F8C5
:103F6000202C43E9072243F8142C0131D1E7607477
:103F700084F89534237B012B02D1204600F008FD04
:103F8000206803F010F8284603B0F0BD90F8943490
:103F9000012B10B5044616D00068012384F8943430
:103FA000C3685B0606D5637B012B02BF836B43F4BA
:103FB0008033836302F03CFC206802F0E6FF0020BF
:103FC00084F8940410BD0220FCE790F89424012AA0
:103FD00010B504460AD0012280F894246174006868
:103FE00002F0C3FF002084F8940410BD0220FCE717
:103FF00070B501F00F05044611F0800F05EBC50008
:104000004FEA80004FF0240620D006FB054600F161
:104010001401012021447075C2F30A028A604A78B3
:104020000D700B7102B14D83022B04BF00234B7145
:1040300094F89434012B12D0012384F8943420682E
:1040400002F043FD002084F8940470BD06FB054691
:1040500000F515710020214486F85502DCE70220A6
:10406000F3E710B5044601F00F0000EBC00311F0B8
:10407000800F4FEA83034FF0240215D002FB004269
:1040800003F11401012321445375087094F894340A
:10409000012B12D0012384F89434206802F054FDDF
:1040A000002084F8940410BD02FB004203F5157152
:1040B0000023214482F85532E7E70220F3E738B5C0
:1040C00001F00F05242404FB050104FB050401F5A0
:1040D0001571C4F864320023C4F86022C4F8683251
:1040E00084F8553284F8545283790068012B08BF54
:1040F000C4F870221A4602F0CFFD002038BD2423F8
:1041000001F00F0103FB0101D1F86802704738B5D7
:1041100001F00F05242404FB050104FB0504C4E998
:1041200008230023A3620123637525758379006842
:10413000012B08BF226314311A4602F0ADFD0020A6
:1041400038BD38B5037901F00F05AB4204462DD3D5
:1041500011F0800F4FF024021ED002FB050102FB7C
:104160000503012214334A7501229A701D7094F8D8
:10417000941491421CD084F894241946206802F0CB
:10418000A0FE2DB904F29C42A179206802F05CFFE8
:10419000002084F8940438BD02FB010302FB0101F6
:1041A000002203F5157381F85522DDE70120F2E7BF
:1041B0000220F0E738B5037901F00F02934204467C
:1041C00029D302EBC20311F0800F4FEA83034FF0B3
:1041D000240017D000FB024003F114010123214405
:1041E000437500258D700A7094F89434012B14D017
:1041F000012384F89434206802F08EFE84F89454ED
:10420000284638BD00FB024003F515710023214408
:1042100080F85532E5E70120F3E70220F1E701F0ED
:104220000F0303EBC3030A064FEA83034CBF03F1FA
:10423000140103F515710144006802F0D7BC0000B9
:104240002DE9F04F056889B00446284602F0E8FEE3
:104250000390002840F07281206802F0B2FE00282E
:1042600000F06C8105F50066B3682068C3F30D2388
:10427000C4F8D43402F0A5FE810748BF2268206844
:1042800042BF536903F00203536102F09AFEC20673
:104290002AD52268936923F0100393612F6AC7F32C
:1042A0004343022B07F00F0940F04B8147F6F073B0
:1042B0001F4214D0C7F30A18242707FB09474246B8
:1042C000D7F86012284602F0D7FDD7F86032434491
:1042D000C7F86032D7F868324344C7F868322268BA
:1042E000936943F010039361206802F06AFE0303B0
:1042F00000F13B81206802F064FE47030DD527469C
:104300004FF0000857F8170B02F067FE05F5106A2A
:104310000490049B002B40F00182206802F051FEC3
:10432000002813DA736823F00103736094F8CC3427
:10433000012B40F0AB82002184F8CC14204600F021
:104340003AFB2268536903F000435361206802F08E
:1043500038FE01050AD5B368DA0702D5204628F0F1
:1043600093FC2268536903F400635361206802F0F0
:1043700028FE030114D523685A6902F000625A61CD
:1043800094F8CC24002A40F085825B6D0121C3F3B0
:10439000830384F8CC14C4F8D034204600F00BFB1F
:1043A000206802F00EFEC70433D57368206823F03E
:1043B00001037360102102F077FA207905F510638C
:1043C0004FF67F31039A904200F26882F36943F01E
:1043D0000113F361E37B002B00F07882D6F8843080
:1043E00043F00B03C6F88430736C43F00B03736423
:1043F000D5F80038206823F4FE63C5F8003804F2CD
:104400009C42A17902F020FE2268536903F4805394
:104410005361206802F0D5FD800416D5206802F0B3
:1044200003FE206802F046FBE071276800F08CFB79
:10443000E2790146384602F087F9204628F011FC5F
:104440002268536903F400535361206802F0B9FDF8
:10445000010707D5204628F000FC2268536903F0C5
:1044600008035361206802F0ACFD020600F13982B6
:10447000206802F0A6FDC3020DD505F512680127DC
:104480004FF024092379BB4200F24282226853692B
:1044900003F480135361206802F093FD870230D546
:1044A00094F804C005F5326101234FF0240E9C45B9
:1044B00022D90EFB03470A6897F85882B8F1010F1A
:1044C00040F03A82002A80F23782D4F8D40402F411
:1044D000803200F00100824240F02E8287F857823D
:1044E000AA6942F08002AA616A69100600F124827A
:1044F000736843F4007373602268536903F4001314
:104500005361206802F05DFD410007D5204628F088
:10451000DFFB2268536903F080435361206802F097
:1045200050FD42070AD523685D686B0702D5204617
:1045300028F0D2FB226853682B43536009B0BDE8D2
:10454000F08F062B7FF4CBAE082204F29C41284664
:1045500002F092FC242303FB0949C7F30A17D9F898
:1045600068321F44C9F86872B9E62068DFF8D4B32E
:1045700002F02BFD00278246BAF1000F3FF4BAAEDD
:104580001AF0010F00F08A805FFA87F94946206827
:1045900002F02BFD10F0010F804620D07B0105F5C5
:1045A00030621A440121D4F800E0916094F806C00A
:1045B000DEF840100EF530621344BCF1010F9A682A
:1045C00040F09780100706D5594508D9120406D542
:1045D0004FF4004202E0900664D520229A6018F061
:1045E000080F21D07B0105F530621A440821916043
:1045F0002268116C02F53062134459459A6804D957
:10460000120444BF4FF400429A602046049128F0FF
:104610000DFB0499594507D9A179012904D104F268
:104620009C42206802F010FD18F0100F1FBF05F526
:10463000306303EB471310229A6018F0020F1AD070
:104640006B691B0642BF736843F480637360242365
:1046500003FB074393F85722012A06D1002283F86F
:1046600057224946204628F02BFB05F5306303EB23
:10467000471302229A6018F0200F1FBF05F5306320
:1046800003EB471320229A6018F4005F1FBF05F563
:10469000306303EB47134FF400529A6001374FEA3F
:1046A0005A0A69E712F0280F99D1594501D9120425
:1046B0008ED4242202FB07421969D2F87432C1F366
:1046C00012015B1AC2F8683277B9D4F8642232B9A1
:1046D00004F29C420121704602F0B6FC04E0D4F8DA
:1046E00060221344C4F860324946204628F0A4FAF8
:1046F00075E79348814207D110043FF569AF9106F1
:10470000F2D520229A60EFE7002FEDD1D4F8643281
:10471000002BE9D104F29C423946DCE7049BD80720
:1047200040F189805FFA88FB5946206802F066FCF8
:1047300010F0010F814624D00121736B08F00F02A5
:1047400001FA02F223EA020373630AEB48130A46F2
:104750009960A179914210D1D7F80930D7F8052096
:104760001344C7F80930B8F1000F06D1636A23B9C2
:1047700004F29C42206802F067FC5946204628F06B
:1047800064FA19F0080F1EBF0AEB481308229A605A
:1047900019F0100F1EBF0AEB481310229A6019F08F
:1047A000400F1EBF0AEB481340229A6019F0020F17
:1047B00010D04146284602F077F83B78012B05D10E
:1047C00000233B705946204628F07EFA0AEB481336
:1047D00002229A6019F0800F2DD0D7F81120D7F857
:1047E0000D309A4227D89B1AD7F8052021680591E9
:1047F000934228BF134603339B08069301F51063C9
:1048000003EB48130793079B06989969D7F8112083
:10481000D7F80D3089B2814214D293420BD8059B50
:1048200008F00F01D3F83428012000FA01F122EA40
:104830000102C3F83428049B5B0808F101080493C3
:10484000243766E59342EAD9002BE8D0A3EB0209AE
:10485000D7F805300598994528BF994609F1030313
:104860009B080693A37900935A461FFA89F3D7F859
:10487000091002F0FCF9D7F809304B44C7F80930A9
:10488000D7F811304B44C7F81130BCE7204628F068
:1048900013FA56E5204628F0F7F981E599601A6881
:1048A00022F400121A60C3F80812D3F8002222F48E
:1048B0000012C3F80022D3F8002242F00062C3F8CD
:1048C0000022039A0132039220337BE5736943F49B
:1048D000005343F02B037361336943F00B033361DF
:1048E00086E5AB6923F08003AB6101274FF0240814
:1048F0002379BB427FF6BCAD08FB074393F85732E0
:10490000012B03D1F9B22046FFF789FC0137EFE70D
:1049100009FB0743D8F800101A7E012A08D10029A4
:1049200006DA67F07F01DA75C9B22046FFF777FC37
:10493000013708F12008A5E501332031B7E500BFB4
:104940000A31544F0A30544F006870B51204446A5B
:1049500019B922438262002070BD836A4D1E04EBA8
:10496000134400235E1CDBB29D4205D83F3100EBAF
:10497000810022434260EEE7403300EB83035B6833
:1049800004EB13443346EDE7036800205962704797
:10499000026803460121C0F8D814002083F8CC0433
:1049A000936943F000639361536D43F0805343F088
:1049B0000303536570477047134908B58B6803F0CC
:1049C0000C03042B03D0082B03D0104800E0104840
:1049D00008BD4A684B68496813F4800314BF0C484B
:1049E0000A48C1F3881118BF002302F03F02A1FB5F
:1049F0000001FCF7F9FC044B5B68C3F3014301338E
:104A00005B00B0FBF3F0E3E7003802400024F40061
:104A100040787D012DE9F0410D46044610B9012092
:104A2000BDE8F081434B1A6802F007028A4228D39E
:104A300021688F072DD4C80740D43E4B1A6802F076
:104A40000702AA4265D8226851076BD4130707D51D
:104A5000394A2169936823F4604343EAC1039360B0
:104A6000FFF7AAFF344B354A9B68C3F30313D35CAB
:104A7000D840334B1860334B1868FCF755FE0020C4
:104A8000CEE7CAB21A701B6803F007038B42C6D187
:104A9000CEE7294B11F0040F1EBF9A6842F4E05292
:104AA0009A600E0742BF9A6842F460429A609A6820
:104AB000A06822F0F00202439A60BCE762681E4BD5
:104AC000012A1CD11B6813F4003FA8D01A4EB3680A
:104AD00023F003031343B360FCF770FE41F2883800
:104AE0000746B368626803F00C03B3EB820FA4D0EF
:104AF000FCF764FEC01B4045F3D9032090E7911EEC
:104B000001291B6802D813F0007FDEE713F0020FC3
:104B1000DBE7EAB21A701B6803F00703AB427FF4CD
:104B20007EAF90E70449E0688B6823F4E0530343C9
:104B30008B608BE7003C024000380240904605083D
:104B40008018002004000020014B1868704700BF47
:104B500080180020044B054A9B68C3F38223D35C72
:104B6000034A1068D840704700380240A046050844
:104B700080180020044B054A9B68C3F34233D35C82
:104B8000034A1068D840704700380240A046050824
:104B9000801800200F2303600B4B9A6802F0030279
:104BA00042609A6802F0F00282609A6802F4E05271
:104BB000C2609B68DB0803F4E0530361034B1B688E
:104BC00003F007030B60704700380240003C0240CE
:104BD00002682DE9F34112F0010504460BD08E491D
:104BE0004569D1F88C3023F0C0632B43B5FA85F5C5
:104BF000C1F88C306D0996070BD58748A169D0F8AC
:104C00008C3023F0C0530B430029C0F88C3008BF10
:104C10000125100730D5002301937F4B7F4E1A6C7E
:104C200042F080521A641B6C03F080530193019B85
:104C3000336843F480733360FCF7C0FD0746336884
:104C4000D9055CD5744E336F13F4407360D1E369BA
:104C500003F44072B2F5407F6F4A78D1916823F037
:104C6000704021F4F81120F4407001439160116FFD
:104C7000C3F30B030B43136723685F0742BF684B03
:104C800094F838201A602268D60608D56249606A0E
:104C9000D1F8943023F440030343C1F894309006D4
:104CA0000CD55D48A16AD0F8943023F000630B4323
:104CB000B1F1006FC0F8943008BF0125510608D546
:104CC0005549206AD1F8943023F080530343C1F84A
:104CD0009430012D3FD0802A3DD02068C20500F1DC
:104CE000908010F4007010D04B4A216BD2F88C30B9
:104CF00023F400430B43C2F88C30002005E0FCF79E
:104D00005DFDC01B02289AD9032002B0BDE8F081E6
:104D1000E26902F44072934299D0336F414A012113
:104D2000116023F44073002111603367336FDA0799
:104D30008DD5FCF743FD41F288380746336F9B075A
:104D400085D4FCF73BFDC01B4045F7D9DCE79168F3
:104D500021F4F8118AE7344D2F4E00232B60FCF725
:104D60002DFD074633681B0145D4304B626B1A603A
:104D70002268D70701D563698BB1960701D5A3696E
:104D80006BB1900603D5A36AB3F1006F07D051064B
:104D900012D5236A83B9A36AB3F1006F0CD1D4E9A9
:104DA00002131B0643EA811361680B43216943EA3E
:104DB00001731949C1F8843012060CD5D4E90223D5
:104DC0001B0643EA821362681343226943EA0273B3
:104DD000114AC2F8843001232B60FCF7EFFC0E4D22
:104DE00006462B681B013FF578AFFCF7E7FC801BFC
:104DF0000228F6D988E7FCF7E1FCC01B0228B1D9EC
:104E000082E7054AE16AD2F88C3023F000430B4375
:104E1000C2F88C3065E700BF0038024000700040E7
:104E2000E0114742400E474268004742D8104742CF
:104E300070B5414CFCF7C2FC236843F00103054602
:104E400023602368980757D5236843F080032360C5
:104E5000FCF7B4FC0023A360374C054641F28836CA
:104E6000A36813F00C0F4ED1FCF7A8FC236823F4C1
:104E700050232360304C05462368990349D4FCF73E
:104E80009DFC236823F0807323602B4C0546236828
:104E90009A0144D4FCF792FC236823F080632360DA
:104EA000254C054623681B013FD4244B6360C4F89E
:104EB0008430E368224A23F4F853E360E36823F480
:104EC0000053E360E36843F41F03E360E36843F4E3
:104ED0000013E360636F23F001036367636F43F0C4
:104EE00080736367174B1A60174B1868FCF71CFC3C
:104EF000003018BF012005E0FCF760FC401B0228D1
:104F00009FD9032070BDFCF759FC401BB042A7D9C4
:104F1000F7E7FCF753FC401B6428ADD9F1E7FCF739
:104F20004DFC401B0228B2D9EBE7FCF747FC401BC5
:104F30000228B7D9E5E700BF00380240103000244E
:104F40000024F40080180020040000202DE9F34123
:104F5000044608B901203FE00368DD0710D4236848
:104F600098075AD423681A0700F19C8023685B07CE
:104F700000F1BA80A069002840F01B8100202BE0DE
:104F8000A54B9A6802F00C02042A07D09A6802F036
:104F90000C02082A0AD15B68590207D59E4B1B6890
:104FA0009A03DCD56368002BD9D1D3E763689A4DA7
:104FB000B3F5803F13D12B6843F480332B60FCF7AB
:104FC000FDFB954D06462B689B03C8D4FCF7F6FB0A
:104FD000801B6428F7D9032002B0BDE8F081B3F547
:104FE000A02F04D12B6843F480232B60E3E72A68C9
:104FF00022F480322A602A6822F480222A60002B60
:10500000DDD1FCF7DBFB06462B689F03A7D5FCF739
:10501000D5FB801B6428F7D9DDE77F4B9A6812F037
:105020000C0F07D09A6802F00C02082A11D15B68B5
:105030005E020ED4784B1A68950702D5E268012A01
:1050400088D11A68216922F0F80242EAC1021A6086
:1050500088E7E268714BB2B101221A60FCF7AEFB3F
:105060006D4D06462B68980707D52B68226923F0FB
:10507000F80343EAC2032B6074E7FCF79FFB801B35
:105080000228EFD9A7E71A60FCF798FB624D0646A5
:105090002B6899077FF566AFFCF790FB801B022811
:1050A000F6D998E762695E4B7AB101221A60FCF783
:1050B00085FB594D06466B6F9F073FF557AFFCF7D1
:1050C0007DFB801B0228F6D985E71A60FCF776FB8A
:1050D000514D06466B6F98077FF548AFFCF76EFBA6
:1050E000801B0228F6D976E74B4B1A6C12F08052DF
:1050F00028D101921A6C42F080521A641B6C03F0A2
:1051000080530193019B0126464D2B68D9051BD581
:10511000A368414D012B27D12B6F43F001032B676F
:10512000FCF74CFB3C4D074641F288382B6F9B0740
:1051300039D5002E3FF41EAF374A136C23F080534D
:10514000136417E70026DFE72B6843F480732B60B6
:10515000FCF734FB07462B68DA05D9D4FCF72EFBA5
:10516000C01B0228F7D936E7052B04D12B6F43F07B
:1051700004032B67D0E72A6F22F001022A672A6F07
:1051800022F004022A67002BCAD1FCF717FB41F278
:10519000883807462B6F9807CBD5FCF70FFBC01B51
:1051A0004045F7D917E7FCF709FBC01B4045BDD9BF
:1051B00011E7194DAB6803F00C03082B49D01A4EC8
:1051C00000230228336037D1FCF7F8FA07462B6832
:1051D00099012BD4D4E907321343626A43EA82135C
:1051E000E26A43EA0263226B43EA0273A26A0A4C50
:1051F0005208013A43EA02436B6001233360FCF733
:10520000DDFA054623689A013FF5B8AEFCF7D6FAF9
:10521000401B0228F6D9DEE6003802400000474273
:10522000800E47420070004060004742FCF7C6FA1B
:10523000C01B0228CBD9CEE6FCF7C0FA04462B6887
:105240009B017FF59BAEFCF7B9FA001B0228F6D94B
:10525000C1E601283FF4C0AE6B68E26903F4800147
:1052600091427FF477AE216A03F03F028A427FF4D5
:1052700071AE616A47F6C0721A40B2EB811F7FF4CB
:1052800069AEA26A520803F44031013AB1EB024F11
:105290007FF460AEE16A03F07062B2EB016F7FF4FD
:1052A00059AE226B03F0E043B3EB027F14BF012041
:1052B000002091E60F230360264B1A6852033BD56A
:1052C0004FF4A02242601B6813F0010318BF0123B2
:1052D000C360204B1A68C2F3C40202611A6F5107FF
:1052E00031D5052282605B6F13F0010318BF0123E3
:1052F0004361184B1A68D2014CBF0222012282611D
:105300005A6802F48002C2615A6802F03F020262E7
:105310005A68C2F3881242625A6802F4403202F5B7
:105320008032D20B82625A68C2F30362C2625B6847
:10533000C3F30273036370471A6812F4803218BF14
:105340004FF48032BEE71A6F12F0010218BF01223B
:10535000C8E700BF003802407047000038B5036856
:10536000094ADA600446FCF729FA05462368DB6837
:105370009B0601D5002038BDFCF720FA401BB0F594
:105380007A7FF3D90320F6E75F3F0100F8B50368A1
:10539000DC6814F04004054617D1DA6842F0800258
:1053A000DA60FCF70BFA042706462B68DB685B061D
:1053B00000D40CB12046F8BDFCF700FA801BB0F514
:1053C0007A7F84BF6F770124EFE70024F2E7036858
:1053D000DA6822F0800210B5DA609B689B0604460A
:1053E00001D5002010BDFFF7B9FF0028F9D0042334
:1053F00063770120F6E710B50446002841D0437FCB
:1054000003F0FF0213B90277FFF7A6FF02236377C9
:105410002368DA68D20603D501236377002010BD24
:10542000CA225A6253225A622046FFF7AFFF10BBCE
:10543000236820699A6822F4E00222F040029A6010
:10544000626899680243606902430A439A60E268AD
:105450001A611A69A16842EA01421A612046FFF7FF
:10546000B6FF40B92368A1691A6C22F480221A643D
:105470001A6C0A431A642368FF225A620028CBD0B0
:10548000CDE70120CBE70023092803D840EA031029
:10549000C0B270470A380133C0B2F5E7037F012B71
:1054A0002DE9F04106460F464FF0020041D001239E
:1054B00031683377707738787D78BC788B68002ACC
:1054C00039D113F0400308BFFB70FFF7DCFF8046C3
:1054D0002846FFF7D8FF02462046FFF7D4FFFB78A7
:1054E00040EA835040EA084040EA0224CA234B6263
:1054F00053234B623046FFF749FFA8B9336804F0E5
:105500007F3424F0FE441C609A6822F480229A6062
:10551000D7E90320996802430A439A603046FFF7AF
:1055200056FF08B9012373773368FF225A620023BC
:105530003377BDE8F08113F040034FEA052508BF3B
:10554000FB7045EA00402043FC7840EA8454CDE7F4
:10555000F8B5037F012B06464FF0020037D0012338
:10556000337770770D78C8784C788F786D037ABB75
:10557000E30603D524F010040A344C70FFF783FFD0
:1055800002464878FFF77FFF04463846FFF77BFF67
:10559000284340EA02403368CA225A62532240EA52
:1055A00004245A623046FFF7F1FE58B9336824F0FC
:1055B0007F4424F0C0045C603046FFF708FF08B960
:1055C000012373773368FF225A6200233377F8BDD3
:1055D00045EA00403843DEE7030903EB830300F0AC
:1055E0000F0000EB4300C0B2704738B50368986AFB
:1055F000486018691B6803F07F3323F0FE43C0F353
:105600000E00C3F30625DCB28860C3F305409B0D92
:1056100008704D708C70CB7052B9FFF7DDFF0870C9
:105620002846FFF7D9FF48702046FFF7D5FF88705E
:10563000002038BD38B503685B6823F07F4323F052
:10564000C003180CC3F30425DCB2C3F34233C870A3
:105650004D708C700B7052B9FFF7BEFFC8702846B2
:10566000FFF7BAFF48702046FFF7B6FF88700020AA
:1056700038BD00002DE9F7431E468846174605460B
:10568000FCF79CF80A9C3444241AFCF797F8254B45
:105690001B68C3F3CB33814663432A680193936845
:1056A00038EA03030CBF01230023BB4201D10020D1
:1056B0002EE0731CF3D0FCF781F8A0EB0900A042A8
:1056C00029D32B685A6822F0E0025A606A68B2F562
:1056D000827F0AD1AA68B2F5004F02D0B2F5806F7E
:1056E00003D11A6822F040021A60AA6AB2F5005F7C
:1056F00007D11A6822F400521A601A6842F4005264
:105700001A60012385F85130002385F850300320BA
:1057100003B0BDE8F083019B002B019B08BF002470
:10572000013BBAE780180020F0B585B00B46009227
:105730000E461746022101220446FFF79BFF05464D
:1057400028B1636D43F020036365032515E0124B18
:10575000124A1B68B3FBF2F24FF47A73534303937C
:105760006368B3F5827F0BD10246009733468021F0
:105770002046FFF77FFF0028E3D1284605B0F0BDA3
:10578000039B002BF9D0039B013B039323689B6889
:105790001B06F5D4F1E700BF8018002000366E012B
:1057A00037B50B464168B1F5827F044622D1816846
:1057B000B1F5004F02D0B1F5806F07D12568286898
:1057C000B1F5806F20F04000286009D00092802160
:1057D00000222046FFF74EFF30B9002003B030BD55
:1057E000009201210022F4E7636D43F0200363651A
:1057F0000320F3E7009201210022EBE7704738B560
:10580000044600285AD0436A002B53D14268B2F5AF
:10581000827F00D0C36194F8513003F0FF0223B9B6
:1058200084F850202046FFF7E9FF2168A568A269A7
:10583000A06A022384F851300B6823F040030B6008
:10584000636805F4044503F482732B43E56805F4AB
:1058500000652B43256905F002052B43656905F0BA
:1058600001052B4302F400752B43E56905F038056B
:105870002B43256A05F080052B4300F400552B438C
:105880000B60636A120C03F01003B0F5005F02F0C6
:10589000040242EA030208BFA38D4A6008BF0B61FD
:1058A000CB6923F40063CB6100200123606584F899
:1058B000513038BD0023C0E90433ACE70120F8E7DC
:1058C00038B5044690F85100C0B2012859D10029DA
:1058D00042D0002A40D094F85030012B51D00323FD
:1058E00084F8513000236365A363E286C4E9103372
:1058F000A387E387A368A286B3F5004F84F850001E
:105900002163226807D1136823F0400313601368F2
:1059100043F480431360A36AB3F5005F07D11368B3
:1059200023F400531360136843F400531360A06C16
:10593000154B0364154BC3630025154BC364056504
:10594000E38E0C32FCF70EFC38B1636D84F85050D6
:1059500043F010036365012038BD23681A685206BE
:105960005EBF1A6842F040021A60002284F850209C
:105970005A6842F020025A605A6842F002025A60A5
:10598000EAE70220E8E700BFB55B0008FB5B000820
:10599000D95B000870B5044690F85100C0B20128E8
:1059A00008D06568B5F5827F79D1A568002D76D1DC
:1059B000042874D1002945D0002A43D0002B41D0BF
:1059C00094F8500001286AD0012084F8500094F81F
:1059D0005100A38604281CBF052084F85100002034
:1059E0006065A387E386E387A36A2163B3F5005F5D
:1059F000A263C4E91000216807D10B6823F40053A7
:105A00000B600B6843F400530B6094F85130E06C6A
:105A1000042B0BBF234B244B036403640CBF234BA9
:105A2000234BC3630026234BC3640665E38F0C310D
:105A3000FCF798FB054638B1636D84F8506043F07D
:105A400010036365012029E02268A06C5368216B74
:105A500043F001035360E38EC0E90F55C0E91355CD
:105A60000C32FCF77FFB30B1636D84F8505043F08B
:105A700010036365E6E723681A6852065EBF1A687A
:105A800042F040021A60002284F850205A6842F026
:105A900020025A605A6842F002025A6070BD022029
:105AA000FCE700BFC15B0008CD5B0008655C000837
:105AB000135D0008D95B0008134690F85120012AB5
:105AC00070B504460D4668D182685AB94668B6F585
:105AD000827F07D1042280F85120BDE870400A4639
:105AE000FFF758BF002D42D0002B40D094F8501043
:105AF000012952D0012184F85010042184F851105A
:105B0000B2F5004F4FF000016165C4E91011E38761
:105B1000A186E186A563A387216807D10B6823F0DE
:105B200040030B600B6823F480430B60A36AB3F55A
:105B3000005F07D10B6823F400530B600B6843F43C
:105B400000530B60E06C164B0364164BC3630026D6
:105B5000154BC3640665E38F2A460C31FCF702FB44
:105B600038B1636D84F8506043F010036365012021
:105B700012E023681A6852065EBF1A6842F04002BB
:105B80001A60002284F850205A6842F020025A60BD
:105B90005A6842F001025A6070BD0220FCE700BF63
:105BA000C15B0008655C0008D95B0008704770475E
:105BB0007047704708B5806BFFF7FBFF08BD704763
:105BC00008B5806BFFF7FBFF08BD704708B5806B19
:105BD000FFF7FBFF08BD7047806B026808B553688C
:105BE00023F003035360436D43F010034365012327
:105BF00080F85130FFF7EFFF08BD37B50546846BDD
:105C0000FBF7DCFD2B681B68DB05024626D4236806
:105C1000596821F020015960596821F0020159604A
:105C200020466421FFF780FD18B1636D43F0200327
:105C30006365A36833B901932368DA6801929B68AE
:105C40000193019B0023E386012384F85130636DA7
:105C500023B12046FFF7BFFF03B030BD2046FFF75A
:105C6000A5FFF9E77FB5064600230393846BFBF796
:105C7000A5FD33681B68DA05054646D422685368DB
:105C800023F020035360A36AB3F5005F0FD1012214
:105C90000090642311462046FFF7ECFC18B1636DB9
:105CA00043F0020363652368DB680393039BA268E8
:105CB000236832BB6268B2F5827F22D15A6822F033
:105CC00003025A6064212A462046FFF769FD08B1A5
:105CD000202363650023E3872268012384F8513081
:105CE0009368DB0606D5636D43F0020363654FF6E8
:105CF000EF739360636D43B12046FFF76CFF04B010
:105D000070BD5A6822F00102DBE72046FFF74FFF23
:105D1000F5E77FB5064600230393846BFBF74EFD42
:105D200033681B68D90505463ED42268536823F0C2
:105D300020035360A36AB3F5005F0FD101220090E6
:105D4000642311462046FFF795FC18B1636D43F0BC
:105D5000020363652368DB680393039B2A4664217F
:105D60002046FFF7E1FC18B1636D43F02003636543
:105D700023685A6822F003025A600022E286E28712
:105D8000012284F851209A68D20606D5626D42F04D
:105D9000020262654FF6EF729A60636D23B120468E
:105DA000FFF719FF04B070BD2046FFF701FFF9E7C8
:105DB000036A026A22F00102026270B544688269D5
:105DC0000D6822F073022A438D6823F002032B43EF
:105DD0000E4DA84202D00E4EB04210D1CE6823F034
:105DE00008033343A84223F0040302D0084DA8421D
:105DF00005D1D1E9055624F4407435432C43446061
:105E000082614A684263036270BD00BF00000140C6
:105E100000040140036A026A22F48072026270B5D3
:105E20004468C2690D6822F073022A438D6823F426
:105E3000007343EA0523114DA84203D005F58065A0
:105E4000A84214D1CD6823F4006343EA05230B4D27
:105E5000A84223F4806303D005F58065A84206D1EB
:105E6000D1E9055624F44054354344EA051444600E
:105E7000C2614A68C263036270BD00BF0000014096
:105E8000036A026A22F48052026230B54468C26931
:105E90000D6822F4E64242EA05228D6823F400539D
:105EA00043EA0533084DA84203D005F58065A842B2
:105EB00004D14D6924F4804444EA85144460C261ED
:105EC0004A680264036230BD0000014070477047B9
:105ED00010B5846B626A82420BD1D26901232377A9
:105EE0000AB984F83E30204637F00AF800232377B9
:105EF00010BDA36A834208D1DB6902222277002BFE
:105F0000F1D1012384F83F30EDE7E36A834208D101
:105F1000DB6904222277002BE5D1012384F840308D
:105F2000E1E7236B8342DED1DB6908222277002B75
:105F3000D9D1012384F84130D5E7704710B5846B7F
:105F4000636A834207D1012323772046FFF7F5FFD9
:105F50000023237710BDA36A834201D10223F3E714
:105F6000E36A834201D10423EEE7236B8342ECD141
:105F70000823E9E7704710B5846B636A834209D14F
:105F80000123237784F83E302046FFF7F3FF0023F8
:105F9000237710BDA36A834205D10223237701230F
:105FA00084F83F30F0E7E36A83424FF0010304D105
:105FB0000422227784F84030E6E7226B824203BF56
:105FC0000822227784F8413084F83D30DCE7000075
:105FD000334A0368904212D0B0F1804F0FD0A2F53F
:105FE0007C4290420BD002F58062904207D002F5CD
:105FF0008062904203D002F57842904219D14A68FB
:1060000023F070031343264A904229D0B0F1804F09
:1060100026D0A2F57C42904222D002F580629042C6
:106020001ED002F5806290421AD002F5784290426A
:1060300016D01C4A904213D002F5806290420FD0D5
:1060400002F5806290420BD0A2F59832904207D0C0
:1060500002F58062904203D002F58062904203D143
:10606000CA6823F4407313434A6923F0800313433F
:1060700003608B68C3620B688362094B984203D04C
:1060800003F58063984201D10B69036301234361E7
:106090000369DB0742BF036923F001030361704713
:1060A000000001400040014010B5044630B390F8B4
:1060B0003D3003F0FF021BB980F83C20FFF706FFDC
:1060C000022384F83D302068211DFFF781FF012362
:1060D00084F84630002084F83E3084F83F3084F85D
:1060E000403084F8413084F8423084F8433084F8FA
:1060F000443084F8453084F83D3010BD0120FCE781
:1061000010B5044630B390F83D3003F0FF021BB9E0
:1061100080F83C20FFF7DBFE022384F83D30206846
:10612000211DFFF755FF012384F84630002084F835
:106130003E3084F83F3084F8403084F8413084F8B1
:10614000423084F8433084F8443084F8453084F891
:106150003D3010BD0120FCE7036A026A22F0100204
:10616000026270B5446882690D6822F4E64242EA30
:1061700005228D6823F0200343EA0513104DA84241
:1061800003D005F58065A84214D1CD6823F08003C3
:1061900043EA05130A4DA84223F0400303D005F556
:1061A0008065A84206D1D1E9055624F44064354300
:1061B00044EA8504446082614A688263036270BD78
:1061C0000000014038B590F83C30012B044657D010
:1061D000012380F83C300C2A50D8DFE802F0074F4A
:1061E0004F4F1C4F4F4F2D4F4F4F3E000068FFF752
:1061F000DFFD236809699A6942F008029A619A6989
:1062000022F004029A619A690A439A6100200023ED
:1062100084F83C3038BD0068FFF79EFF23680969A9
:106220009A6942F400629A619A6922F480629A61E2
:106230009A6942EA0122E8E70068FFF7EBFD23686C
:106240000969DA6942F00802DA61DA6922F00402C7
:10625000DA61DA690A43DA61D8E70068FFF710FE0D
:1062600023680969DA6942F40062DA61DA6922F4C2
:106270008062DA61DA6942EA0122ECE70120C6E7CE
:106280000220C7E710B584680A4324F47F4442EA39
:1062900003232343836010BD90F83C30012B70B57D
:1062A00004464FF002001AD084F83D002068012314
:1062B00084F83C30836823F47F4323F077038360C2
:1062C0000B68402B6AD016D8102B0DD008D85BB1C4
:1062D0000120012384F83D30002384F83C3070BD58
:1062E000202B01D0302BF3D1826843F0070322F03A
:1062F0007002134350E0702B2CD01BD8502B35D09C
:10630000602BE5D1036A4D68CE68016A21F0100167
:106310000162826923F0A00322F4704243EA05136C
:1063200042EA063282610362836823F0700343F01D
:10633000670331E0B3F5805F16D0B3F5005FC7D1D6
:10634000CB68D1E90121FFF79DFF2268936843F4F0
:10635000804308E0CB68D1E90121FFF793FF226871
:10636000936843F0770393600020B2E74A68CE68F1
:10637000016A056A25F001050562836921F00A01B9
:1063800023F0F00343EA06130A4383610262836841
:1063900023F0700343F057038360E5E74A68CE6853
:1063A000016A056A25F001050562836921F00A0189
:1063B00023F0F00343EA06130A4383610262836811
:1063C00023F0700343F04703E6E7036A01F01F017F
:1063D00010B501248C4023EA04030362036A8A4057
:1063E0001A43026210BD000070B5044616460D4601
:1063F00029B990F83E00C0B202281CD170BD042912
:1064000007D190F83F00C0B20228F7D094F83F209F
:1064100013E0082907D190F84000C0B20228EDD05F
:1064200094F8402009E090F84100C0B20228E5D07D
:1064300094F8412001E094F83E20511E4A424A411E
:106440000AB90120DAE7002EFBD0002BF9D0022296
:1064500055BB84F83E20606A4A4AC2634A4A0264D5
:106460004A4AC264226831463432FBF77BFE002878
:10647000E7D12268D36843F40073D3602946012230
:106480002068FFF7A2FF2368414A934256D0414952
:106490008B4253D0B3F1804F57D19A6802F0070274
:1064A000062A69D10020A9E7042D14D184F83F20E1
:1064B000A06A344AC263344A0264344AC26422681D
:1064C00031463832FBF74EFE0028BAD12268D36835
:1064D00043F48063D1E7082D14D1E06A84F84020AA
:1064E000284AC263284A0264284AC26422683146A4
:1064F0003C32FBF737FE0028A3D12268D36843F46F
:106500000063BAE7042D84F84120D1D00C2D02D0CD
:10651000002D96D19FE7206B1A4AC2631A4A026483
:106520001A4AC264226831464032FBF71BFE00283B
:1065300087D12268D36843F480539EE7596C934215
:1065400041F400415964A8D0A4E7134A9342A4D06F
:1065500002F580629342A0D002F5806293429CD003
:1065600002F57842934298D002F57052934294D04B
:10657000A2F59432934290D01A6842F001021A6058
:1065800090E700BFD15E00083D5F0008775F00081C
:10659000000001400004014000040040FFF724BF58
:1065A00038B504460D460C2960D8DFE801F0075FD6
:1065B0005F5F3E5F5F5F455F5F5F4C000268406A00
:1065C000D36823F40073D360FBF706FE002229464C
:1065D0002068FFF7FAFE2368254A934203D002F5AC
:1065E000806293420DD1196A41F21112114208D111
:1065F000196A40F24442114202BF5A6C22F400422E
:106600005A64196A41F21112114208D1196A40F212
:106610004442114202BF1A6822F001021A600123AB
:10662000C5B984F83E30002038BD0268806AD3685E
:1066300023F48063D360C7E70268C06AD36823F499
:106640000063D360C0E70268006BD36823F4805313
:10665000D360B9E7042D02D184F83F30E3E7082D79
:106660000CBF84F8403084F84130DCE70120DBE7E0
:1066700000000140FFF794BF82B000230193019B0B
:1066800001330193019BB3F1706F16D80369002B9E
:10669000F5DA00230193036943F001030361019BD1
:1066A00001330193019BB3F1706F06D8036913F0B6
:1066B0000103F4D1184602B070470320FBE784B011
:1066C00038B505AD85E80E009DF81930012B04465C
:1066D00027D1836B23F480338363C36823F484035B
:1066E00023F04003C360C36823F44013C3609DF8E4
:1066F0002030012B02BFC36843F48013C360FFF74F
:10670000BBFF9DF81630012B07D1A36843F00603A9
:10671000A360A36843F02003A360BDE8384004B041
:106720007047C36843F04003C360FFF7A5FF9DF8BF
:106730001D3023B9A36B43F48033A363E1E7A36B5C
:1067400023F48033F9E70000022A58D12E4B2F4A58
:106750000B44934247D92E4B2E4A0B44934244D9C3
:10676000A1F574032C4AA3F5105393423FD9A1F12C
:10677000837302F5C332A3F5E743A032934238D9BD
:10678000264B274A0B44934235D9264B02F59222D9
:106790000B4402F5787293422FD9234B02F5C322A2
:1067A0000B4402F52072934229D9A1F1B77302F587
:1067B000B712A3F5585302F55872934221D91B4BD7
:1067C00002F512220B4402F5F862934294BF0723AC
:1067D0000623C26822F47052C260C26842EA832370
:1067E000C360002070470F23F3E70E23F1E70D236A
:1067F000EFE70C23EDE70B23EBE70A23E9E7092397
:10680000E7E70823E5E700BF405327FFFF340C000C
:10681000401E1BFF3F420F007F4F120060B6E5FE97
:106820005FE3160000D3CEFEC05BB3FEE05459FE1A
:10683000836843F00103836000207047836823F07E
:10684000010383600020704738B5C368012923F035
:10685000C0430546C36010D1C36843F00053C36012
:1068600000240A20FAF7B0FF6B69D90704F10A0483
:1068700015D4C82CF5D1012038BD0029FBD1C3683F
:1068800043F08043C3600C460A20FAF79DFF6B6912
:10689000DA0704F10A0402D5C82CF5D1EBE7A4F11C
:1068A000C80358425841E7E782B000230193019B97
:1068B00001330193019BB3F1706F16D80369002B6C
:1068C000F5DA8901002341F0200101930161019B68
:1068D00001330193019BB3F1706F06D8036913F084
:1068E0002003F4D1184602B070470320FBE782B0C2
:1068F00000230193019B01330193019BB3F1706F5E
:1069000014D80369002BF5DA0023019310230361E7
:10691000019B01330193019BB3F1706F06D80369AA
:1069200013F01003F4D1184602B070470320FBE7C0
:10693000D0F800381943C0F8001800207047000054
:1069400084B02DE9F843044609A880E80E0000232E
:106950009DF824709DF82E60194603F1400204EB67
:10696000820201330F2B5160F7D104F50065002E30
:106970006CD16B6843F002036B60A36B23F40013CC
:10698000A363236843F040032360236843F080033C
:1069900023600023C4F8003E9DF82930012B5CD110
:1069A0009DF82710002956D12046FFF7C1FF10217E
:1069B0002046FFF779FF02462046FFF798FF0028A0
:1069C0004DD1101C18BF012000232B6104F510626B
:1069D0006B611946EB614FF0904C4FF0006E4FF633
:1069E0007F389F423DD8002204F5306311464FF0B6
:1069F000904C4FF0006E4FF67F38974244D82B6989
:106A000023F480732B610023A3616FF080436361E3
:106A10009DF826301BB9A36943F01003A361A26956
:106A2000234B1343A3619DF82A301BB1A36943F0A4
:106A30000803A361012E01BFA36943F0804343F023
:106A40000403A361BDE8F84304B07047A36B43F4AB
:106A50000013A3639DE71946A6E70321A4E70120DD
:106A6000B2E7D2F80090B9F1000F0BDA3BB9C2F8E7
:106A700000E011610133C2F808802032B1E7C2F8AA
:106A800000C0F6E71160F4E7D3F80090B9F1000F09
:106A90000BDA3AB9C3F800E019610132C3F8088093
:106AA0002033AAE7C3F800C0F6E71960F4E700BF97
:106AB00000383C80D0F8083813F0060004D013F0FA
:106AC000020F14BF02200F20704730B50D7801244B
:106AD00005F00F039C404B7800F50062012B00EBA2
:106AE0004510D36918D11C43D461D0F800391A0479
:106AF00010D48B680979D0F80029C3F30A0343F056
:106B0000805343F4004343EA814343EA85531343EC
:106B1000C0F80039002030BD43EA0444D461D0F805
:106B2000003B1B04F6D48B680979D0F8002BC3F323
:106B30000A0343F0805343F4004343EA8143134381
:106B4000C0F8003BE6E7000010B50A784978012953
:106B500000EB421302F00F0100F5006020D1D3F8E2
:106B60000029002A0BDAD3F8002942F00062C3F8AA
:106B70000029D3F8002942F08042C3F800290122FD
:106B8000C46B8A40D2431440C463C1690A40C261E5
:106B9000D3F80019134A0A40C3F80029002010BD99
:106BA000D3F8002B002A0BDAD3F8002B42F0006256
:106BB000C3F8002BD3F8002B42F08042C3F8002B1F
:106BC0004FF48032C46B8A40D2431440C463C1691D
:106BD0000A40C261D3F8001B034A0A40C3F8002BE5
:106BE000DCE700BF007833EC0078F3EF82B00023DD
:106BF0004A7801930B78012A4FEA43131DD100F51F
:106C00001060C118C258002A15DAC25842F000625A
:106C1000C250C25842F08042C25042F21072019BF0
:106C200001330193019B934202D9012002B07047C6
:106C30000B68002BF3DB0020F8E700F53060C1188B
:106C4000C258002AF7DAC25842F00062C250C25855
:106C500042F08042C25042F21072019B0133019314
:106C6000019B9342E1D80B68002BF6DBE3E710B5FC
:106C70009DF808404CB9033300EB02309B0800F547
:106C8000805001EB8303994201D1002010BD51F8DF
:106C9000042B0260F7E700002DE9F3414C7891F8EE
:106CA00000C00B690E79DFF8C8E1DFF8C881012C5C
:106CB00000EB4C1540F08A8005F5106453BB236946
:106CC00003EA0E032361236943F40023236123694C
:106CD00003EA08032361012A0E794CD1CB6903B181
:106CE0006361012E0CD1D0F8083813F4807FD5F8F9
:106CF00000390CBF43F0005343F08053C5F800390E
:106D0000D5F8003943F00443C5F80039002002B03B
:106D1000BDE8F081276907EA08072761276907EAC4
:106D20000E0727618F68BCF1000F0CD1BB422369AD
:106D300088BF0F6143F4002323610B692669C3F305
:106D400012033343C6E73B44013BB3FBF7F3474F22
:106D5000D4F810C007EAC34747EA0C07012E2761A1
:106D6000EBD1266926F0C046266126695B0703F051
:106D7000C0433343E0E7D5F80039012E43F0044324
:106D8000C5F800390B690CD0002BBFD00B78D0F8B8
:106D9000344803F00F02012393402343C0F83438F2
:106DA000B4E7D0F8084814F4807FD5F800490CBF48
:106DB00044F0005444F08054C5F800490C78009227
:106DC0009BB22246C968FFF752FF9FE705F530677F
:106DD0003C6904EA08043C613C6904EA0E043C6135
:106DE0008C68BCF1000F26D103B10C610C623B69C9
:106DF000C4F312041C433C613B6943F400233B6130
:106E0000012A02D1CB6803B17B61012E0CD1D0F8ED
:106E1000083813F4807FD5F8003B0CBF43F00053D3
:106E200043F08053C5F8003BD5F8003B43F00443E2
:106E3000C5F8003B6AE7002BD9D02344013BB3FBE4
:106E4000F4F31FFA83FC04FB0CF4DFF820C0D7F83E
:106E500010E00C620CEAC34343EA0E033B613B695A
:106E6000C4F312041C433C61CAE700BF0000F81FD2
:106E7000FFFF07E00000F8FF70B50023940800F55D
:106E8000805502F00302A34216D301EB84018AB1BC
:106E900000F580500C4605680023D80025FA00F064
:106EA000013304F8010B98B28242F6D1013A92B252
:106EB00001321144084670BD2E6841F82360013349
:106EC000E1E74A780B78012A00EB431012D1D0F8A1
:106ED0000029002A06DB2BB1D0F8003923F08043CB
:106EE000C0F80039D0F8003943F40013C0F8003975
:106EF00000207047D0F8002B002A06DB2BB1D0F819
:106F0000003B23F08043C0F8003BD0F8003B43F443
:106F10000013C0F8003BEBE70B784A7800EB431016
:106F20000B79012AA3F10203DBB20FD1D0F80029BB
:106F3000012B22F40012C0F8002905D8D0F800393E
:106F400043F08053C0F8003900207047D0F8002B80
:106F500022F40012012BC0F8002B9EBFD0F8003B9A
:106F600043F08053C0F8003BEEE7D0F8003823F43C
:106F7000FE63C0F80038D0F80038090101F4FE6162
:106F80001943C0F8001800207047D0F8003E23F0E5
:106F90000303C0F8003ED0F8043823F00203C0F821
:106FA000043800207047D0F8003E23F00303C0F8F7
:106FB000003ED0F8043843F00203C0F80438002043
:106FC00070474269806910407047D0F8183800F562
:106FD0000060C0691840000C7047D0F8183800F500
:106FE0000060C069184080B2704700EB411100F5A5
:106FF0000060D1F8082B40691040704710B5D0F8F8
:107000001048D0F8343800EB411001F00F01CB40AC
:1070100000F51060DB018068DBB22343184010BD2F
:10702000406900F001007047D0F8003923F4FF6395
:1070300023F00703C0F80039D0F8043843F4807314
:10704000C0F804380020704730B5056C104CA542DC
:1070500000F5306303D9D0F8004B002C16DB002478
:107060001C611C6944F400241C611C6944F0180470
:107070001C611C69012944F0C0441C6101BF5A61B4
:10708000D0F8003B43F08023C0F8003B002030BD27
:107090000A30544FF8B51D4B1D4D1B6898471D4BCA
:1070A00028801B7853BB1C4F1C4B3A7893F8443113
:1070B0000AB183F040031A4E1A483278C3F38013A2
:1070C00063F38202436A3270984700214FF0010453
:1070D000FAF7ACF808B14FF000043278C2F380033D
:1070E0006340DBB263F3000232703A7842B12A782F
:1070F000C2F300010B4063F300022A702888F8BD38
:107100002A78C2F300010B43F5E700BFFC1D002005
:1071100008000020091E0020081E0020489D0020B5
:107120000A000020101E0020094A137803F0FE0315
:1071300061F3C30310B51370064B1870064B1B6840
:107140002BB1064C0122227098470023237010BDFA
:107150000A000020081E0020F81D0020091E002043
:1071600082B00B4B10B100229A70DA7018680023BD
:10717000C2B262F30703C0F3072262F30F23C0F326
:10718000074262F3174363F3170002B0704700BF72
:107190000A1E002008B5054B1B689847044B5B8806
:1071A000003318BF012363F3082008BDF41D00203D
:1071B0000A1E002070B50C4CB4F8A63113B1D4F8F7
:1071C00090317BB970BDA8B2D4F8903100219847B6
:1071D0000135B4F8A6319D42F5D3D4F89831BDE815
:1071E000704018470025F4E7F0990020012810B5F9
:1071F000044610D10C48436A98470021FAF716F864
:1072000008B14FF00004094B93F84401C0F380101B
:107210006040C0B210BD064B1B681BB1984700F020
:107220000100F7E71846FAE7101E0020489D0020ED
:10723000001E0020F8B5184B1B6807469847064605
:1072400000B3164C00256566A4F8145200F02EFA1F
:1072500097F8BE212346BAB1114A1278A2B194F828
:107260000D32104843F001031922294684F80D32EB
:1072700005F012FA0C4BC4F8B0300C4BE26E1A60F9
:107280000B4BE3663046F8BD93F80D226FF3000216
:1072900083F80D22F6E700BFC41D0020F0990020FE
:1072A000C81D0020DD72000861710008F41D002077
:1072B00095710008064B10B51B68044698472CB919
:1072C00004490548BDE8104011F030BF10BD00BFB3
:1072D000041E00203D750408427504082DE9F0479E
:1072E000304F314C97F8BE314FF0000884F80280DF
:1072F00084F80380002B52D0414619222B4805F018
:10730000CBF92B4897F8BE61057897F8BF714146D5
:107310004FF0010CA94212D36388002B3FD017F025
:10732000FBFE40F20113184239D1224B1B689847EB
:10733000214B40F480701B6FBDE8F047184700EB0D
:10734000C102137926FA03FE1EF0010F25D0D2F8F0
:1073500008E027FA03F89EF809209EF80A9008F042
:10736000010868F382028EF80920DEF8102002F18D
:1073700004721032520112F8292042450DD09EF8B5
:107380000020172A8CBFE278A2780CFA03F3DBB254
:107390008BBF13431343E370A3700131BAE7BDE819
:1073A000F08700BF489D00200A1E0020DD72000803
:1073B000C81D0020F41D0020F099002010B50B4BD3
:1073C0001A78D40019190132886001781A70A1F175
:1073D0000F02D2B2072A05D9A1F11802D2B2032AAC
:1073E00028BF002223441A7110BD00BFC81D002011
:1073F00070B5304C94F80F3288B06FF3861384F870
:107400000F3200220323012101A88DF8033007F079
:107410008BF80379002B47D00023079D1A460DF106
:10742000030101A8A847054600283DD000221D21E0
:1074300006F0DCFE2B46204D03F130061868596833
:107440002A4603C20833B3421546F7D11B4BD4F882
:107450001C211A601A4BC4F81C311A4BD4F818219D
:107460001A60194BC4F81831184BD4F820211A604F
:10747000174BC4F82031174B174A996E1160174A01
:107480009A6694F8073243F0020384F80732002129
:10749000134805F097FA134BA26B1A60124BA363C3
:1074A00022F012FC08B070BD1049114805F08AFAAC
:1074B000EDE700BFF0990020101E0020FC1D002009
:1074C00095700008F81D002029710008001E00209A
:1074D000ED7100080C9C0020041E0020B57200080D
:1074E000B5710008C41D0020357200080475040839
:1074F00027910108004870470C000020014B1878C4
:10750000704700BF401E0020F8B50F4FBB6FC5B2DB
:1075100006460C469847C0B2A84214D07B6F30464E
:1075200098475DB154B1094B20469D78F9F792FC1C
:107530000749F9F79BFD29460DF0EAFD2020BDE83B
:10754000F84013F085BAF8BDF0990020409900206A
:1075500000007A4438B50F4B1A780546C2B95C78FA
:10756000B4B90D4B5B6F984715F0FF0F0BD00B4B69
:10757000B3F8C80038B1F9F76DFC0949F9F776FDA1
:1075800021460DF0C5FD2020BDE8384013F060BA5B
:1075900038BD00BF40990020F0990020489D002090
:1075A00000007A4438B5054617F0B6FD022808D029
:1075B0000FF056FF044610B12846FFF7CBFF2046D8
:1075C00038BD0124FBE730B501444FF6FF734AF2A2
:1075D0000104884201D1184630BD10F8012B5340F8
:1075E000082203F001055B080DB163409BB2013A2C
:1075F000F7D1EEE701440023814201D118467047DC
:1076000010F8012B82EA132282EA121242EA0323C3
:1076100083EA023383EA42139BB2EDE70346272B4A
:107620004FF0000018D8242B3AD2182B11D00AD8CA
:10763000102B35D002D80F2B0BD07047112B32D026
:10764000122B2AD070471A2B2DD029D31F3B032B86
:107650002BD84FF001007047852BFAD00AD8302B79
:1076600005D82E2B19D2293B032B1CD97047842B0C
:107670000DD07047882B10D004D8862B10D0872BC4
:1076800011D070478E2B05D08F2B06D070474FF04E
:107690000F0070474FF0030070474FF0080070472D
:1076A0004FF0020070474FF0040070470F4890F809
:1076B000143210B5CBB90E4B90F8112293F8B431B7
:1076C0000C49DB43DBB21A4002F00F04D24302F054
:1076D0000F020A7090F813224C70134003F00F024F
:1076E000DB4303F00F03CA708B7010BDF0990020CC
:1076F000489D0020411E0020094B18680023C2B29B
:1077000062F30703C0F3072262F30F23C0F30742BB
:1077100062F3174382B063F3170002B0704700BFF3
:10772000411E002037B50D4D0D4995F814520A78C9
:107730004B788C78C978C0B22DB922430B430240F4
:10774000034001400440002062F3070063F30F2070
:1077500064F3174061F31F6003B030BDF09900205F
:10776000411E002010B50C49BE22013AD30011F889
:10777000324084420BD10B445B681AB1002BF4D029
:10778000184610BD054A002B08BF1346F8E7002A2B
:10779000EBD1024BF4E700BF147C040845CD04088C
:1077A0001FB5A0F11104032C9FBF074B0FCB0DF1A8
:1077B000100C0CE90F009BBF634603EB8404002010
:1077C00054F8100C04B010BD087404080D289DBFB7
:1077D000012303FA00F080B20020704770B5C0F3B7
:1077E000072303F03803082B8AB0064612D10A4D4E
:1077F0000FCD6C460FC40FCD0FC495E80300C6F340
:10780000834684E803000AAB03EB860656F8280C8F
:107810000AB070BD0148FBE718740408FC1C050899
:10782000014B1878704700BF451E0020024B1A68B4
:1078300018609060704700BF240000200048704727
:1078400018000020044B1B6823B11A88824201D023
:10785000DB68F9E718467047441F0020074B9A6918
:10786000074B2AB1C3F8F800064B00221A60704794
:10787000D3F8F83042695A61F6E700BF0C9C00204B
:10788000409800209C1F00202DE9F04F3D4D93466D
:1078900000F0FD021C46012A4FF0FF3385B0C5F809
:1078A0009830E87116D1384B0846DB69984747682D
:1078B000EB7900930026E3B2019303244FF0010912
:1078C0004FF00008B246009B032B16D8DFE803F008
:1078D00004234D340027EBE705EB84024B46106C84
:1078E000039341460292F9F7A1FCDDE9022300B1BE
:1078F00053461E43F6B2C2F8408014F1FF34E2D280
:10790000002E3BD04FF4806013F0A2F805B0BDE824
:10791000F04F1AF099BD57F8242005EB8403186C3A
:10792000039211460293F9F781FC0028E5D1DDE9C5
:10793000023201261A64E0E757F8242002924B46EF
:10794000104641460393F9F771FCDDE9022300B1CB
:1079500053461E4305EB84031146186C0293F9F756
:10796000C9F9029BF6B21864C7E7019BE340DB0745
:10797000C3D505EB84035BF82420D0E705B0BDE850
:10798000F08F00BF409800200C9C002010B4084CE1
:1079900094F8A330013303F0030384F8A33004EB1D
:1079A00003140FC8A43484E80F0010BC1AF04CBDB7
:1079B000409800202DE9F0470124DFF83C908046F4
:1079C00017464D080026A24615B93046BDE8F08797
:1079D000EB0709D514F8093033B10AFA04F216435B
:1079E00058F803101FB1F95001346D08ECE7A0B24C
:1079F0000CF0D2FBF8E700BF589A040870B50446B3
:107A00000D460E48002116460CF0E2FD00210C4800
:107A10000CF0DEFD0B4B2046D3F8283132462946C8
:107A20009847FE28044606D00DF056F9FF2C08BFF3
:107A30002724204670BD0024FBE700BF3C9A0408C1
:107A4000439A04080C9C00202DE9F04101F1200824
:107A500000F1200704460E460C223946404636F017
:107A60009DFF654BDB6AA3B194F8302096F8303067
:107A700002F0010203F001039A4240F0BB80E36A86
:107A80005B68DA68336E9A4240F0B480031C18BF1A
:107A900001235A4D2B7140B1D8F80000D8F80410DA
:107AA0003B4603C3D8F808001860B379A2799A421C
:107AB0002A781ABFA3710121002161F382022A7082
:107AC00033792279297882EA03009A4260F3C3016C
:107AD00018BF2371A278B37829709A422A781ABF06
:107AE000A3700121002161F34512F3782A70E27836
:107AF00029789A4282EA030018BFE370E279F379A9
:107B000060F386119A426A78297014BF012100211E
:107B100061F3000206F1400704F140086A7018BFE3
:107B2000E37110224146384636F038FF78B16B7861
:107B300043F001036B7042463B4606F1500C186857
:107B40005968174603C7083363453A46F7D194F896
:107B5000322096F83230307A9A426A781ABF84F826
:107B600032300121002161F34102237A6A7083429D
:107B70006B7814BF0122002262F3C3036B7004D040
:107B8000207204F10C0115F0ADF996F8213094F84B
:107B900021209A426A781ABF84F8213001210021FD
:107BA00061F3451273796A70627969789A4282EA60
:107BB000030018BF6371627F737F60F386119A427E
:107BC000AA78697014BF0121002161F30412AA7020
:107BD00018BF6377228E338E9A42AA781ABF238603
:107BE0000121002161F34512AA701CBF044AD3830E
:107BF000BDE8F08101234CE740980020481E00209A
:107C000040990020F8B5154B9A6906460D468AB191
:107C1000DB69984704465DB1006848B1F8F702FB9C
:107C2000013036F099FE286010B1216838F08DFCE3
:107C30006068F8BD0A4B0B4AD3F8F830154603F1DB
:107C4000100718685968144603C40833BB4222461B
:107C5000F7D1186820606E610248EAE70C9C0020AA
:107C600040980020D01F002008B50C2036F074FE8C
:107C7000034638B1084A07CA83E8070007490A687B
:107C80002AB90B60181C18BF012008BD0A4691686C
:107C90000029FBD19360F5E72C1F0020981F0020DE
:107CA000363038B50F49C4B20F4838F04EFC3B2C83
:107CB0000546204628BF3B200DF0A8F8014628467F
:107CC00038F027FC3B2C0BD90849074838F021FC39
:107CD000A4F13B000DF09AF80146034838F019FC76
:107CE000014838BDB0880408501E0020E2EB0408AB
:107CF0000048704738000020F8B50025094E2C4692
:107D00004FF07E57731964003946D869E4B2F9F729
:107D10008DFA08B944F00104043D15F1100FF1D1BA
:107D20002046F8BD2800002010B5FFF7E5FF0E4BF8
:107D30004FF07E510022DA609A605A601A60D96171
:107D4000996159611961094B0022C4B283F833204B
:107D5000FFF7D2FFC0B2A04204D00220BDE810401D
:107D600012F076BE10BD00BF280000204098002011
:107D7000F0B585B06D46064610220021284636F043
:107D800040FE0B2E13D1144B144C93F84171002379
:107D900084F8E43095E80F00E83484E80F00BA076F
:107DA00003D42946304615F071F805B0F0BDB21F76
:107DB000D3B2022B05D8084B93F84831D340DB07E8
:107DC000F3D40648037AB342EBD1102200210C30E1
:107DD00036F017FEE5E700BF489D002040980020E0
:107DE000F8B50446124D861C00F11007D1B1114BB5
:107DF000B3F83C2140F20113934313D018F026FE50
:107E000000280FDB04EB800405EB840405EB8606F9
:107E1000D4F8A4107068F8F76DFF55F82710F8F73C
:107E200069FFF8BD3A3405EB860655F82410F1E7F2
:107E300040980020489D00202DE9F04F0F4685B066
:107E400006462E4D28B1022835D0E87105B0BDE8B0
:107E5000F08F2B4B9B690193D5F8F83005F1500951
:107E6000044604274FF0010B4FF0000A024651462A
:107E700059F8040DCDE90232F9F7D8F9013FD84697
:107E8000DDE9023200B190460199C9F800A044EA48
:107E90000804E4B209B943F827A0002FE7D1EE7136
:107EA000002CD3D04FF4806012F0D2FD05B0BDE8B5
:107EB000F04F1AF0C9BA1046F8F7D0FF114A242340
:107EC00003FB072307F11009196BF9F7CFF8804678
:107ED000014655F829004FF00104F9F7A7F908B158
:107EE0004FF00004064B45F829809B69E4B2002B53
:107EF000D5D1D5F8F83043F82780D0E74098002056
:107F00000C9C0020489D0020022331B1012909D09A
:107F1000012243700270002302E0012201704270CE
:107F200083707047037000234370817070470000B6
:107F3000F8B50646002848D0264F3D78002D44D19C
:107F40007B78002B3FD1244C244D01462046FFF77F
:107F50007BFD336DA367338EFB83AB78980603D527
:107F6000D6E916010EF020FAAB78D90605D51C4BE0
:107F7000607FB3F8C810FFF7C7FA6B781A0705D50A
:107F80004FF4007012F064FD1AF05EFA6B785B0635
:107F900002D5082012F05CFD2D79C5B194F830109F
:107FA000E06A01F0010116F00DFC18B9316EE06ACB
:107FB00016F066FB0A4BA26AB3F8D03094F8201092
:107FC000E06A16F03FFD2846F8BD0025FBE70125D5
:107FD000F9E700BF4099002040980020481E00208B
:107FE000489D002008B5FFF72DFC20B143688B4267
:107FF0000CBF8068002008BD0048704760980020D2
:1080000008B5064B0020C3E90000986016F046FD55
:108010001020BDE8084012F01BBD00BF6098002092
:1080200008B5054B5877054B5B6F98472020BDE896
:10803000084012F00DBD00BF40980020F0990020CC
:108040000D4B186810B508B1FFF708FC0B4CD4F8BD
:108050009810002905DD4FF0000300220120FFF7F2
:1080600013FC074BD4F8F800D3F8DC309847802095
:10807000BDE8104012F0ECBC9C1F0020409800208E
:108080000C9C002010B500B910BD846836F06CFC63
:108090002046F8E7104B70B50022104C1A604FF0E4
:1080A000FF33C4F898300E4B0E4D1868FFF7EAFF07
:1080B0002B6833B12868C66836F056FC2E60002E57
:1080C000F8D1D4F8FC0000B970BD856F36F04CFCD7
:1080D000C4F8FC50F5E700BF9C1F0020409800202A
:1080E000981F0020441F002010B5044618B1FE2838
:1080F00001D0FFF7CFFF204610BD00002DE9F04F63
:108100005E4B5F4C93F88E905E4F8BB0984601901B
:10811000B9F1000F64D05C4D00214FF4807220460D
:1081200036F06FFC95F84231D90606D5FB69D5F8D3
:10813000C40198474368C4F8F830D4F8F80020B96F
:10814000FB6998474368C4F8F830B96969B91822DF
:10815000D4F8F80036F055FC95F84231DA0604D52B
:10816000D4F8F830D5F8C4215A61FFF793FF474D92
:10817000B8F81E3023860020656716F081F9E062AA
:10818000FFF7D2FDA5F11401207A14F0ABFE10B96F
:10819000BB680720984798F88E3073B13A4B93F834
:1081A00041319B0709D43A4D0B20294614F09AFE21
:1081B00000283CD1BB68072098473C6D24B198F853
:1081C0008E30002B3DD1A0470AF0E2FF0CF006FEF6
:1081D0003B6B002B4ED02A480BB0BDE8F04F184740
:1081E00004F1400595E80F0006AE86E80F00E8228E
:1081F0004946204694F808A094F807B036F001FCF0
:1082000096E80F0085E80F00D4F8F8004369C4F839
:108210009430204BD3F830310BB149469847019B3D
:10822000002BA2D084F808A084F807B09DE795E859
:108230000F0094F9A34005EB0414443C84E80F00BC
:10824000BBE71022002102A836F0DBFB02A91022B6
:10825000114836F0A3FB01460028B4D1102206A82D
:1082600036F0CFFB102206A9094836F097FB00280C
:10827000A9D1A9E70BB0BDE8F08F00BF409900205D
:10828000409800200C9C0020489D00206098002011
:1082900028990020F09900204C98002070B50669BC
:1082A000F56B03460C461DB9FFF7F4FE142070BDB4
:1082B000027D6FF345120275194AD1671960194999
:1082C00000228260CA8B120A42F0400242760120EC
:1082D00088771876CA7F0243CA775A7E02435A7655
:1082E00073686422DA60A84701682046F8F70AFE3E
:1082F00000210446F8F79AFF18B1FFF7CBFE2920BA
:10830000D5E7094B0949D86FF8F7FCFD2146F8F786
:1083100097FF0028CBD0FFF7BDFE2B20C7E700BF9B
:108320004098002040990020489D00206666663FE6
:1083300010B5044678B1084BD3F8D03003B1984754
:1083400023781BB10021204610F094FE2046BDE8A2
:10835000104036F009BB10BD0C9C00202DE9F74FF2
:108360008946164603785A1E1F2A044600F101006A
:10837000F8D93B2B05D02F2B0AD1414B1B89DA06AC
:1083800005D500232370204603B0BDE8F08F0446D6
:10839000DFF8F8B0DFF8F880274625464FF0000AEE
:1083A0002A780AB93A70EEE7202A07D9292A0DD08F
:1083B0003B2A05D0282A55D105F1010A0135EFE7FE
:1083C000BAF1000FFAD185F800A0E9E7BAF1000F81
:1083D000F4D02C4B93F8A120002A3ED1019216F044
:1083E0009BFE0228019A49D02A709BF806221307A7
:1083F00026D42EB332681ABBD8F8CC2012B150461E
:10840000904730603268DAB904221F49504638F08C
:10841000A4F8A8B9A5EB0A02033A1046019236F077
:108420009BFA306060B1019A0AF104018A46013179
:108430009AF800C0BCF1200F12D0514636F0BDFAB8
:108440009AF80020D2B10EB1326832B9D8F8D420EF
:10845000A2B15046904789F800004FF0000AADE7FE
:10846000013AE3E7BAF1000FA8D1A2F1610119299D
:1084700098BF02F05F023A7001379FE792469DE78E
:108480004099002040980020289A0408F099002084
:108490000C9C00202DE9F04F934AB7B000231893AD
:1084A0008DF85B3092F89D10904B9046D3F80831D0
:1084B000A9B1B3FA83F4640924B1003318BF0123CE
:1084C00088F89D3018AA0DF15B01FFF747FF9DF872
:1084D0005BA00746BAF1000F05D05046C3E01C1C54
:1084E00018BF0124E8E70378252B19D14378002B26
:1084F00045D180F800A098F89D30002B38D0DCB929
:1085000098F89C30C3B939238DF85B309DF85B3007
:1085100033B9774BD3F8F83013B198F89C009847EB
:108520003B7863BB189808B1FFF702FF9DF85BA08A
:10853000504637B0BDE8F08F88F89C40002CE5D15C
:108540006B4D0EF08DFFEB6808209847AB6D002B4C
:10855000DCD016F0E1FD0446023841424141AB6DEA
:10856000FF209847023C18BF012488F89D40CDE7C2
:1085700098F89C3083F0010388F89C30C6E75D4C86
:10858000594EEC220021204636F03BFA0FCE04F182
:1085900008050FC50FCE0FC50FCE0FC596E80F000B
:1085A00085E80F00D8F874300493002308938DF801
:1085B00018309B46BDF82030ADF814303B78242BA2
:1085C00006D10123ADF8143023819DF82030A37229
:1085D000BDF81430002513F0010FCDE91B550CBF79
:1085E0002B46032319932E462C460B950795099588
:1085F000199A531C199317F80280B8F1000F19D17A
:108600001BF4004F384C3B4D00F0728795F8E86042
:10861000002E00F0DA86D4F8FC30002B40F0D5862E
:1086200095F8D230DB0700F1BA86FFF733FD4FF043
:108630001C0A7DE7B8F1230F60D12B4A92F8A120E4
:10864000002A7FF475AFFB5C3C2B2CAA19A9384695
:108650001BD109F0B7FE30B9199B5A1C1992FB5C6B
:108660003D2B04D00220FFF73FFD824660E71AAAA7
:1086700019A938460AF01EF80028F4D11A992CA836
:108680000BF0A6FF0028B3D1ECE70AF013F800289E
:10869000E9D12C98F8F738FE80B20BF06BFD08B3E7
:1086A000199B5A1C1992FB5C3D2BDBD11AAA19A904
:1086B000384609F0FFFF0028D5D1099B092B00F2AD
:1086C0009C802C98DFF83080F8F71EFE099B28F874
:1086D000330008EBC3081A9BC8F80430099B013328
:1086E000099385E72720BEE740980020F0990020F5
:1086F0000C9C0020581E0020481F0020B8F14F0F8E
:108700001DD1DFF8F89199F8D1206FF3861289F81E
:10871000D120FB5C5B2B27D12CAA19A938460AF083
:108720009FFA00289FD199F8D13043F0800389F84F
:10873000D1302C9BC9F8C830199B013319936F486D
:108740006F4AD0F8D030126813422AD0934328D110
:10875000199BD0F8C80036AA013B42F8743D39464F
:10876000684B0AF081FD7EE73C2BE8D12CAA19A9C1
:10877000384609F027FE00287FF475AF99F8D1300C
:1087800043F0800389F8D1302CA80CF0FDF9C9F82A
:10879000C80000287FF42CAFFFF77CFC4FF0530A91
:1087A000C6E6B8F1400F07D8B8F1240F07D0FFF79D
:1087B00071FC4FF0010ABBE6B8F15A0FF7D8022D51
:1087C00020D1199BFB5C2BB1A3F14102192A01D9DD
:1087D000242B17D14C4B1A934C4B93F8A1301BB15F
:1087E000B8F14F0F7FF4A4AEDDF86890022D494632
:1087F00048460FD0F8F74CFD78B1FFF74BFC4FF02F
:10880000020A95E61AAA19A9384609F053FF00286A
:10881000E2D028E7F8F73CFD88B94846F8F774FD40
:108820000446F8F717FB01464846F8F761FA38495D
:10883000F8F768FB3CF024FCF8F766FD0646DFF825
:10884000CC90D9F8FC308BB11A78A62A0ED15B688F
:108850000A930CF0B1FA0A9B834207D1D9F8FC3095
:108860001A78264B4BF4004B83F8E820B8F1470FF9
:1088700050D0B8F14D0F00F086820023A8F12408F3
:108880001B93B8F1360F00F2FC81DFE818F0720597
:10889000FA01FA01FA01FA01FA01FA01FA01FA0100
:1088A000FA01FA01FA01FA01FA01FA01FA01FA01F0
:1088B000FA01FA01FA01FA01FA01FA01FA01FA01E0
:1088C000FA01FA01FA01FA01040432043D044804F1
:1088D00052045C04FA01660470047E048C049A0459
:1088E000FA01AF04BC04DD04E804F304FE04090546
:1088F0001405290534053F0550056105581E002063
:10890000549A0408E19800200000C07F409800209D
:108910000000C84200231C93632C00F2B281DFE800
:1089200014F0D900D900D900D9008400D900B001D1
:1089300064006400B0017A00B001B001B001B00180
:10894000B001B0011301130113014D014D01B0013C
:10895000B001B001B001B001B0017A00B0017A00FD
:10896000B001B001AD00B001B001B001B001C20072
:10897000B0015C01B001B0016301B001B001B00110
:10898000B001B00163011F021F02B00184008A011F
:108990008A018A018A018A018A01B001A701B00116
:1089A000B001B001C301C301EA01B001B001B001DF
:1089B000B001B001F600B001B001AD00B001B001EE
:1089C000B001DE00F600F600F600F600F600F60054
:1089D000B001B001F6001E011E017A003801380115
:1089E00043010102010213021302A84B1B7E022B5A
:1089F00040F047819DF87130E11F43F040038DF84E
:108A000071304A42A24B4A415A730EB3FFF742FB00
:108A10004FF0170A8CE546B9079B23B1FFF73AFBE5
:108A20004FF0180A84E5012307939DF87030984AA7
:108A300043F0010324F002018DF870301C29E3B2E9
:108A400013700FD116B10A2E40F01B811E44167010
:108A50001C9B1BEA030500F09281FFF71BFB4FF004
:108A6000150A65E55C2CD0D11E2E00F20A81894BD7
:108A7000F340DB0740F105815C36E8E7002E40F06B
:108A80000081079B002BC9D19DF870309DF81C20F8
:108A900043F002038DF870307D4B1C8183F83C203D
:108AA00002230793D4E77C4BD3F81C31002B00F052
:108AB000E880A6F114021E2A00F2E380754BD34031
:108AC000DB4313F0010340F0DC800A24B6FBF4F42E
:108AD0001E468A34079B002BA0D1022307939DF8E2
:108AE0007030052C43F002038DF870300CD15EB16C
:108AF0000A2E40F0C680664B33221A810026644B52
:108B0000002283F83C2080E7614B1C81F7E7079B3C
:108B1000002B83D19DF8703043F002038DF8703044
:108B20005B4B012283F83C20A2B21A815B4B1B886D
:108B30009B1ABDF8142018BF012363F34102ADF85E
:108B400014200223079360E79DF87030504A43F0E9
:108B500004038DF87030A4F11103937355E79DF869
:108B6000703066B943F00803A4F15B088DF87030EB
:108B7000D8F10002464B42EB08021A7368E743F053
:108B800010030A2E8DF870307BD15A2C79D05B24DB
:108B90005EE79DF870303E4A43F020038DF8703058
:108BA000C4F15E03937230E79DF8703043F0200308
:108BB0008DF87030364B02229A7226E79DF870309D
:108BC000A4F1140C43F040038DF87030DCF1000286
:108BD0002F4B42EB0C02DA7217E79DF8703043F02E
:108BE00080038DF8703010E79DF87130312C43F020
:108BF00001038DF8713003D1254B0022DA7327E78A
:108C000036B9274B9B69002B3BD0214B0122F5E75E
:108C1000142E05D1224B9B699BB31D4B0322EDE71C
:108C20000A2E2ED1079B002B7FF4F8AE184B0222A0
:108C3000DA73032335E79DF87130154943F00803D3
:108C40008DF87130A4F13603DBB23B2C0B747FF44A
:108C5000DCAE002E3FF4FCAE1E2E12D8114AF240BC
:108C6000D5070ED50A22B6FBF2F633440B74EFE6B5
:108C70009DF8713043F010038DF87130002E3FF4F1
:108C8000E7AEFFF707FA4FF0140A51E4489D0020C1
:108C9000581E002001041040F09900204098002048
:108CA0000C9C002000041040B74B1A681BEA020F0E
:108CB00008D0B64991F8D13043F0200381F8D13083
:108CC0002BEA020BB24BD3F82831002BD9D0422C1F
:108CD00014BF00230A239E42D3D89DF8713043F07D
:108CE00080038DF8713006EB8606A84B04EB460630
:108CF00083F8E860ACE6A64BD3F82831002BC0D04F
:108D00001BF4004F03D0A34BD3F8FC302BB99DF8D4
:108D1000713043F080038DF871309C4B002283F852
:108D2000E82072E69C4B1B7E022BAAD19DF8713085
:108D3000964A43F020038DF87130A4F1600383F06C
:108D4000010382F8613060E69DF871308F4A43F08C
:108D500002038DF87130A4F1620382F83A3054E6D0
:108D60009DF87130A4F1330043F004038DF87130A5
:108D70004242864B424183F83B200423E2E64BEA21
:108D8000030B2E4634E4814B1A9AC3F8842093F8DF
:108D9000E820A2F14101012901D9A62A0ED193F8B8
:108DA000D120910605D5FFF775F94FF0190AFFF7A5
:108DB000BFBB42F0200283F8D12019E4632C02D813
:108DC000002E7FF423AE0025382C1C9500F0128174
:108DD0004FD8092C1CD8072C80F0E480052C00F219
:108DE000B180032C7ED39DF8722042F008028DF8EA
:108DF0007220611F93F8602018BF0121201F61F3CA
:108E000000024142414161F3410283F8602079E070
:108E1000332C24D8302C24D21E2C63D05C4BD3F8B6
:108E20000431002B3FF42DAF1FFA84F83EB108EB5C
:108E3000880808EB880806EB88081FFA88F840467F
:108E40009847054600283FF41CAF504BA3F8048018
:108E50009DF8723043F040038DF8723052E0352CAB
:108E6000DCD19DF8722042F020028DF872209C70B7
:108E700047E0442C14D8432C80F0F180412C00F2C0
:108E8000D4803E2C80F0BD803C2C2BD03D2CC5D115
:108E90009DF8722042F004028DF872205C7031E07F
:108EA000622C00F0E48006D8A4F14602032AB5D86B
:108EB00083F8E94026E0632CB0D1002E7FF4E1AEC8
:108EC000364AD2F808212AB9314AD2F82C21002A90
:108ED0003FF4D7AE9DF8722042F001028DF8722067
:108EE00063220CE09DF8722042F001028DF872209E
:108EF00024B1012C0FD083F8244002E0032283F830
:108F0000242000251C9B1BEA030F7FF4A6AD4BEA2F
:108F1000030BFFF76DBB214B93F80C2295060AD586
:108F2000DB6E984780F02005C5F34015002DE9D091
:108F3000164B0122E3E71A4B1D89C5F3801585F016
:108F40000105F3E7DFF85480D8F838319847B0B915
:108F5000114B1B7F042B00F09C80D8F8E0500035AB
:108F600018BF0125002D3FF48CAE9DF8723043F000
:108F700004038DF87230054B06225A70C1E70228AF
:108F8000F0D1D8F83451EAE7389A0408581E002086
:108F90000C9C002040980020489D0020F099002063
:108FA000409900209DF8723043F010038DF8723024
:108FB000BDF81430082C43F48073ADF814300FD092
:108FC000092C13D0C14B93F8163299077FF559AE8F
:108FD000BF4A92F8253043F0020382F8253091E72A
:108FE000BB4A92F8253043F00103F6E7B84B83F80B
:108FF000255087E7B74A92F8502152077FF541AED6
:109000002FE705F07FF983077FF53BAE0121084686
:1090100004F0C8FF00283FF434AE9DF8723043F0EE
:1090200002038DF87230E3B217E005F06BF9000728
:109030007FF527AE2946012004F0B4FF014620B990
:1090400004F0B0FF00283FF41CAE9DF8723043F0EE
:1090500002038DF87230002542230B9352E705F08E
:1090600051F941077FF50DAE01212846D0E7002ECA
:109070007FF407AE984AD2F82821002A3FF401AEC7
:109080009DF8712042F080028DF8712083F8E8404D
:1090900037E7054636E79DF86C301A9A43F002032D
:1090A0008DF86C309DF8183043F008038DF81830B7
:1090B000874BC3F8BC20864ADDF86C90D2F8D0808C
:1090C00018EA090F7FF46FAE844B1B6819EA030F8F
:1090D00000F05F8100211A980A92F8F7B1F80A9A15
:1090E000002800F05681FEF7D5FF4FF0040AFFF785
:1090F0001FBA9DF86C301A9A43F004038DF86C3057
:10910000734BC3F89C20D6E79DF86C301A9A43F055
:1091100008038DF86C306E4BC3F8A020CBE79DF8A8
:109120006C301A9A43F080038DF86C30684B5A66A5
:10913000C1E79DF86D301A9A43F001038DF86D3048
:10914000634B9A66B7E79DF86D301A9A43F00203B5
:109150008DF86D305E4BDA66ADE79DF86D301A9A8A
:1091600043F008038DF86D30594B1A67A3E7089B4D
:109170001A9A43F0010308939DF86C3043F01003F2
:109180008DF86C30524B5A6795E7089B1A9A43F05A
:10919000020308939DF86C3043F020038DF86C3087
:1091A0004B4B9A6787E7089B1A9A43F0040308938E
:1091B0009DF86C3043F040038DF86C30444BDA6717
:1091C00079E7002E7FF422AC9DF86D301A9943F0B8
:1091D000100308468DF86D30F8F75AF820B9E3B25D
:1091E0003B4AC2F8CC3066E7FF23F9E79DF86D30C3
:1091F0001A9843F040038DF86D30F8F75FF8344B60
:10920000C3F8C40057E7002E7FF400AC2F4991F853
:10921000B6305A060ED5A0B2FEF714FB804648B110
:10922000D1F80801C8F804001AF06CFAC8F8080070
:10923000FFF77EB99DF86D3043F080038DF86D30F7
:10924000234BC3F8C84036E79DF86E301A9A43F0B6
:1092500001038DF86E301E4BC3F888202BE79DF874
:109260006E301A9A43F002038DF86E30184BC3F833
:109270008C2020E79DF86E301A9A43F004038DF895
:109280006E30134BC3F8902015E79DF86E301A9A94
:1092900043F008038DF86E300D4BC3F894200AE7B5
:1092A0009DF86E301A9A43F010038DF86E30084B1B
:1092B000C3F89820FFE69DF86E301A9A43F0200319
:1092C0008DF86E30024BC3F8A420F4E6F09900202C
:1092D000581E0020489D00200C9C0020789A04080D
:1092E0009DF86E301A9A43F040038DF86E308D4B26
:1092F000C3F8A820DFE69DF86E301A9A43F0800389
:109300008DF86E30874BC3F8AC20D4E69DF818304A
:109310001A9A43F001038DF818309DF86F3043F02E
:1093200001038DF86F307F4BC3F8B020C3E69DF882
:1093300018301A9A43F002038DF818309DF86F30F8
:1093400043F002038DF86F30764BC3F8B420B2E6D9
:109350009DF818301A9A43F004038DF818309DF8E0
:109360006F3043F004038DF86F306E4BC3F8B820B4
:10937000A1E6002E7FF44AAB9DF86C301A9843F0BA
:1093800001038DF86C30F7F799FF664BC3F8C00006
:1093900091E648EA0903C2F8D030FFF729B96249DB
:1093A000D5F88800F7F76AFF28B1FEF773FE4FF093
:1093B000270AFFF7BDB895F8D130DF0602D5D5F8FA
:1093C000CC3013B90123C5F8CC3095F8D2306FF307
:1093D000000385F8D23095F8D1306FF3041385F887
:1093E000D130A6F14103012B01D9A62E24D10023AF
:1093F00008939DF820308DF81830412E4FF4004B23
:1094000033D10BF0D9FC04EB00200BF04BFC28B956
:10941000FEF740FE4FF0520AFFF78AB8089AD5F8D7
:10942000D0104248FEF7C6FAD5F8D030C5F8E400AF
:1094300023EA0003C5F8D0309DF8186026B1079BD9
:10944000002B08BF0223079394F8A030002B56D0BE
:10945000079B022B53D1BDF81430DC074FD4FEF725
:1094600019FE4FF0280AFFF763B8D4F8FC30F3B1C7
:109470001A78A62A1BD15E680BF09EFC864216D194
:10948000D4F8FC20D5F8D030516F28481940083264
:10949000FEF790FAD5F8D03023EA0000C5F8D000E6
:1094A000204B93F8E830422BC6D1FFF741B87C201F
:1094B00035F052FA05460028AAD01A4ED4F8FC30EE
:1094C000836796F8E8300370C4F8FC000BF074FC76
:1094D0006860D4F8FC00D6F8D03043676C220023D3
:1094E00006F164010830C6F8D03035F066FAD7E7E7
:1094F00095F8D13068F3451385F8D1309CE7094BD6
:1095000093F8D12012F0400F1D4613D0D3F8C42099
:10951000074B9A420EDDFEF7BDFD4FF01B0AFFF729
:1095200007B800BF581E002000FF7F47BC1E002068
:1095300080969800CBF3074414F0400700F0828037
:10954000AF88002F00F08680A04BA148D3F80831E7
:10955000D5F8D070984700287FF485A8D5F8D0308A
:109560007B400A939B4B0A9A1B6813400AD0C3F3B3
:109570004002C3F3076362F3C303DBB226EA0303CB
:109580008DF818300A9B089AC3F3021322EA0303EA
:1095900008930A9BC3F307218D4B11F0020F1CBFE8
:1095A000D86E0D904FF0000214BFDA660D9211F0E4
:1095B000800F4FF000011CBFD3F8C800C3F8C810DB
:1095C0000A9B08BF0E91C3F3074318BF0E901807FC
:1095D00049BF7F490021D1F894000F904CBFC1F8DA
:1095E00094200F91D9063CD5794BD3F898100C9163
:1095F000C3F89820764D95F8D230DB063FD5D5F8E4
:1096000098000BF06BFD00283FF400AAD5F8986095
:1096100000213046F7F714FE00287FF464AD6B4D4F
:10962000AB690BB33046F7F749FEEB6998474368DF
:10963000B3FA83F35B0913B3FEF72CFD4FF0260A50
:10964000FEF776BF00230C930F930A970E97002323
:109650000D93CFE700230C930F930A970E970C9B63
:10966000F6E700230C93C5E74FF09E4130464FF0DC
:109670000105F7F703FE00B90546EBB2DBE7544DF1
:1096800095F8D1301F070CD5286F0BF027FD002867
:109690003FF4BCA90021286FF7F7D2FD00287FF422
:1096A00022ADBDF814304A4D13F0010109D095F8F0
:1096B000D1309E0777D4FEF7EDFC4FF0160AFEF787
:1096C00037BF2A89212A51D195F8D03058063ED487
:1096D000414BDB6FC5F880303D4B93F8D020D70766
:1096E00040F1878093F8D22016076DD45FFA8BF291
:1096F000950708D51B89212B66D040F24B118B4270
:1097000062D04C2B60D0900603D5314B9B7A022B54
:109710005AD01BF4005F57D1CBF3074313F020035B
:1097200005D02B4B9B78A3F133014B424B412207D1
:1097300001D4002B5DD0264AD2F8C010581E8142B9
:109740004EDA002B0CBF27200420FEF78CBF61F3FC
:10975000861385F8D030EB7AE86F1BB11F49F7F715
:10976000D1FBE8671A4BC3F88000B5E7AB7A012B51
:109770000BD1079B022BAFD1502AADD0002AABD022
:1097800095F8D1309907A7D495E713F0FD0FA3D131
:1097900095F8D120920706D40F4A917899429BD12F
:1097A000936FEB6698E7EE6E00213046F7F748FDC1
:1097B00000287FF498ACEB7A002B8DD00749304617
:1097C000F7F7A0FBE86687E70123B0E70C9C0020D1
:1097D000581E0020249A0408409800203333CB41BF
:1097E00000293FF7E2AD92F8D0306FF3000382F822
:1097F000D030904B9B7A022B08D1049B002B3FF476
:1098000040AADB68DB6B002B3FF43BAACBF30725B8
:1098100015F0200F874B00F0DE8093F86120012ABD
:1098200040F0C580049AD468A27AD7077FF529AAA8
:1098300093F8D22016077EF5F8AE93F9D020002ACF
:1098400080F2B1805F6E00213846F7F7F9FC0028FE
:109850007FF449ACA66938463146F7F7F1FC00B110
:109860003E466368DE61734B93F8D0206FF3C712F6
:1098700083F8D0206F4B049A93F8613053706D4C8D
:1098800094F8D200C0F3C00310932246002B00F0DE
:10989000AC80D4F8946000213046F7F7D1FC002862
:1098A0007FF421AC049B5B78012B0ED1E37A002B73
:1098B00000F0998060493046F7F724FB5D4BC3F810
:1098C0009400049BDB685B6818615A4C627894F8DA
:1098D000D2303D2A40F0A38098077EF5A6AED4F89A
:1098E0008C000BF0FBFB00283FF490A8D4F88C0010
:1098F000524CA369002B00F08880F7F7DFFCE36986
:1099000098474368B3FA83F35B09002B7FF494AE66
:10991000484CD4F88C20C4F8982094F8D22063F3F3
:10992000924B63F34102464B84F8D220D3F80831BE
:1099300013B3444B4FF0FF32C3F894203F4A92696F
:10994000AAB1E90713D4D3F8980094F8D1300028CD
:10995000CCBF0122002262F3C30384F8D13006DDBC
:10996000F7F77CFA01234BF4807B2067E373354BD8
:109970004FF0FF32C3F89820CBF30744A60740F11D
:1099800097800B9B002B00F093803E3B294E062BCB
:1099900000F28E80DFE813F05A005A005A005A0095
:1099A000DA00490149016368A269DA6162E7049B50
:1099B0005B78012B7FF45EAF049B5B6823B1049A54
:1099C000002353600DF04CFD049B049ADB685B6838
:1099D0001B6893604EE7049A002A3FF450AF527818
:1099E00083F861204BE7184965E7049B002B3FF49F
:1099F0006CAF5B7823B9049B9B68C2F8943064E732
:109A0000049BDB685B68DB69F7E74FF09E414FF032
:109A10000104F7F733FC00B90446E3B275E7DF064B
:109A2000AAD4084BD3F89400F7F718FAC4F89800B2
:109A3000A2E700BF581E0020666698430C9C0020D9
:109A4000F09900204098002000007A4496F8D23027
:109A5000DD077EF5EAADD6F8885000212846F7F7F5
:109A6000EFFB00287FF43FAB0121084604F09AFA8F
:109A700007462846F7F748FCB842BFF496AC0125E4
:109A800086F8D450D6F88800F7F73EFC0B9B86F892
:109A9000D5003E2B03D0A3F1400045424541C64BC3
:109AA00093F8D220C3F8D8506FF3000283F8D22085
:109AB00063070FD5C04B5A78062A0BD1D3F898000C
:109AC000F7F7FCFBBD4BD3F8F8305B69984208BF51
:109AD0006FF3924B1BF4002FB74B00F0D78093F835
:109AE00060309F0706D5049BDB689B7A13F00A0F52
:109AF0003FF4C7A8B14BB04C5A7F94F82510CBF374
:109B0000005391420CBF002303F0010363F3145B85
:109B10001BF4001F00F0E58094F8D250EE0700F12E
:109B2000BD804FF07E53C4F88830A34CA378303BFF
:109B3000082B00F2CD80DFE813F0BF0033014B01AA
:109B40005B01CB006B01CB00CB007901D6F8D030A4
:109B500013F4043F3EF469AD994A32EA030305D198
:109B6000FEF798FA4FF0300AFEF7E2BCD6F8CC3098
:109B7000042B3FF61AAC3BB10021D6F88C00F7F766
:109B800055FB00287FF411AC8B4E96F8D230D907E4
:109B90001DD5D6F8885000212846F7F751FB01461D
:109BA00000287FF4A0AA012004F0FCF9074628460B
:109BB000F7F7AAFBC0B2B842BFF4F7AB012386F8AF
:109BC000D430D6F88800F7F79FFB86F8D5007A4D99
:109BD00095F8D130DA0716D5A86EF7F795FB002176
:109BE000C6B2084604F0DEF98642BFF4DEAB95F853
:109BF000CC30002B7FF4D9AB85F8D430A86EF7F7C2
:109C000083FB85F8D5006C4B93F8D22002F0FD025F
:109C10006FF3000283F8D22093F8D12002F0EF0214
:109C20006FF3000283F8D12042E7D6F8D030654ABE
:109C30001A423EF4FAACB06EF7F766FB0121054616
:109C4000002004F0AFF9854205D3FEF723FA4FF068
:109C50002C0AFEF76DBC002586F8D450B06EF7F7DD
:109C600053FB86F8D500D6F88C00F7F727FB96F85B
:109C7000D230C6F8D80065F3410386F8D23096F8A2
:109C8000D13065F3000386F8D13011E7049A002A39
:109C90003FF430AF127883F860202BE70021D4F82E
:109CA0008800F7F7CDFA00287FF41DAA2B4660F351
:109CB000000384F8D23038E794F839306FF30003AA
:109CC00084F8393094F8383023F0010384F83830C0
:109CD000394B3A4A1B8F128E9B1A18BF012363F32C
:109CE000555B354C2378042B11D194F8D250E807FA
:109CF0007EF59BAC0021D4F88800F7F7A1FA002884
:109D00007FF4F1A92B4660F3000384F8D2302A4D8A
:109D100017A8A97BFEF7F8F8EB7ADBB12A4B9DF880
:109D2000187093F82D81DFF8A4900424013C27FAE1
:109D300004F3D9070CD528FA04F3DA0708D405EBA5
:109D400084064946D6F8B000F7F7DCF8C6F8B0004C
:109D5000002CEBD1184C637B5BB19DF81830DB070E
:109D600007D5D4F8B0004FF07C51F7F7CBF8C4F822
:109D7000B000079B042B40F0BC8094F83B30002BD4
:109D800000F027819DF81830002513F0FF0F84F8AC
:109D90003B505FD1FEF77EF94FF01A0AFEF7C8BBC1
:109DA00094F8393043F0010384F8393094F83830AE
:109DB00043F001038AE700BF581E002040980020AE
:109DC0000001010000010200489D00203333CB4117
:109DD0000021D4F888004FF00105F7F727FA00B901
:109DE000054694F8393065F3000384F839306FE79D
:109DF0000021D4F8880094F83850F7F717FA20B10A
:109E000045F0010584F8385062E725F00105F9E7CF
:109E10000021D4F888004FF00105F7F707FA00B9E0
:109E2000054694F8393065F34103DEE7A94B93F812
:109E300050315D077FF54CAF0021D4F888004FF01A
:109E40000105F7F7F3F900B9054694F8393065F3E1
:109E50008203CAE7079CDFF88C829F4E9DF818901A
:109E6000013C29FA04F3DF071ED5A30008EB030227
:109E700033441069D3F8B030119319460692F7F7BE
:109E8000D5F94FF00107069A119B08B14FF0000772
:109E900013610123A3403D4329EA03030220EDB2ED
:109EA0008DF8183010F0D4FD96F83B30002B40F0C0
:109EB0008E804FF07E5158F82400F7F7B7F9B0FACA
:109EC00080F0400986F83B00002CC7D1834AD6F8C1
:109ED000D030126823EA0203814AC6F8D03092F8E3
:109EE000333082F8330043402B4302D0022010F07D
:109EF000AFFD7B4B93F83330DBB1774D9DF8188085
:109F00002B7B784F11930424013C28FA04F3DE07DD
:109F10000DD5A300EE18119AD6F8B0003B441B698A
:109F2000002A59D01946F6F7EDFFC6F8B000002C0C
:109F3000EAD11BF4807F2FD0674CE37B022B59D0F2
:109F4000032B75D0012B27D1674B9B69002B3EF467
:109F500098AE94F8D1301D0757D50021206FF7F740
:109F600065F938B15B4B93F8C03158075CBFD4F842
:109F700098302367584B186FF7F7A0F95A4BDB69F5
:109F800098474368002B3FF457AB534B93F8D120CD
:109F90006FF3C30283F8D120514B4F4F1A7A387CAC
:109FA000CBF3C02382420CBF002303F0010363F311
:109FB000CB2B002B53D007F1140112F093FF002894
:109FC0004DD1FEF767F84FF0070AFEF7B1BA01204E
:109FD00078E7FDF7A9FE8CE757F8249012934946DD
:109FE000F6F786FE129B1946F6F78CFF4946F6F700
:109FF00081FE9AE79DF8183013F0FF0FCCD1FEF7E1
:10A0000049F84FF0250AFEF793BA1BF4802FC3D10D
:10A0100094F8D230D90604D5D4F898002E4B18679E
:10A02000BAE72F4BD3F8F8305869F6F717FFF5E782
:10A030002D4DAB69002B3EF424AE94F8D1301A07B5
:10A040007EF5F3AA246F00212046F7F7EFF80028E9
:10A050007FF4F2AA2046F7F731F9EB6990E7204C3C
:10A060007B7B62793E785340CBF3803213400A2EDB
:10A0700063F38E3B3AD05C2E9DF8185000F0768149
:10A080001DB93B89023B012B19D8079B032B16D026
:10A09000114BDFF84C801A7B129204271193013F79
:10A0A00025FA07F3DA0700F18C81119ABB001A44F4
:10A0B0004344D3F88030C2F8B030002FEFD11E2EC9
:10A0C00000F0AA81352E00F0C0811C2E40F0828065
:10A0D0000920A2E1489D0020581E0020249A04086F
:10A0E00040980020280000200C9C0020D7F8CC507D
:10A0F000002D3DD09DF8183011933BB9142D3FF43D
:10A1000049AE97F8D2305B077FF544AEBE4CD4F829
:10A11000D03013F4883F3EF488AAD4F88860002138
:10A120003046F7F78DF800287EF4DDAF30463BF07F
:10A1300031F8F7F7E9F80B2DC0B20ED80A2D80F0F0
:10A14000A780012D00F0A480022D7EF49AAD94F832
:10A15000D2305F073EF595AD02E0142D7EF491AD4F
:10A1600009284DD9FDF796FF4FF01D0AFEF7E0B91B
:10A17000A64DEB6A002B3EF484ADD4F8F82052696A
:10A180002AB1FDF787FF4FF0570AFEF7D1B998477C
:10A1900000287EF468AAD4F8F820EB695069984743
:10A1A000436853B1403403F11005186859682246DA
:10A1B00003C20833AB421446F7D1934B93F8D22035
:10A1C0006FF3000283F8D22093F8D1206FF30412CA
:10A1D00083F8D1208C4B1C89502C1A4640F0928178
:10A1E0009DF8183013F0FF0F00F03C81079B012B06
:10A1F00000F03881FDF74EFF4FF01F0AFEF798B9C7
:10A20000E0B9814B187C8DF89C0028A912F06AFEF9
:10A2100000283FF4D6AE7E4B93F848318BB19DF8C1
:10A220009C20063AD1B202290BD8D340DE0708D5CC
:10A23000FDF730FF4FF0380AFEF77AB90138C0B2A7
:10A24000E1E7714EDFF8CC91D6F8CC80042427AF3B
:10A25000119A631E22FA03F3DD0713D5A5007319C3
:10A26000B8F1140FD3F8AC100FD14D44E86FF6F7E6
:10A270003FFDD5F8E410F6F73BFDE96BF6F738FD46
:10A2800047F82400013CE3D197E747F82410F9E7A9
:10A290005E4B9A69002A3EF4F4ACDB699847456846
:10A2A000002D3FF4C9A9584B93F8D220540708D584
:10A2B000D3F890202A6193F8D2206FF3820283F8BA
:10A2C000D220D3F8CC300B2B06D12CA9082012F0C9
:10A2D00009FE00283FF475AE4B4EDFF83881D6F802
:10A2E000CC700424A7F10A09119B013CE340D80774
:10A2F00035D5012F06D106EB8403D3F8B03045F8ED
:10A30000243018E00A2F20D1A20002EB0803139298
:10A31000D968D3F880001293F6F7EAFC129BD3F8C1
:10A32000E810F6F7E5FC139AB318D3F8B010F6F777
:10A33000DFFC45F82400002CD6D1012F7FF43DAF7F
:10A34000324B28465B6A984737E70B2FF3D106EB71
:10A350008403D3F8B0102CAB53F82400E7E7B9F12D
:10A36000010FE8D808EB84031B6CC8E7002D3FF40D
:10A3700011AD00260427013F25FA07F3D90718D5A8
:10A38000214B04EB060803EB0609D8F88C00D9F83A
:10A390002010F6F7ADFCD9F8BC10F6F7A9FCD8F8F8
:10A3A0004C10F6F7A5FCC9F8BC00043E002FE2D122
:10A3B00010E7154BA2193344D2F8F420C3F8BC209F
:10A3C000F3E7352E3FF479AE119B129ABC0003EBF4
:10A3D0000409D9F8B03042B144441946D4F8800099
:10A3E000F6F788FCC9F8B00067E64444D9F81400D1
:10A3F000D4F8E8101393F6F77DFC216CF6F77AFC9D
:10A40000139B1946ECE700BF581E00200C9C00204F
:10A41000489D0020409800200A2028A912F062FDE3
:10A4200000283FF4CEADDDB176490422013A25FA89
:10A4300002F3DB0706D4930027A818440B44D3F893
:10A4400080304360002AF1D1C4E66F4B1B89012B99
:10A450007FF6C0AEFDF71EFE4FF01E0AFEF768B88D
:10A460000795B7E6002382F83A30BDF81430664A03
:10A4700013F0010100F0538692F8D13003F0FD0390
:10A480006FF3861382F8D130079B5F4C3BB15F4A74
:10A49000D4F8D030126823EA0203C4F8D030D4F8DC
:10A4A000D010002940F0A780564D28222CA834F067
:10A4B000A8FA95F8A3308DF8CA302B8EADF8C830C5
:10A4C000534B9DF8C52093F8AD30B3FA83F35B0985
:10A4D00063F3410263F38202BDF814308DF8C520A6
:10A4E00013F0010308932E4600F06D86494B1B685C
:10A4F0003BEA030300F03486FDF7CCFD4FF0100A71
:10A50000FEF716B8079A022AAFD13E4ABDF81410DA
:10A5100012881392A21A18BF012262F34921ADF8E2
:10A5200014103CB99DF8183013F0FF0F9DD1002393
:10A5300007939AE793F83C200AB983F83A20324B04
:10A5400093F86120012A0FD193F86020D70705D531
:10A550000021D3F89400F6F769FE28B1FDF79AFDC3
:10A560004FF0290AFDF7E4BF212C2BD1049BDB68B7
:10A57000DB6B002B3EF485AB234B0021D3F880002E
:10A58000F6F754FE00287EF410AFBDF8143043F007
:10A590002003ADF814301C4B93F83C20002A00F047
:10A5A000AA82BDF8142012F0020900F0C681154AF3
:10A5B0009178012940F0A281FDF76CFD4FF0030A6C
:10A5C000FDF7B6BF4C2C40F08281049BDD68EB6B3D
:10A5D000002B3EF456AB0C4B9A7B012A05D0FDF7BD
:10A5E00059FD4FF02A0AFDF7A3BF9DF818201192DC
:10A5F00012F0FA0F10D0FDF74DFD4FF0240AFDF7D1
:10A6000097BF00BF40980020581E0020249A0408DD
:10A6100040990020349A040893F8D220560708D5B0
:10A620004FF07E51D3F89000F6F70AFE00287EF432
:10A63000BCAE119B5C077DF5F8AFAA4CAA4BD4F8D1
:10A64000D0201340002B3DF4F0AFD4F888900021C7
:10A650004846F6F7F5FD002600287EF444ADA76FC6
:10A6600031463846F6F7ECFD00287EF43CADD4F8D0
:10A670007C8031464046F6F7E3FD00287EF433AD9A
:10A68000636F129331461846F6F7D0FD00287EF42A
:10A690008CAE31463846F6F7C9FD00287EF485AE0B
:10A6A00041463846F6F7E0FD00287EF47EAE94F889
:10A6B000D130D80604D594F8CC30032B3EF675AED5
:10A6C000049B69699C682046F6F7BAFD00287FF470
:10A6D000BCAAA9692046F6F7D1FD014600287FF4FF
:10A6E000B4AA139B814C4C2B06D01822A01834F02E
:10A6F00088F94FF07E5363617A4DC4F80090D5F825
:10A70000B8306360002112981393F6F799FD2B4639
:10A71000002800F0D980764A744CDB7A6262129A83
:10A72000E76022F00040A060C4F810806BB171496E
:10A73000F6F7E8FB6F49A0603846F6F7E3FB6D4992
:10A74000E0604046F6F7DEFB2061664B5B7B93B131
:10A75000664D4FF07C51A868F6F7D4FB4FF07C5162
:10A76000A860E868F6F7CEFB4FF07C51E8602869F6
:10A77000F6F7C8FB2861119BD90737D5594D5E4FB5
:10A780006869D7F8E810DFF86481F6F7B3FA396C36
:10A79000F6F7B0FA0146D5F8B000F6F7A9FAD7F8FF
:10A7A0008810C8F8180011901398F6F7A1FA119ABA
:10A7B00020F000431146C5F8883004461046F6F7ED
:10A7C000A1FB214607462046F6F79CFB014638468A
:10A7D000F6F790FA3AF0EEFD01464846F6F792FB9E
:10A7E000D5F88810F6F742FCC8F800003D4B93F806
:10A7F000D140220704D5186FF6F786FD3B4B9862CF
:10A80000E30648BF374B394D42BFD3F8CC20374B16
:10A8100083F82C2014F0010F18BF324B334C1CBFAF
:10A820009B6EEB610021E869F6F714FD10B995F80D
:10A830002C301BB90023E66184F82C3094F82C30BE
:10A8400093B12D4B6068D3F88810F6F751FA4FF0AA
:10A850007C5120F00040F6F755FB0146E069F6F721
:10A860000DFD00287EF4A1AD1E4A92F8D2305F079C
:10A8700042BFD2F890101D4A516113F0020F194BDC
:10A880001EBF1A4AD3F88C101162BDF8142093F839
:10A89000D01042F02002ADF8142093F8D22002F03C
:10A8A000F9026FF3000283F8D22093F8D12001F06F
:10A8B0009F0102F0E7026FF304116FF3000283F8C7
:10A8C000D01083F8D12066E64FF07E5224E7054B86
:10A8D0000021D86EF6F7AAFC00283FF45CAEFEF724
:10A8E000EABE00BF581E002070000100A01F00201B
:10A8F000000080BF3333CB414098002093F8D23022
:10A900005E077DF592AE9DF818309DF85E10CB4045
:10A91000DD077DF58AAE9DF85C301633002142F8E4
:10A9200023109DF85D309166163342F82310012301
:10A9300082F87030002382F871308D4A92F8D1305D
:10A9400013F0100F134656D10122C3F8CC2093F810
:10A95000D220540717D5D3F89000DB7A002B54D0BF
:10A960008449854DF6F7CEFA814B9DF85E401A7BFF
:10A970000646002A4CD0203455F824103046F6F70D
:10A98000B9F97D4BD8667A4E9DF818301193337B18
:10A990009DF85E501293784BDF6E984605F11603D2
:10A9A000139305F1200304241493119B013C23FA13
:10A9B00004F2D0070ED5A200B1184244D1F8B0007D
:10A9C0009065A54234D0D2F880101592F6F790F930
:10A9D000159A9065002CE8D11635674B53F8255031
:10A9E00038462946F6F72CFC88B3FDF753FB4FF0A9
:10A9F000360AFDF79DBDD2F8CC20002AA7D1FDF77D
:10AA000049FB4FF0130AFDF793BD4FF07E51A8E7C5
:10AA100003EB840304F13A02103455F8221058690C
:10AA2000F6F768F955F82410F6F764F90146A5E73A
:10AA3000129B002BCED0149B58F82310F6F758F930
:10AA40003946F6F757F9139B48F82300C2E7484BFD
:10AA500093F8D1201E8964F3041283F8D12093F86F
:10AA6000D22064F3820283F8D220A6F149021C4668
:10AA7000102A40D8DFE802F0533F3F3F3F3F3F3FBF
:10AA80003412531234093F3F0900A6F156013A4BE4
:10AA90004A424A4183F8712083F87020542E09D12C
:10AAA000049BDB689B7A5A077EF5EBA8324B0022A9
:10AAB00083F87020DFF8B88098F8D240E30729D5F2
:10AAC000D8F8889000214846F6F7BAFB00287EF4B3
:10AAD0000AAB294B60F30004C3F8689088F8D240B1
:10AAE00029463846F6F704F9234C552E606602D104
:10AAF000002384F870301E4C2389332B00F0CF8262
:10AB000000F2A180022B00F0C88037D8012B3FF45F
:10AB100009ADAAE4B9F1000FE2D0FDF786BD94F8C3
:10AB2000D23098071FD5D4F88C5000212846F6F76C
:10AB300091FB00287EF4D7AAE37A8BB10D49284611
:10AB4000F6F7E0F90C4B5866094B93F8D2206FF3F7
:10AB5000410283F8D220084B4FF07A529A66CAE736
:10AB60004FF07E51EBE7B9F1000FF4D0FDF75DBD7A
:10AB7000581E00203333CB4140980020032B00F0B7
:10AB80009280052B7FF471ACA37B002B7FF427AD63
:10AB90009DF8183013F0FC0F7DF440AFAB4AD4F8A9
:10ABA000D03012689A437DF440ADBDF81420910571
:10ABB00005D5A74A126832EA03037DF436ADA54CE9
:10ABC00094F8D030E77AD4F88860D4F88C5013F039
:10ABD000300F40F0338206F10043636705F1004314
:10ABE000A367002F40F04D829A4BD3F88810D3F81A
:10ABF0008C50994B93F8333063B1984E954C306933
:10AC0000F6F780F92946C4F888007069F6F77AF9F2
:10AC1000C4F88C008F4A904BD2F888109963D2F810
:10AC20008C10D96392F8D03003F0DF036FF3041374
:10AC300082F8D03092F8D23003F0FD036FF30003B6
:10AC400082F8D23011E48D2B20D01AD88C2B7FF4CF
:10AC50000CAC8E3B012B9EBFBDF8143043F00803B3
:10AC6000ADF814309DF8183013F0FF0F3FF492A8A0
:10AC700010227B497B4833F091FE00287FF4F5AB2E
:10AC80008FE08E2BE5D08F2B7FF4EFABBDF8142037
:10AC900042F01002ADF81420DBE7BDF8143043F0A9
:10ACA0000403ADF814309DF8180000283FF472A892
:10ACB0009DF85C309DF85D10012202FA03F302FA60
:10ACC00001F10B43034205D1FDF7E4F94FF0200AEF
:10ACD000FDF72EBC5F4C94F8D230D90767D5D4F875
:10ACE00088000AF0FBF900283DF490AED4F8880003
:10ACF000F6F70AFBC4F8E00000283EF456AB94F8DF
:10AD0000D2306FF3000384F8D230524F9DF85C606C
:10AD1000514C07EB860306F12002D3F8B00054F83B
:10AD20002210F5F7E5FF9DF85D5007EB850305F16F
:10AD30002002804654F82210D3F8B000F5F7D8FF6F
:10AD400094F833900746B9F1000F18D0434B321DE9
:10AD5000291D53F8220053F82110F6F7D3F80021EB
:10AD6000F6F76EFA58B1BDF81430BDF8142083F030
:10AD70000403C3F3800363F38202ADF81420354C5F
:10AD800094F8D23013F0040200F0BA806FF382031B
:10AD900084F8D230102204F1B001324833F0FEFDC5
:10ADA00040B9FDF777F94FF0210AFDF7C1BBC4F8B0
:10ADB000E020AAE7E37AD4F8900023B12A49F6F715
:10ADC000A1F8C4F89000234BD3F890200892B9F171
:10ADD000000F14D0214B0436043553F8264053F8A5
:10ADE000255020462946F6F749FA089A00B125462B
:10ADF00011462846F6F786F8164BC3F890004146F0
:10AE00004046F6F77FF8134C054639463846F6F7C4
:10AE100079F8D4F8909006464FF081414846F6F70D
:10AE200071F84946F6F76EF82946F5F761FF3146A5
:10AE3000F5F75EFF00218146F6F702FAB0B1FDF7A3
:10AE400029F94FF0220AFDF773BB00BF749A04087A
:10AE5000309A0408581E0020409800202800002046
:10AE6000081F0020C09800203333CB4148463AF0F9
:10AE7000A1FA314681462846F5F73CFF3AF09AFAA6
:10AE800009F1004901464846F6F7F0F82389AC4C31
:10AE9000D4F89060032B05464FF0000108BF00F185
:10AEA00000453046F6F7CCF928B106F1004605F129
:10AEB0000045C4F8906039462846F6F723F89DF817
:10AEC0005C6001464046F5F713FF4FF07C51F6F702
:10AED00019F81C3604EB86069DF85D3070601C3353
:10AEE0004146284604EB8304F6F70CF83946F5F79B
:10AEF00001FF4FF07C51F6F705F86060FFF7B5BA37
:10AF0000012303FA06F1AB400B4308990B4205D12C
:10AF1000FDF7C0F84FF0230AFDF70ABB94F8D030D4
:10AF200003F09F0362F3041384F8D030E37A83B113
:10AF30007C340322089B013AD340DB0706D5206806
:10AF400080491192F5F7DEFF119A2060043C002A37
:10AF5000F0D1B9F1000F17D0DFF800927A4A03243C
:10AF6000089B013CE340D8070AD502EB8403D9F8DB
:10AF7000000019691192F5F7C5FF119AC9F8000090
:10AF8000A9F10409002CEBD16D4C04EB8606404678
:10AF9000716FF5F7ADFE04EB85050646696F38461F
:10AFA000F5F7A6FE314605463046F5F7ABFF2946D4
:10AFB00006462846F5F7A6FF01463046F5F79AFE05
:10AFC0003AF0F8F99DF85C3004EB83030646596FBC
:10AFD0009DF85D3004EB830308465F6FF5F792FF41
:10AFE000394605463846F5F78DFF01462846F5F700
:10AFF00081FE3AF0DFF9C4F890000146054630467C
:10B00000F5F776FE20F0004450492046F6F736F971
:10B0100000283FF42AAA4FF07C512046F6F72EF97B
:10B0200000287FF4BEAE4A492846F5F76BFF21465B
:10B03000F6F706F900283FF418AAB2E64FB14149E5
:10B04000606FF5F75FFF3F496067A06FF5F75AFF44
:10B05000A067404B93F83330002B01F09F81384CB0
:10B06000DFF8E480606FD8F81010F5F74BFFD8F8E0
:10B0700014106067A06FF5F745FFA067002F01F07F
:10B08000878130492E4C3046F5F73CFF2D49C4F8F6
:10B0900088002846F5F736FFC4F88C00A4E5A37BAA
:10B0A000002B7FF49CAA9DF8183013F0FC0F7DF460
:10B0B000B5AC294BD4F8D0201B6893437DF4B5AAD6
:10B0C000656F00212846F6F7B1F800287EF46DA9D7
:10B0D000E37A4BB11B492846F5F714FF194960671D
:10B0E000A06FF5F70FFFA0671A4B93F833305BB1F1
:10B0F000134C154D606F2969F5F704FF69696067A6
:10B10000A06FF5F7FFFEA0670D4A92F8D03003F06C
:10B11000DF036FF3041382F8D030FFF7A6B992F87B
:10B12000D23061F3041361F3C30382F8D23092F892
:10B13000D13061F3410361F38613FFF7A3B900BF78
:10B14000581E00203333CB41280000200AD7A33BF0
:10B150006F12833A40980020309A0408D41E0020D1
:10B160002378352B02D0002B7FF4C6A9734D05F14F
:10B1700028030FCB2DAC84E80F00737F8DF8C63009
:10B1800096F89F30EBB995F8283013F0020303D0FE
:10B190006B6B9B7AC3F3C0039DF8C420684C67496E
:10B1A00063F3C7128DF8C4202CA8224606F00EFCCB
:10B1B000054618B9634B0FCB84E80F002846FDF70E
:10B1C00052BA0123E8E713F0A7FF1BF4004F8146B2
:10B1D0001AD094F8E8307BB1412B15D194F8CC50BB
:10B1E000D4F88800F6F790F8D4F8E4102A4680B234
:10B1F000FCF704FCFDF737BAD5F8FC0020B1846FEA
:10B2000033F0B2FBC5F8FC40049B7BB3DB689B7A50
:10B210001A072BD5494B1B895A1E022A09D9052B1F
:10B2200007D0332B1EBFBDF8143043F04003ADF8F8
:10B2300014309DF8183013F0FF0F62D0079B022BDB
:10B240005FD1BDF8143043F08003ADF81430049B97
:10B250009DF814201B7813F0020318BF82F04003FE
:10B26000394A18BFC3F3801382F89F30334B364AF4
:10B27000189CD3F8C430C2F8903033936CB1B9F154
:10B28000020F0AD02046F4F7CDFF013033F064FB03
:10B29000349010B1214635F058F9284B2A4C1BF058
:10B2A000200F1CBF9A7AA270DA6EA267049A5278B5
:10B2B000012A5DD11B89502B00F0C880002B00F0C3
:10B2C000C580049B049ADB689DF85D005D6805F10C
:10B2D0001003536000216862FCF782FD049B286222
:10B2E0005D689DF85D302969203354F82300F5F737
:10B2F000FFFC00210646F5F7ADFFEC6830B32546AC
:10B3000033E0049B1B7803F00303012B9FD1BDF8AE
:10B31000143003F040020C4B1B88591E022903D93C
:10B32000052B01D0332B06D1002A90D0BDF8143064
:10B3300043F0200389E7002AF8D088E7581E002050
:10B34000C0980020081F002040980020584930462F
:10B35000F5F7D8FD01462868F5F788FE0546014651
:10B360002046F5F76DFF0028C9D1524BC3F8945021
:10B37000504B9DF81440D3F89450049B294698688C
:10B38000F5F754FF08B1A3061DD5049B1B78DF0712
:10B3900014D5260612D4049BDB685B681D600CF094
:10B3A0005FF8049B6506D8685CBF424BD3F89420D5
:10B3B000049B48BF0022197813F09CFA3D4B049A75
:10B3C000D3F8943093603B4D14F0400F08BFD5F88C
:10B3D0009430D5F8980018BF00232F93F5F76EFF2F
:10B3E000354BD3F89420824220D0B9F1020FC3F834
:10B3F00094001BD00021FCF705FC6B783D2B044624
:10B400003BD02E4B93F8061211F004011A462BD0B4
:10B41000D2F83431002B30D00021284BD3F8303112
:10B42000002B41D081F00101204698470B9B002B57
:10B430004CD03E3B1F4C062B48D8DFE813F04500AC
:10B440004500DB00DB00EB004500FC00049B5B6873
:10B4500023B1049A002353600CF002F8049B9A680D
:10B46000144BC3F8942083E71548007F042804D0C8
:10B47000D3F8E030002BD0D1CAE72046FCF7EEF934
:10B48000104BD3F8D8305BB1049A15789847049BD9
:10B490001B78AB421EBF074A4BF4002B82F860308A
:10B4A000FCF7CEFD0121B8E780200FF0D1FABDE70F
:10B4B000DB0FC940581E002040980020F099002062
:10B4C000489D00200C9C0020FCF7CEFB1BF4802F35
:10B4D0004FD0754B5B78062B4BD1B9F1020F48D09A
:10B4E000724BD3F89400349B002B40F0AE8034A90B
:10B4F000FCF788FB6E4C20600BF0B2FF349818B15B
:10B50000FCF716FF00233493684B2068D3F8F8301B
:10B5100042695B699A422CD0664BD3F8D8305BB154
:10B52000049A14789847049B1B78A3421EBF5E4A76
:10B530004BF4002B82F860305F4BD3F83421002AA3
:10B5400000F0858059489047044628B1FF280CBF79
:10B55000012400247DF487A880200FF079FA002CC4
:10B5600040F0818013F0D8FDB0F5007F7BD0FCF770
:10B5700067FD1BF4002F2CD04B4C049B94F86010FB
:10B580001B788B4213D0049B04985B782F9AC06879
:10B5900013F032FA38B1049BDB685A6894F86030D3
:10B5A0001372049A137080F00100C3B21093434BDE
:10B5B000DA7F6FF3C302DA77109B53B13D4B1C6CFB
:10B5C0003CB1049B049904985B782F9A0978C06871
:10B5D000A0473649344C049B4B6794F8E930A3F1FB
:10B5E0004602032A00F28680DFE812F06C00870131
:10B5F0009A016C00D4F8D800F5F730FC0021F5F77B
:10B6000015FE294BB0FA80F1490993F8D50003F0F3
:10B6100001F85BE7D4F88C3094F8CC2094F8D5107E
:10B6200094F8D40003F008F8244B18644FF4006039
:10B630000FF00EFA4AE7D4F8D800F5F70FFC0146F0
:10B6400094F8D50002F0D8FF40E7002150E7174AF0
:10B650001B6C1B48012182F8A0104FF480619847B1
:10B660000BF036FC7EE7134B9B69002B81D01BF45B
:10B67000807F3FF47EAF0C4BDA7B012A7FF479AFF9
:10B680001C6F002120466FF3082BF5F7F7FD30B152
:10B690002046F5F713FE054BC3F8980069E7044B05
:10B6A0001B685869F7E700BF581E0020409800202B
:10B6B0009C1F00200C9C0020F09900204099002045
:10B6C00078990020002225928D4A106952692492AF
:10B6D000CA6A239012B15268D2682592A3F1490434
:10B6E000884863426341826F23A909F073FA0028F6
:10B6F0003DF452A8834CA36F2C93A378012B02BF77
:10B700009DF8C43043F020038DF8C430636FDA68CD
:10B710003092186859682DAA03C21B789DF8C4207E
:10B720008DF8B43094F89F3063F3C7128DF8C420BD
:10B730000BB194F89E309DF8C520CBF3074463F31A
:10B740000002E5068DF8C52009D56F4D95F8250056
:10B75000FBF728FF18B16B4B95F825205A77694FF6
:10B7600067487B7F8DF8C630002114F0200F80F8E9
:10B7700020100B9717D0644B97F8312093F839308D
:10B7800002F0010203F001039A4206D0C27F63F384
:10B790000002C27708460AF007FE5B4B188F594B30
:10B7A000188606F0F7FB584CA388F3B1B9F1020FE5
:10B7B0001BD0A3790BB10BF053FE0A9BC4F8D03019
:10B7C0000D9BE3660E9BC4F8C8300F9BC4F8943001
:10B7D0000C9BC4F898304D4BD3F80C5113F09CFCE3
:10B7E0004949A8470023C4F8D030474C2378042B9C
:10B7F00003D1D4F8880006F037F95FFA8BF616F01B
:10B80000040F404B1CBFA27B9A71700644BFE27AC2
:10B81000DA70CBF30725E90709D5206FF5F74EFD60
:10B820009DF818303A4A0146E07BFCF72DF82A07CC
:10B830000ED5DFF8E8C0374FBCE80F000FC7DCF8C3
:10B8400000303B604FF400700FF002F916F0FCFD81
:10B8500016F0080F2B4E1CBF237B33716B0604D5EB
:10B86000637B737108200FF0F3F8AF0744BF94F8BF
:10B870003A3086F832302378282B00F0EE8100F23F
:10B88000CE801C2B00F03E8100F2B9800A2B00F024
:10B8900008811D4C1B4D268994F83C302E80502E7B
:10B8A00085F834302F46A04600F0E982079B022B32
:10B8B00040F0E582184B1B68359395F8313003F062
:10B8C0000102069206999DF8C420332E61F30412FA
:10B8D0008DF8C42000F04983094A00F21082032E3B
:10B8E00000F2DE81022E80F0F582002E00F09A82B6
:10B8F000012E00F044820026B3E209F0A3F9F9E634
:10B900004099002040980020581E00200C9C0020E8
:10B91000081F002048980020981F0020681E002063
:10B9200009F0ACF9054600283FF4E4AE01466A4848
:10B93000FCF78AF8694A2B6D9367694B197888067A
:10B9400044BFA17A91705A78D10719D56FF30002DC
:10B950005A7016F079FD4FF480600FF079F8614A63
:10B960005E4BD27BDA7105F1500605F1400240339F
:10B97000106851681C4603C40832B2422346F7D10E
:10B98000574CA3789F0606D56FF34513D5E91601EA
:10B99000A3700AF009FDA378DE060CD56FF304133B
:10B9A000A370504B93F825004C4B58774E4BB3F88F
:10B9B000C810FBF7A9FD4A4B1B79DBB14B4B4C4C34
:10B9C00093E8070084E80700203C94F83010E06A10
:10B9D00001F0010112F0F6FE18B9296EE06A12F0CA
:10B9E0004FFE414BA26AB3F8D03094F82010E06AC1
:10B9F00013F028F83A4B1B684BEA030B7AE61E2B30
:10BA000000F09B80262B7FF444AF3A4B0FCB28AC41
:10BA100084E80F002146092011F038FA39E7662B37
:10BA20002E4C00F0228122D85C2B7FF432AF324EB4
:10BA30003046FBF7ABFF012384F8E43096E80F00B3
:10BA400004F1E80585E80F0010222C49284632F061
:10BA5000A5FF254B003093F8413118BF012084F831
:10BA6000E40098073FF515AF29460B20D4E7702B6B
:10BA700000F009817A2B7FF40CAF23AD29460B200F
:10BA800011F030FA2846FBF781FF10221B492846A7
:10BA900032F084FF003018BF012084F8E400E8345D
:10BAA000F9E0D4F8CC30022B02D0142B7FF4F1AEA5
:10BAB00028AC21469DF89C0011F0E8F9327A9DF8F7
:10BAC0009C309A427FF4E5AE94E80F000C4D85E877
:10BAD0000F0016F0B9FCDCE6601E00204098002044
:10BAE000481E0020581E0020489D0020801E002077
:10BAF00060980020C0980020081F00201CA904089E
:10BB00004C980020BA4A9DF8181092F82D3192F8FE
:10BB10002E210B40134032797AB173B1D6F88C10D4
:10BB2000D4F8BC0094F8EA501E0706D5F5F77EFB62
:10BB300018B145F0080384F8EA309DF8C43043F0AA
:10BB400001038DF8C430079B1BB12CA9A94805F04F
:10BB500021F9A94D95F8EA3028AE002B78D00BF0EA
:10BB60007FFC96E80F0023AC84E80F0095F8EA30DC
:10BB70001D0738D5A149269839F0BEFB002105469E
:10BB80002690F5F75DFB20B19C492846F5F7B2F801
:10BB900026909B4B9949D3F88C0039F0ADFB0021DE
:10BBA0000546F5F74DFB20B128469449F5F7A2F874
:10BBB000054626992846F5F79BF892490646F5F77B
:10BBC0003FFB002839D08D492846F5F793F8054604
:10BBD000874B2846D3F89C10F5F794F938F0F6FF18
:10BBE000894BC3F8A8000AF05DFB8849884816F025
:10BBF00041FC2CA9204605F0CDF80BF031FC7E4B22
:10BC000093F8EA301C070AD5794B2B98D3F89C108F
:10BC1000F5F778F938F0DAFF7B4BC3F8A8000AF0A3
:10BC200041FB7A497A4816F025FC28AB0FCB784CBB
:10BC300084E80F00FCF778F82BE676493046F5F7F4
:10BC40001DFB0028C4D06D492846F5F751F8BEE722
:10BC50002CA9304605F09EF8E7E76D4B0FCB28ACDA
:10BC600084E80F0021460A20D6E6614B93F8411183
:10BC700011F0020107D110221FA832F0C2FE1FA945
:10BC80000B2011F003F9644D2846FBF77FFE0023DB
:10BC900084F8E430614C95E80F0084E80F00F8E583
:10BCA000052E00F03F81212E7FF425AE05920BF08A
:10BCB000D7FB059AD4F88010D58B2CA8FCF7EEFAA8
:10BCC000064600287CF4CFAC9DF8B43043F08003E6
:10BCD0008DF8B4309DF8C43043F010038DF8C430B3
:10BCE0009DF8C9302CA943F0020304F1B0008DF88F
:10BCF000C93005F04FF8284606F04CF9B1E0542E53
:10BD000023D8512E80F07581492E00F0EF814C2E02
:10BD10007FF4F1AD424F05920BF0A2FB059A396812
:10BD200092F81F80D48B2CA8FCF7B8FAC8F340080F
:10BD3000064600287CF497AC2CA843463A4605F109
:10BD4000800105F0D1FC2046D6E78C3E032E3FF65D
:10BD5000D2AD274B9DF8C42093F8443183F01003F3
:10BD6000C3F3001363F304128DF8C4202CA9BDF8AB
:10BD7000142004F1B00005F0B7FF064671E0AB787F
:10BD8000022B18D19DF8C43043F040038DF8C43025
:10BD9000174B1B7E022B18D1D5F88810D4F8B800A9
:10BDA000F5F744FAB0FA80F040099DF8B43060F33A
:10BDB000C7138DF8B4302CA90E4804F0EBFFD7F868
:10BDC000FC3023B96FF3CF3B95E50120EDE75C68CC
:10BDD00008F0F2FF84420CBF0123002363F3CF3B42
:10BDE00002BFD7F8FC301B7888F8E83083E500BF45
:10BDF000489D0020081F0020581E00200000B4436A
:10BE000040980020000034C340990020DC990020B5
:10BE1000C0980020000034431CA904082899002081
:10BE2000A01F00209DF8C4302CA943F0010304F1A9
:10BE3000B0008DF8C43004F0ADFFD5F8FC30002B15
:10BE4000C0D05F6808F0B8FF87420CBF0123002311
:10BE500063F3CF3B7FF44FADD5F8FC301B7884F80B
:10BE6000E830B84BB849359A1A604B783BB9002E88
:10BE700040F04181B54BB64C0FCB84E80F001BF46A
:10BE8000004FB44F00F0838197F8E830622B00F048
:10BE90003A81A62B02D0422B40F0798108F08CFF2A
:10BEA000AD4C04EB002008F0FDFE00283DF4B0AAE4
:10BEB000D4F8FC000022416F0830FBF77BFDD4F87A
:10BEC000FC4094F87050E06AF5F71EFA2A46616F5C
:10BED000FFF78DB9AB78022B0BD19DF8B43043F04E
:10BEE00080038DF8B4309DF8C43043F040038DF8E2
:10BEF000C430BDF81410D8F8E030D8F89020009283
:10BF0000490748BF5B420293179BADF804301B0CF6
:10BF10008DF80630914B8E4A2CA903F13C0004F0B9
:10BF2000FFFFE8E4616FD5F88000F4F7E3FEA16F4E
:10BF30001D90D5F88400F4F7DDFEA96B1E90D4F8AF
:10BF4000B000F4F7D7FEE96B2390D4F8B400F4F70F
:10BF5000D1FE23AB2490009305F180021DAB2CA9E8
:10BF600004F1B00005F0B6FAC5E4626FD5F8808040
:10BF7000069211461046F4F7BDFE7949F5F776F8BA
:10BF80004146F4F7B7FEA36F1D9019461846D5F841
:10BF900084600593F4F7AEFE7149F5F767F8314612
:10BFA000F4F7A8FE069AD4F8B0701E9011464046E9
:10BFB000F4F7A0FE3946F4F79BFE0146F4F79AFE2B
:10BFC0006749F5F753F83946F4F794FE059BD4F822
:10BFD000B470239019463046F4F78CFE3946F4F7D6
:10BFE00087FE0146F4F786FE5D49F5F73FF83946CE
:10BFF000ADE7542E7AD1C3F34006309B0B9A5B68B1
:10C00000B2F8308092F83020DB680892032414F0F4
:10C0100002051CBF3546012614F00104059342F0C9
:10C02000010261D0484B0792D3E9047164200AF001
:10C03000BBF90123079A069C0693069B62F3070847
:10C0400063F3082866F34928404605F0A3FF4149F9
:10C05000414ED1F894302F9396F8323086F87230F2
:10C0600033462CAA33F8580B0293D1F8CC30019305
:10C07000179BADF800301B0C8DF80230B03106F183
:10C08000800305F001FD3388542B7FF434AC9DF818
:10C09000203086F83030089B43B91946309812F0AA
:10C0A00091FB18B90599309812F0EAFA40F2013381
:10C0B0001B0A9A0742BF96F8312065F3410286F8C1
:10C0C0003120DB070CD5204B1F6196F8312064F33B
:10C0D000000286F831201CB9596938460AF064F923
:10C0E000308E05F057FF06E42746A6E700252C46CC
:10C0F00005952F46ABE7012E7FF4C1AE9C31144865
:10C1000016F0B8F9BBE6D7F88800F5F7FDF8B9F1F5
:10C11000020F84B235D1134B2046D3F80851FBF7F8
:10C1200091FB00287CF4D9A91021012032F004FBF6
:10C1300018B30D4A048013684560C3B91060FCF75A
:10C14000CCB900BF981F002040990020081F002094
:10C15000C0980020581E002040980020CC1E0020CF
:10C1600000004040F0990020441F00201346DA6888
:10C17000002AFBD1D860FCF7B0B94FF0530AFCF7A6
:10C18000ACB997F8CC2001212046FFF731B834989C
:10C1900008B1FCF7CDF897F82430834C23771BB90E
:10C1A000824B1B891D060FD5A9F10200464246416C
:10C1B0000BF056F9207F632821D17D4BD3F82C2139
:10C1C000BAB1904700232377099B002B3CF4B0A918
:10C1D000784C099B013B099304EBC3035968099B05
:10C1E00034F8330007F0D8FF099B002BF1D1FCF79E
:10C1F0009FB99B6D002BE5D031469847E2E70328B5
:10C2000000F0A98097F82430012B00F0B9803C2B76
:10C2100000F0BA80654D2A89110600F1B180B9F1AC
:10C22000020F06D01E2B04D1634BD3F8F03103B1BB
:10C23000984701222280227A002384F89C3087F8D4
:10C240003C30A3712371A37022B14FF400702372AC
:10C250000EF0FEFB94F83120002363F3000284F813
:10C260003120E26A637784F830304AB1526884F84A
:10C270002030117A636263F3041184F82130117263
:10C280004E4F97F8403113F0020104D0049BDB6855
:10C290005B686422DA6097F85031DA070AD503F058
:10C2A00006039A1F5342534194F8312063F38202EC
:10C2B00084F83120238EEB8319B1642108460AF0FB
:10C2C00073F8B9F1020F28D03D49207A10F00AFE28
:10C2D00000283DF476AE97F841319B070ED423A990
:10C2E0000B2010F0FFFD48B11022364923A832F090
:10C2F00055FB18B133490B2010F0C8FD16F0A4F817
:10C30000002012F0CBFB2C4B607F5B6F9847102016
:10C310000EF09EFB20200EF09BFB254DAB6D13B164
:10C320003146207F9847244B93F8B63013F0400FE6
:10C330000CBFFD20FE20FBF7D7FE08F083FCB9F10F
:10C34000020F04D197F94231002BFFF63BAFEB68A7
:10C350000820984736E7B9F1020F3FF433AF97F85A
:10C3600024303C2B04D1144BD3F8F03103B198475F
:10C37000114B15481B6C082198470AF0A9FD21E7CD
:10C38000B9F1020FF4D11DE7B9F1020FEBD119E7B2
:10C39000D4F88810D4F88C50FEF72FBC002F7EF410
:10C3A00070AEFEF737BC00BF4098002040990020D7
:10C3B0000C9C0020481F0020F0990020489D002080
:10C3C0004C98002028990020789900207047002080
:10C3D00070470000074B07B5DB6D98470022C3B2DA
:10C3E00063F30702C0F3074363F30F22104603B061
:10C3F0005DF804FBF0990020024B034A1B68D2F859
:10C40000C00018470C9C0020F0990020074B1B68C7
:10C4100010B5044603B19847E4B2A4F10F035C429F
:10C420005C41034B83F8914010BD00BFF81F002012
:10C4300040990020074B70B51B6804460D4698478D
:10C44000054B9B6F23B129462046BDE87040184735
:10C4500070BD00BFE81F00200C9C0020034B93F828
:10C460000602400800F00200704700BFF09900206B
:10C470002DE9F84F354C236803B3354B93F89030D2
:10C48000E3B1344E336D984725680DB10023236026
:10C49000F36C984795B10027336D98476369D5F8D9
:10C4A0000C80EF60D5E9019A6F6003B96561F36CA8
:10C4B000984745465046C847002DEDD1264E337863
:10C4C00063B9244F01233370D7F8E8319847234BE1
:10C4D0001A688242804603D100233370BDE8F88F8A
:10C4E000D4E90125AA42F7D01860F5B94FF0000948
:10C4F0006568002DF0D02B68A3EB0803002BEBDC64
:10C500003B6D98476368AB4214D1EB686360636925
:10C51000C5F80C90D5E901ABC5F8049003B9656185
:10C52000FB6C98475846D047E2E7D5E90130984779
:10C53000ED68DAE7002BEAD0DA68002AE7D0AA42F1
:10C5400002D1EA68DA60E2E71346F5E7FC1F002053
:10C5500040990020F0990020F01F0020EC1F0020DF
:10C5600008B50EF043FA024B0022C3F82C2108BD97
:10C570000C9C00201FB5FBF7BFF80E4B0290DB6D43
:10C5800098479DF808209DF809409DF80A309DF8CD
:10C590000B1004EA1024024001EA106103EA104380
:10C5A0002243002062F307000B4363F30F2004B023
:10C5B00010BD00BFF099002010B50D4B0D491C783F
:10C5C0008AB0E443E4B268461C7033F0BEFF2046F4
:10C5D00008F01CFC0146684633F09BFF064968469C
:10C5E00033F097FF002168460CF044FD0AB010BDFF
:10C5F00048000020A89A0408EDEE04082DE9F04751
:10C600000F4E104CD6F8C0300F489847E368ABB1D6
:10C610004FF00008336DE56898476369EF68C5F827
:10C620000C80D5E9019AC5F8048003B96561F36C03
:10C6300098475046C847E760002FEBD1BDE8F08728
:10C64000F0990020FC1F00207C9A04084AB1064A99
:10C6500092F84521920704D5044A1846D2F82421BD
:10C6600010470020704700BF489D0020F09900202F
:10C67000074B93F84221D20608D54269D3F8C4117A
:10C680008A4203D0C3F8C4210FF042BA704700BFFA
:10C69000489D0020704700002DE9F8431F4E814659
:10C6A000336D884617469847B9F1000F33D01C4DBB
:10C6B0006C69A4B100236B61D6F8E8319847002378
:10C6C000E3606B68C4F808803844C4E9000923B10A
:10C6D0001A68821A002A15DCE3606C600AE02824DC
:10C6E000013C20012B18DB6913B918302C18E3E743
:10C6F000002CF5D1F36C9847201C18BF0120BDE831
:10C70000F8831346DA681AB11168411A0029F8DA79
:10C71000E260DC60EEE74C46ECE700BFF0990020F9
:10C72000FC1F002010B50B480B4C0189C1F34021C0
:10C7300059B10A4B012138301B6C9847A28A08482E
:10C740000021BDE81040FFF7A7BFA28A0AB1054843
:10C75000F7E710BD40990020489D0020F099002087
:10C7600025C7000869C70008064B07481B8913F452
:10C77000007F064B9A8A064B4FF0000108BF18460F
:10C78000FFF78ABF4099002025C70008489D002078
:10C7900069C70008C30704D5322200210148FFF70A
:10C7A0007BBF7047FDC500082DE9F041114C236D9A
:10C7B00080460F469847104A536883B1002659684F
:10C7C000DD68414511D117B19968B9420DD156B113
:10C7D000F56000215960D960516901B95361E36C7A
:10C7E000BDE8F04118475560F3E71E46002DF6D02E
:10C7F0002B46E4E7F0990020FC1F002010B504460A
:10C80000E30708D500210848FFF7CEFFC822002122
:10C810000548FFF741FF054B1B681BB12046BDE8EB
:10C820001040184710BD00BFF9C30008F41F0020D6
:10C83000F8B5164D06462B6D0F46984726B3144B98
:10C840005C694CB100225A610022E2609A68C4E936
:10C850000167A2B99C600BE02824013C22019918D1
:10C86000C96919B902F118041C44EDE7002CF4D190
:10C87000EB6C9847201C18BF0120F8BD1A46D368FE
:10C88000002BFBD1D460F3E73446F1E7F0990020A8
:10C89000FC1F00202DE9F041114C236D074688460E
:10C8A0009847104A93687BB100265968DD68B94201
:10C8B00010D1996841450DD156B1F56000215960FC
:10C8C000D960516901B95361E36CBDE8F041184783
:10C8D0009560F3E71E46002DF6D02B46E5E700BF36
:10C8E000F0990020FC1F0020F8B5164D06462B6D70
:10C8F0000F46984726B3144B5C694CB100225A612D
:10C900000022E2601A68C4E90167A2B91C600BE06A
:10C910002824013C22019918C96919B902F11804A7
:10C920001C44EDE7002CF4D1EB6C9847201C18BF99
:10C930000120F8BD1A46D368002BFBD1D460F3E781
:10C940003446F1E7F0990020FC1F00201A4B2DE936
:10C95000F04193F88E500746884655BB174E336D0D
:10C96000984727B3164B5C6944B15D610022E260D1
:10C970001A69C4E90178AAB91C610BE02824013CBA
:10C9800022019918C96919B902F118041C44EDE78C
:10C99000002CF4D1F36C9847201C18BF0120BDE88F
:10C9A000F0811A46D368002BFBD1D460F2E73C46F5
:10C9B000F0E70024F0E700BF40990020F099002044
:10C9C000FC1F00201A4B93F88E3070B505460E46BA
:10C9D00053B3184C236D984721461DB3164B5C6921
:10C9E0004CB100225A610022E260DA68C4E90156C3
:10C9F0009AB9DC600AE02824013C20011A18D269A7
:10CA000012B918301C18EEE7002CF5D1CB6C984702
:10CA1000201C18BF012070BD1A46D368002BFBD123
:10CA2000D460F3E72C46F1E7BDE87040FFF75CBF48
:10CA300040990020F0990020FC1F00202DE9F74FBD
:10CA4000BD4EBE4DBE4CBF4FB0220021304631F02E
:10CA5000D8FF4FF426720021BB4831F0D2FF4FF4CB
:10CA600098720021284631F0CCFFB84BC5E9173346
:10CA7000B74BC5F82031B74BC5F82431B64BAB6680
:10CA8000B64B2B67B64BC5F88430B64BC5F888302B
:10CA9000B54BC5F88C30B54BC5F8DC304FF4077298
:10CAA0000021B34BC5F8CC30204631F0AAFF0A2351
:10CAB0002360B04BC4F8B031AF4BC4E91333AF4B74
:10CAC00063654FF4E863C4F8B8314FF08043E36125
:10CAD000012384F81632AA4B2366AA4B2367AA4B7C
:10CAE000C4F89C30A94BC4F80032A94BC4F83831C3
:10CAF0004FF6FF73A4F80E32012386F88E3003F050
:10CB0000ABF810F071FE0DF071FF2EF009F93B78D3
:10CB100060F300033B7008F02BFD08F04FFD10F0B0
:10CB20006DFE1022002106F19C0031F06AFF994B46
:10CB3000D4F88C201A6094F80422974BC4F88C30F7
:10CB400002F06001A1F1600CDCF100013B7841EBE7
:10CB50000C0142F0600261F3C30384F80422C2F3C3
:10CB6000400262F304133B70DBB24FF00009FF2B6D
:10CB70000CBF01234B4686F8929086F88F30A8466A
:10CB80000FD1864BD4F814211A60854BC4F81431A8
:10CB90008448A36B98473B7886F88F9060F34103F5
:10CBA0003B70804D0DF1060195F8CC0011F006FCAC
:10CBB000814688B911F056FB494611F027FB002841
:10CBC00000F0A58190F900308DF80630002800F0C3
:10CBD000A081437885F8CC300DF1070195F8CD00A0
:10CBE00011F0ECFB18B995F8CC3085F8CD309DF9F3
:10CBF000060011F073FC3B7860F382033B70002861
:10CC000000F08B81002011F03BFCC36A002B00F088
:10CC10008281036B003318BF01233A7863F38202E9
:10CC20003A7094F8053213F0040304BF95F8C0215C
:10CC300063F341023B7808BF85F8C021FF2B06D083
:10CC400010230021584886F88C30FFF7BBFED4F83B
:10CC50008C3095F82C0101219847012011F01EFF1E
:10CC6000636F4FF000009847D4F8FC310BB14F4888
:10CC700098474FF00F0004F047F896F88C30103BBF
:10CC800018BF012386F89030636E1BB195F8B3315D
:10CC9000DF0707D594F81112454B464A002908BF13
:10CCA00013466366AA8A1AB100214348FFF7F4FCD1
:10CCB00094F8053213F00C0F0FD0C3F3C0024FF0FD
:10CCC000040162F34101C3F3800363F30001012215
:10CCD000C9B240F28A2010F0B7FB94F8B63003F0E6
:10CCE0000C03042B06D1354BD4F804211A60344BC5
:10CCF000C4F80431D8F8BC304BB994F8073298071F
:10CD000005D5D4F8243113B12E4BC8F8BC3094F9B2
:10CD10000632002B0BDA94F90C32002B07DAE36EA3
:10CD2000984741B2C943C90F2748FFF74BFE024F4E
:10CD30004FF000094AE000BF409900200C9C002001
:10CD4000F099002048000020FC1F002071C400085A
:10CD500061690108450D0208CDC30008712202086F
:10CD6000F57400083D780008B9CD010871C60008C7
:10CD7000652E010861C5000871530108CFC3000882
:10CD8000BDF20008991E020855FC0108550C020866
:10CD90005DC40008F81F00200DC40008E81F002033
:10CDA00035C40008489D0020B9C50008DC99002062
:10CDB00075C50008D5C3000825C70008F41F00206A
:10CDC000FDC700084DC60008756801080DF00EFE8D
:10CDD000F278D6E904AB22B195F9B221002A80F2AB
:10CDE000A58040220021384631F00BFE6FF0010291
:10CDF000326496F88E20002A40F09A8095F842110D
:10CE000011F0400F08BF4FF0640AC6F810A0002AC6
:10CE100040F0918095F8423113F0200F08BF4FF099
:10CE2000640B0020C6F814B011F01CFB28B10020E0
:10CE300011F026FB43686422DA60AB8A3289003342
:10CE400018BF012363F34922328195F85031D90785
:10CE500041BFF27FC3F3400363F38202F27708F02D
:10CE6000E3FDD4F8D430984795F84201C0F3400070
:10CE7000FBF744F995F84A01A36D4FF0000100F06B
:10CE80000100984708F0A6FE13F052F802F0AEFE3B
:10CE900014F0E6FF09F006FA3249334815F0EAFAD1
:10CEA000D4F8903013B100210846984794F8063220
:10CEB0005A0701D416F008F9D8F80030D4F8C400A5
:10CEC000984795F94131002B07DB12F025F9B0F5B1
:10CED000807F02D1012012F05FF994F80632DB075F
:10CEE00007D596F89230002B14BF872080200AF0D7
:10CEF000C9FA1E4B1B6923B1236C1D484FF48041B6
:10CF000098470AF04FF8C8B186F88E905EE703465E
:10CF10005AE60B235EE601237FE611F0BFFA11F01B
:10CF2000DDFA3B7860F382033B707AE68C2259E7A6
:10CF30004FF0640A69E74FF0640B72E7D4F8E4310C
:10CF40006BB19847834686F88E90BBF1000F7FF453
:10CF50003DAF08F0EBFC584603B0BDE8F08F4FF052
:10CF6000010BF0E7DC990020C0980020FC1F002096
:10CF7000789900202DE9F74F4B4E4C4C96F89000D5
:10CF8000002832D0E368002B68D12369DBB1DFF8D9
:10CF900020814FF00009C246D8F8503025699847E3
:10CFA0006369EF68C5F80C90D5E901B0C5F8049045
:10CFB00003B96561DAF84C30019098470198D84779
:10CFC0002761002FE8D196F89030002B68D1384BBC
:10CFD000384D93F8B620520744BF374AC3F80421AE
:10CFE000EC6D12F099F8A047FAE7E2683AB3676986
:10CFF000DFF8C88084461346054686465968414591
:10D0000010D0D96865B1E9601146C3F804E0C3F8EF
:10D010000CE017B91F464FF0010C2DB90A4605E088
:10D020000120F2E711461D460A46E9680B46002931
:10D03000E4D1BCF1000F00D0676100B1E260636829
:10D040003BB9A368002B9DD058680021FFF722FC54
:10D05000F7E758680021FFF7A7FBF0E796F8903054
:10D06000134F1BB997F8B63059078ED44FF000090B
:10D070003B6DE56898476369D5F80C80C5F80C905E
:10D08000D5E901ABC5F8049003B96561FB6C98471D
:10D090005846D047C4F80C80B8F1000FE8D174E7C7
:10D0A00003B0BDE8F08F00BF40990020FC1F0020B6
:10D0B000F09900200C9C002095C7000827910108DA
:10D0C000C0B215F02DBAB0F9BC30013BC21892F8CD
:10D0D000C0208A4202D1D9B208467047002BF4D151
:10D0E000FAE700795368984296BF0120002011703A
:10D0F0007047000008B543798B4203D30846F3F725
:10D10000A9FE08BD0048FCE7000080BF2DE9F84FEC
:10D11000284B294E1C6841EA4007DC2303FB0763C8
:10D120001A444FEA410992F8C0A080460D4609EB27
:10D13000010B2378434537D1236A5B4459788A45EC
:10D1400032D39B7853452FD3AAEB01016369C9B24F
:10D150002846984740B3DC2101FB0761226A91F819
:10D16000BE3044790260A3421CD891F8BF30A3427C
:10D1700034BF00230123417E4D4463F386112A44CA
:10D180004176037952781A4401239340DC2202FB52
:10D190000766D6F8B0201340427F63F386124277C9
:10D1A000BDE8F88F0023E6E7646A002CC1D1204671
:10D1B000F6E700BF142300204C000020F0B4054621
:10D1C00008461249124E0C68DC2740EA450107FB6D
:10D1D00001610A4400EB400792F8C0102278AA428D
:10D1E0000ED1226A3A445678B14209D392788A42E3
:10D1F00006D32469891B1A46C9B22346F0BC1847D6
:10D20000646A002CEAD1F0BC704700BF14230020F0
:10D210004C0000202DE9F04F85B0484E039341EAC1
:10D22000400BDC2303FB0B630190D3F8B040107874
:10D23000C44014F00104884691467DD1404B1F68DC
:10D240004B00204602935D183B78019A93426FD1C0
:10D250003B6A99F800102B445A78914268D39B7826
:10D260008B4265D3891A7B69C9B240469847044608
:10D2700000285DD0437E5B0659D54FF0DC0A99F853
:10D2800000200AFB0B6A01239340DAF8B020134315
:10D29000CAF8B03099F8003000250AEB050292F880
:10D2A000C0209A4227D1DC2303FB0B6696F8B430EA
:10D2B000AB4206F1B40B20D8029A3B6A99F80010F1
:10D2C0004244134440465B78039AC91AC9B23B6989
:10D2D00098473B6A236096F8B43099F800201E44C2
:10D2E000012086F8C0205A1E8BF8002089F80030F3
:10D2F00005B0BDE8F08F0135CFE70AEB050292F8E3
:10D30000C13082F8C030FF2B0FD0B368EAB243B10E
:10D31000092D05EB45008CBFA5F10A010021014450
:10D320000B4441460198FFF749FF0135BEE7012054
:10D330007F6A002F88D1DBE70020D9E74C0000206E
:10D34000142300202DE9F041164D174B2A181B68B5
:10D3500092F89C4106460F469A68EAB11978D9B905
:10D36000196A0879844217D34979A14214D3201A43
:10D370003946C0B29047804688B10C4B9B6C43B194
:10D380000121D5F88C21A140114002D13A46304606
:10D3900098474046BDE8F0815B6A002BDCD14FF036
:10D3A0000008F6E74C000020142300200C9C00200D
:10D3B0002DE9F047194D1A4B2A181B6892F854436F
:10D3C000074688465A681AB31E78012E20D1196A7A
:10D3D000087984421CD34979A14219D3201A4146C5
:10D3E000C0B290470F4BD3F84890B9F1000F12D05C
:10D3F000D5F8443306FA04F41C420CD14046F3F746
:10D4000029FD314602464B463846BDE8F0471847ED
:10D410005B6A002BD6D1BDE8F08700BF4C0000202E
:10D42000142300200C9C00209446124AF0B4146887
:10D43000114A4500DC2606FB0525294491F8C01059
:10D44000E56885B1227882420DD1276A7E78B142A3
:10D4500009D3BA788A4206D3881B1A4661462B46FE
:10D46000C0B2F0BC1847646A002CE9D14FF0FF301D
:10D47000F0BC7047142300204C000020F0B4104D85
:10D48000134605440F4A95F878521468E66986B148
:10D490002278012A0DD1226A5778BD4209D39278A9
:10D4A000AA4206D3ED1B0A46B4460146E8B2F0BCD8
:10D4B0006047646A002CE9D12046F0BC704700BF89
:10D4C0004C0000201423002008461146034A10B4E3
:10D4D00014681A46234610BC184700BF18230020C2
:10D4E0002DE9F04FA0F5B97085B0032852D8DFE8D8
:10D4F00010F004005500AD000301AC4FAC4BD7F861
:10D500009042D3F890510C40AC4298463AD0002655
:10D51000DFF8A492ADF80C6065408DF80E6007F559
:10D52000DC7AE8075FFA86FB28D5D9F868310193E1
:10D5300059465046FFF7C7FD00210246019B0120D6
:10D540009847D8B1036ACBB1417997F876C28C4538
:10D5500014D897F877C28C4510D3027F012101FAC5
:10D560000BF1C2F3C10221428DF80E2014BF01223B
:10D5700000228DF80C2003A9002298476D0806F1BF
:10D580000106CED18B4BC8F890411B6813B14FF404
:10D59000B9709847002005B0BDE8F08F834F844BE9
:10D5A000D7F86442D3F894510C40AC42984642D02C
:10D5B00000266540ADF80C608DF80E6007F5DC7A4A
:10D5C000E9075FFA86F932D57B4B49465046D3F8D6
:10D5D00068B1FFF778FD002102460120D84730B33B
:10D5E000D0F820B0BBF1000F21D0012202FA09F3DC
:10D5F000234208BF1346427F18BF02238DF80E3026
:10D6000012F004030AD0417997F876328B421BD886
:10D6100097F877328B4234BF00230123C2F3800294
:10D620008DF80D208DF80C30002203A9D8476D0825
:10D6300006F10106C4D15F4BC8F894411B68002B6A
:10D64000A8D040F27310A4E70023E7E7574F584BE8
:10D65000D7F86C43D3F898510C40AC42994699D016
:10D6600000266540ADF80C608DF80E6007F5257A50
:10D670004FF0010BEA075FFA86F82FD54E4B414673
:10D68000D3F8683101935046FFF71DFD0121024692
:10D69000019B0846984708B3036AFBB1427F12F02A
:10D6A00030021BD190F805C097F852E3E64515D833
:10D6B00097F853E3E64511D3017F0BFA08F818EA0F
:10D6C000040FC1F3800114BF4FF0010C4FF0000CA8
:10D6D0008DF80D108DF80CC003A998476D0806F160
:10D6E0000106C7D1334BC9F898411B68002B3FF4A2
:10D6F00051AF4FF4BA704CE72C4F2D4BD7F8404345
:10D70000D3F89C510C40AC4299463FF443AF0026FD
:10D710006540ADF80C608DF80E6007F5257A4FF086
:10D72000010BEB075FFA86F82FD5234B4146D3F860
:10D73000683101935046FFF7C6FC01210246019B68
:10D740000846984708B3036AFBB1427F12F0300CD9
:10D750001BD112F004020AD0417997F852238A4271
:10D7600021D897F853238A4234BF002201220BFAB2
:10D7700008F818EA040F8DF80C2014BF01220022CB
:10D780008DF80D2003A9002298476D0806F10106C7
:10D79000C7D1084BC9F89C411B68002B3FF4FAAE77
:10D7A00040F27510F5E66246E1E700BF4C0000204C
:10D7B000489D002008230020F0990020006938B51A
:10D7C0000D46144628B19168F2F722FD10B9257074
:10D7D000012038BD0020FCE72DE9F0410446184641
:10D7E0000E4617461D4607F079FC40B30021284637
:10D7F000F3F73AFD00B3154BD3F868812368284648
:10D800001C78F3F781FD124BC5B2DC20294600FBE2
:10D810000430FFF758FC04F0010102466008C047DD
:10D8200078B1437E5B060CD517B183691F420AD0DD
:10D8300035700020BDE8F081FF233370FAE7022045
:10D84000F8E73A20F6E75620F4E700BFF099002009
:10D850004C00002000B58BB02422002101A831F03B
:10D86000D0F8242201A9114831F098F8104B114A40
:10D8700098B91149C3F864111049C3F86C111049E3
:10D88000C3F85C110F49C3F858110F49C3F8601170
:10D890000E49C3F86821C3F87411D3F86801831ADC
:10D8A000584258410BB05DF804FB00BF449B002078
:10D8B000F09900200DD10008BDD1000815D2000854
:10D8C00045D30008B1D3000829D400087DD400084E
:10D8D00008B52821012030F02FFF18B1054A136840
:10D8E00013B9106008BD13465A6A002AFBD158626A
:10D8F000F8E700BF1423002042EA410270B5164940
:10D9000033B3DC2505FB021595F8BA404470B5F930
:10D91000BC50E618AE42C4BF2B1BDBB2013C1C441A
:10D920008470DC2404FB02156E6806B9686004FB91
:10D9300002144FF6FF75A4F8B650DC2404FB021263
:10D94000B2F8BA101944A2F8BA100370184670BDA4
:10D95000FF2444708370F0E74C0000202DE9F04F65
:10D960004FEA410B87B01E4601294BF0010300939B
:10D9700082461346894600F103054FF00002964C9B
:10D9800040F00281FFF7B8FF94F85431184484F84E
:10D99000540133464A4649462846FFF7ADFF94F8FE
:10D9A0005531184484F85501009A8C4DDC2303FB53
:10D9B00002F003FB0BF32918EA18B1F9BA40B2F9E7
:10D9C000BA108C42B8BF0C460194002C00F0D580F0
:10D9D0009268002A00F0F0800026F2182A4492F89B
:10D9E000C020FF2A40F0E380009BDC225A434FF026
:10D9F000000808EB02032B4493F8C030FF2B40F0E3
:10DA0000D880774B774AB9F1010F08BF1A46009BBF
:10DA1000DC204343E9180C338A6000FB0BF16C18DF
:10DA2000CDE90401A26001F10C02AA18EB180292E0
:10DA3000039300249AF80030002B3FD09AF801108D
:10DA4000A1423BD89AF80230A34237D30598634BE2
:10DA500003449819E2B280F8C020109880B19B6806
:10DA6000521AD2B243B1F1B2092901EB41008CBF85
:10DA70000A39002101440B4400214846109FB84751
:10DA8000172C06F1010619D8059A544B02989918DB
:10DA9000012303FA04F2D1F8D8301343C1F8D83087
:10DAA000514B5249002C08BF194632F032FD204636
:10DAB00007F0ACF90146029832F02BFD9AF80330DA
:10DAC000002B47D09AF80410A14243D89AF80530A9
:10DAD000A3423FD3049B009F1846404B00FB0733F3
:10DAE00003EB0800E2B280F8C020109888B19B6870
:10DAF000521AD2B24BB15FFA88F1092901EB410009
:10DB00008CBF0A39002101440B4401214846109F73
:10DB1000B847172C1CD8049B009903981A462F4B22
:10DB200002FB0131012303FA04F2D1F8D830134388
:10DB3000C1F8D8302C4B2D49002C08BF194632F0C3
:10DB4000E8FC204607F062F90146039832F0E1FC58
:10DB500008F10108019B0134A342BFF46BAFDC2242
:10DB600002FB0B53D3F8D810C3F8AC10009B02FB98
:10DB70000355D5F8D830C5F8AC30019B181C18BF38
:10DB8000012007B0BDE8F08FFFF7B6FE94F85631DC
:10DB9000184484F856013346012249462846FFF7C7
:10DBA000ABFE94F85731184484F85701FCE601366F
:10DBB00013E708F101081CE71826FF21013E82192E
:10DBC0002A4482F8C010F2182A4482F8C010002EAD
:10DBD000F4D1B04615E700BFF09900204C000020BA
:10DBE000E39A0408CB9A0408C69A0408C59A040864
:10DBF0000388A3F5B973032B14D8DFE803F00202FE
:10DC00000C0C094BD3F8BC0168B1D3F8900200307A
:10DC100018BF01207047044BD3F8980218B1D3F80D
:10DC20006C03F4E7002070474C000020A0F5B970A9
:10DC300003281AD8DFE800F0020A0E150C4BD3F8BF
:10DC400090010C4BD3F8643218407047084BD3F85E
:10DC50009401F6E7064BD3F89801064BD3F840330E
:10DC6000F2E7034BD3F89C01F7E70020704700BFB1
:10DC7000489D00204C0000201B284FF0000313D0CB
:10DC80001D2818D00E2823D1124A4B7092F8443127
:10DC9000C3F300030B7092F8443183F00203C3F323
:10DCA00040038B70012070470A4A4B7092F845314F
:10DCB000C3F38003EEE7074A4B7092F84431C3F395
:10DCC00080130B7092F84431DB43C3F3C013E8E7D1
:10DCD00018467047489D0020A0F10F03DBB20B2BC4
:10DCE00010B594BF0124002411D800224A70094ABB
:10DCF000072B92F8BF2105D9A0F11803DBB2032B43
:10DD000028BF002322FA03F303F001030B7020461F
:10DD100010BD00BF489D0020794B1B682DE9F347DB
:10DD2000054603B19847774B93F88F30002B00F0EE
:10DD3000B180754CD5F89421D4F89002D5F89011A3
:10DD400002400140C5F89421D4F86C03D5F89C2119
:10DD5000C5F890110240D5F89811C5F89C21D4F867
:10DD6000BC2100230140ADF800308DF80230ADF841
:10DD700004308DF80630C5F89811002A3DD094F88B
:10DD80007262002E39D0013EDFF88091F6B204F5C0
:10DD9000DC7A9846F1B25046FFF795F9D9F86871E8
:10DDA000024600210120B847074618B3036A0BB3A7
:10DDB000437F4079C3F3C0138DF8013094F8763275
:10DDC00083426AD894F87732834266D30123D5F828
:10DDD0009021B340134214BF012300238DF800307B
:10DDE0003B7FC3F3C1038DF802303B6A00226946D2
:10DDF0003846984716F1FF36CCD2D4F89832002B2B
:10DE000044D094F84E63002E40D0013E3F4FDFF8DF
:10DE10000481F6B24FF00109F1B24046FFF753F921
:10DE200001210246D7F868A10846D04758B3D0F878
:10DE300020A0D4F86C3309FA06F1BAF1000F56D0DD
:10DE4000194254D0427F12F0300C50D1D5F89821AD
:10DE500011EA02030AD0427994F85233934244D82B
:10DE600094F85333934234BF002301238DF80430D8
:10DE7000D5F89C31194214BF012300238DF80530D9
:10DE8000002201A9D04716F1FF36C5D2204B1B68EE
:10DE900003B1984702B0BDE8F08769468DF800806D
:10DEA000FFF7EAFE0028A0D169467879FFF714FF52
:10DEB00000289AD178790D2897D8F9F787FC80B295
:10DEC00070B1B5F8C030184214BF012300238DF89B
:10DED0000030B5F8C23018420CBF0123002382E79E
:10DEE0007B791E2B81D101237DE76346BEE70022AB
:10DEF00023EA01014FF4BA700FF0A6FAC3E700BF9E
:10DF00000C230020409900204C000020F0990020B4
:10DF100010230020E0020020204B2DE9F74F41EABA
:10DF20004007DC2606FB07368246B6F9B620019389
:10DF300001328B460DD11A4BD3F8684199464CBB40
:10DF40002546019ADC2303FB07232C1BE4B2A3F82C
:10DF5000B640019ADC2303FB072797F8B60003B00D
:10DF6000BDE8F08F08F101085FFA88F5D9F868314B
:10DF70002A465946504698470028E2D0437996F8F9
:10DF8000BE209A4203D896F8BF209A42EAD20134C2
:10DF9000E4B2E7E74FF000084446E5E74C00002014
:10DFA000F09900202DE9F047174F41EA4006DC23A5
:10DFB00003FB06738046B3F9B8200132894607D1C6
:10DFC000124AD2F868110025A3F8B8509246C1B998
:10DFD000DC2303FB067696F8B800BDE8F087013530
:10DFE000DAF86831EAB24946404698470028EFD04F
:10DFF000437F5B06F3D4B4F8B8300133A4F8B830EB
:10E00000EDE71C46ECE700BF4C000020F099002033
:10E010002DE9F04F554D85B0D5F86C6103938146DD
:10E0200088469246002E6AD001286FD100296AD115
:10E0300095F854419AF80030029348EA4903019355
:10E04000019A4B4B4FF0DC0B0BFB023BDBF80470EF
:10E050000FB19BF8BA70D5F86831002B65D0002F4E
:10E0600063D0013FFFB2D5F868313A464146484691
:10E07000984706460028F2D0437F5906EFD4019B0B
:10E0800040791A463A4BDC2101FB023292F8BE304D
:10E09000984242D392F8BF2082423ED3C01AC0B207
:10E0A000029B1A1A53425341002F3BD0029B8342DA
:10E0B000D7D1737F5B0638D4039BD5F86C71524679
:10E0C00041464846B847737F60F38613737760B361
:10E0D000019A1146264ADC2303FB0123B9F1010F03
:10E0E0004FF6FF72A3F8B8202CD1B8F1000F21D160
:10E0F00095F85431A34202D1013C85F85441304691
:10E1000005B0BDE8F08F95F8554193E711B995F842
:10E1100056418FE795F857418CE731795846FEF71D
:10E12000D2FFBDE70BB1002EC3D1FF238AF8003028
:10E130000026E4E795F85531A342E0D1013C85F88B
:10E140005541DCE7B8F1000F07D195F85631A342ED
:10E15000D5D1013C85F85641D1E795F85731A34216
:10E16000CDD1013C85F85741C9E700BFF0990020A7
:10E170004C0000202DE9F8430E461F4609784379EC
:10E180008B420546904603D2FF233370002425E0DE
:10E19000144BD3F8689103681C78134BDC2000FB08
:10E1A0000430FEF790FF04F0010102466008C84702
:10E1B00004460028E8D0437F5B06E7D41FB1A3697B
:10E1C00037EA0303E2D12B681878324600F00101E8
:10E1D00043464008FFF71CFF0028D7D02046BDE883
:10E1E000F88300BFF09900204C0000202DE9F8438F
:10E1F000477F414B87F008071E68C7F3C003077FBE
:10E20000C7F3400704460D46914647EA4307002EF0
:10E210006ED0326A23689A4268D1E36A002B65D0D7
:10E22000294620469847804600285FD0227F336ADF
:10E2300032486571C2F3400203EB42031344247970
:10E240005978DC237B43C2180C44012101FA04F401
:10E25000C35CD2F8D810022B21EA04014FF6FF74F8
:10E26000A2F8B840A2F8B640C2F8D810044604D0CC
:10E27000032B25D04046BDE8F883B9F1000F07D045
:10E280001F4AB9F80010B2F80C320B43A2F80C3256
:10E29000A5F10E030D2B0AD8DC2303FB0747002250
:10E2A000D7F8D8104FF4B9700FF0CEF8E2E71D2D73
:10E2B000F2D02846F9F78AFA80B20028ECD1D9E7E3
:10E2C000962D05D0972D0BD000224FF4BA70EBE7B6
:10E2D0000B4A92F8163243F0020382F81632F3E743
:10E2E000074A92F8163243F00103F6E7766A8EE7A2
:10E2F0004FF00008BEE700BF142300204C000020B0
:10E30000F0990020134AD2F8683130B54FF0000080
:10E31000E3B1D2F86C51D2F85C11D2F85841D2F87E
:10E320006031003518BF0125003118BF01210034CC
:10E3300018BF0124003318BF012365F3000064F304
:10E34000410061F3820063F3C30030BD19461C46EF
:10E350001D46F2E7F09900202DE9F84F99463B4B16
:10E36000154641EA4004DC2202FB04340746636898
:10E37000884613B90020BDE8F88FB4F9BA30002BF5
:10E38000F8D0FFF7BFFFC307F4D5002D5AD0B4F97A
:10E39000BA60A2462E4B013EF1B22046D3F868B1D6
:10E3A000FEF791FE414602463846D847834610B9EB
:10E3B000002EEFD1DEE7836935EA0303F8D1407917
:10E3C0009AF8BE1088420DD39AF8BF30834209D321
:10E3D000401AC0B201460A9A5846C8470028E7D0FA
:10E3E0000120C8E79BF804102046FEF76CFEF1E719
:10E3F000E9B22046FEF767FEDAF868B10246414608
:10E400003846D847834628B90135B6F9BA30AB4209
:10E41000EED8AFE7407996F8BE1088420CD396F854
:10E42000BF30834208D3401AC0B201460A9A584608
:10E43000C8470028E8D0D3E79BF804102046FEF731
:10E4400042FEF2E72646DFF808A0DEE74C00002097
:10E45000F0990020F0B587B000241746FF220394FE
:10E460008DF80C204FF48072049205460E46224629
:10E470000BB1197879B90592059A03AB0093B2B143
:10E480000C4B4FF4804231462846FFF765FF9DF85C
:10E490000C0007B0F0BD184604AA02A90593029427
:10E4A00006F064FD049BFF2B98BF0594E4E7024B44
:10E4B0003A46E8E7BDD70008E3D000082DE9F0416F
:10E4C00043F4804604460D461346D2B9607905B937
:10E4D00038B323681978FF2D4FEA510701F0010482
:10E4E00005D085428CBF00F1FF3005F1FF3006F00A
:10E4F0008DFC3246034621463846BDE8F041FFF721
:10E50000A9BF1278002AE1D0026810784FF4804247
:10E5100000F001014008FFF79DFFFF28D6D0BDE8BD
:10E52000F081FF20FBE700002DE9F84F42EA4106A9
:10E530001C25DFF8A480754308EB0504074694F812
:10E5400004B089469246BBF1000F27D11C4BD3F88B
:10E550006C311BB311464846FFF7DEFC2071E8B171
:10E56000184BDC2202FB063651465B464FF48042D4
:10E57000484648F80560FFF76DFF134BE360134B07
:10E580002361134B6361134B6071A36106F03EFC82
:10E590000635014608EB050031F0D7FF3B4604F194
:10E5A0001805224603CAAA4218605960144603F1AE
:10E5B0000803F6D1106818603846BDE8F88F00BF30
:10E5C000F09900204C000020F5D00008D9D70008B1
:10E5D000BDE4000875E100089422002038B5054C20
:10E5E000D4F8645105B1A847D4F86401003018BFCD
:10E5F000012038BDF099002008B5054BD3F85C31F7
:10E600001BB1984700F0010008BD1846FAE700BFAB
:10E61000F099002010B5074CD4F858211AB10031F8
:10E6200018BF01219047D4F85801003018BF0120CD
:10E6300010BD00BFF099002010B4054CD4F8604123
:10E6400014B1A44610BC60474FF0FF3010BC7047B7
:10E65000F099002008B5054BD3F874311BB19847E9
:10E6600000F0010008BD1846FAE700BFF09900204D
:10E67000036837B51A78DB78DA42044603D10025FF
:10E68000284603B030BD144BC2681A60FFF7E2F8A9
:10E690000028F4D020681149C37802780091002145
:10E6A000FFF75CF905460028E9D0FFF711F90028CB
:10E6B000E6D00023E26803702368026122694261A8
:10E6C000DA7803620AB1626882601B78002BD7D0C7
:10E6D000A368C360D4E700BF18230020C9D4000892
:10E6E000F8B5334B1B680D46002B38D004681A6A06
:10E6F000A24246D1017F437F0279C1F3400104EB7E
:10E7000041040C4483F00803C3F3C00341EA43030C
:10E7100061780A44012101FA02F22649DC2404FB53
:10E720000314D4F8D840224207D0234E2F78D6F8CD
:10E7300090411FB31443C6F89041DC2404FB03133B
:10E74000D3F8AC301A420AD01B49AC78D1F89431D6
:10E75000012C14BF1A4323EA0202C1F89421407924
:10E760000E2812D1144B297893F8442161F300024A
:10E7700083F84421BDE8F8400DF0CAB924EA020448
:10E78000D9E75B6A002BB2D1E9E70D28F2D8F9F797
:10E790001DF882B2002AEDD007492C78B1F8C030BC
:10E7A0001CB11343A1F8C030E4E723EA0003F9E702
:10E7B000142300204C000020489D0020244B1B689F
:10E7C00070B4002B36D004681A6AA2423BD1057F90
:10E7D000437F0279C5F3400504EB45042C4483F0E4
:10E7E000080360780244012000FA02F2C3F3C00378
:10E7F000184845EA4303DC2404FB0304D4F8D8405A
:10E800002242044607D0144D0E78D5F89801A6B1DF
:10E810001043C5F89801DC2000FB0343D3F8AC306B
:10E820001A4207D00C484978D0F89C3141B11A43BC
:10E83000C0F89C2170BC0DF06BB920EA0200E8E73B
:10E8400023EA0202F4E75B6A002BBDD1F2E700BFC6
:10E85000142300204C000020489D00205A4A1268D2
:10E860002DE9F3411AB1904702B0BDE8F081574A53
:10E87000D2F8BC110029F7D0B2F97242002CF3D0C3
:10E88000112804D04FD8062853D00E28ECD10023ED
:10E89000013C4F4FDFF840814E4EADF804308DF80B
:10E8A0000630E4B2E1B24046FEF70DFCD7F86851FD
:10E8B000024600210120A847054600282FD0036A00
:10E8C0006BB340790D282AD86B7FC3F3C0138DF842
:10E8D0000530F8F77BFF012380B203FA04F2002829
:10E8E00062D0B6F8C030184214BF012300238DF85F
:10E8F0000430B6F8C23018420CBF012300239DF843
:10E9000004108DF80630D6F89031002958D0134302
:10E91000C6F8903100222B6A01A92846984714F1C5
:10E92000FF34BFD2A0E7132803D040F2E92290427F
:10E930009AD10023013C264FDFF89C80254EADF88C
:10E9400004308DF80630E4B2E1B24046FEF7BBFB7E
:10E95000D7F86851024600210120A8470546B0B10A
:10E96000036AA3B101A94079FFF786F948B19DF880
:10E970000410D6F890210123A34061B922EA0303D1
:10E980000AE001A96879FFF7A7F90028EFD114F18F
:10E99000FF34D9D268E71343C6F8903100222B6ABE
:10E9A00001A928469847F2E7D6F890311A4214BFD9
:10E9B000012300238DF804302B7FC3F3C1039EE7AE
:10E9C00023EA0203A4E700BF082300204C00002034
:10E9D000F0990020489D00200402002018B10C4B43
:10E9E0001A6802B9186019B10A4B1A6802B919609D
:10E9F000094B1A7852B901221A70084B084A996FCC
:10EA000011600848084A9A670EF0CEB9704700BFF7
:10EA10001023002008230020042300200C9C002049
:10EA20000C230020BC03002019DD0008036837B563
:10EA30001A78DB78DA42044603D10025284603B071
:10EA400030BD164B02691A60FEF704FF0028F4D0AF
:10EA500020681349C378027800910121FEF77EFFF8
:10EA600005460028E9D0FEF733FF88B1012322696B
:10EA700003702368026162694261DA7803620AB155
:10EA8000626842601B781BB1E368C360A368C3611E
:10EA900000210846FFF7A2FFD0E700BF182300209F
:10EAA000C9D400082DE9F84381461F461AB3134B19
:10EAB00093F84460CDB22E421AD00424013C26FAC9
:10EAC00004F3DA0712D525FA04F3DB070ED559F85B
:10EAD000248057F824104046F2F7B2FB58B907EBF0
:10EAE000840340461969F2F7C9FB20B9002CE5D12F
:10EAF0000120BDE8F8830020FBE700BF409900201B
:10EB00002DE9F04F95B00F460AA981E80C00209B33
:10EB10000093994BD3F814310693984B93F8AD10AA
:10EB2000974B1B781942044606D1219B069C012273
:10EB3000A04715B0BDE8F08F0A9B01930B9B029391
:10EB40009DF87C3003939DF87D300593BDF90C3022
:10EB500004934FEA830850F82330019918461D4664
:10EB6000F2F7C6F8BDF914B002994FEA8B020646D7
:10EB700054F82B000792F2F7BBF807EB0803089351
:10EB8000049B019957F8239082464846F2F7B0F863
:10EB9000079A0990BB188046029957F82B000793F3
:10EBA000F2F7A6F8009B002B0246099B4FDD009B65
:10EBB000012B40F0E7800021F2F756FB00210028EE
:10EBC00078D04046F2F75AFB002100285ED050462C
:10EBD000F2F74AFB002100283ED03046F2F73AFB1C
:10EBE000002840F0508131464046F2F733FB0028C0
:10EBF00040F04B810346009A002ADEB200F3C38046
:10EC000023460DF1300C04F1100E18685968624665
:10EC100003C2083373459446F7D149462846F2F7B4
:10EC20002DFB00287FD0039B14AA02EB830343F83B
:10EC3000209C079B54F82B80D3F80090414648460F
:10EC4000F2F71CFB002800F0C180C846BEE0504629
:10EC5000B04692461E46AEE73046F2F7FBFA002871
:10EC600014BF03230723009A002ADEB200F38B802F
:10EC700023460DF1300C04F1100E186859686246F5
:10EC800003C2083373459446F7D18CE05046F2F73F
:10EC9000EBFA002130B13046F2F7F0FA0028A2D0AA
:10ECA0000E23E0E73046F2F7D5FA002814BF02231E
:10ECB0000623D8E74046F2F7C3FA0021002834D0F3
:10ECC0005046F2F7BDFA002170B13046F2F7D6FA9D
:10ECD000002840F0EB8031464046F2F7C5FA0028A4
:10ECE00040F0F580064606E03046F2F7C7FA002805
:10ECF00014BF0C260D26009B002B40F3C880F6B2F3
:10ED00003B460DF1300C07F1100E18685968624649
:10ED100003C2083373459446F7D149462846F2F7B3
:10ED2000ADFA002844D1A94642E05046F2F788FAED
:10ED30000021C0B13046F2F783FA0028CBD00B2671
:10ED4000009B002B40F3B480F6B23B460DF1300C33
:10ED500007F1100E18685968624603C208337345FC
:10ED60009446F7D11FE03046F2F788FA002814BF26
:10ED700008260926BFE700BF0C9C00204099002010
:10ED80001D9C04080F233A460DF1300C07F1100EBC
:10ED900010685168664603C608327245B446F7D11A
:10EDA000DEB2B007B9D51E990198F1F7A1FF8146EF
:10EDB000039B14AA02EB8303710743F8209C7FF5A1
:10EDC00038AF1E990298F1F793FF8046059B069D88
:10EDD0004FEA830914AB4B44012243F8208CDFF83F
:10EDE000F880219B98F8AD100CA8A84700283FF4A4
:10EDF000A0AE009B002BD4BF3D46254610AA05F1CE
:10EE0000100728686968134603C30835BD421A46CF
:10EE1000F7D132071ED501991E98F1F76BFF054611
:10EE2000039B14AA02EB830343F8105CF3071ED57F
:10EE300002991E98F1F75EFF044614AB9944254BE6
:10EE400049F8104C0122D3F8144198F8AD10219BD9
:10EE500010A86DE6089B1F68049B54F823503846A1
:10EE60002946F2F70BFA0028DAD03D46D8E7079B8F
:10EE700054F82B401D6821462846F2F7E1F9002896
:10EE8000DBD02C46D9E70123B5E60F23EBE622467B
:10EE90000CAB04F1100E106851689C46ACE80300FE
:10EEA000083272456346F6D1F6B236E7042622E709
:10EEB00022460CAB04F1100E106851689C46ACE879
:10EEC0000300083272456346F6D1F6B26BE70F26AF
:10EED00036E700BF0C9C0020409900202DE9F04F40
:10EEE00093B004AC80468A46934600211022C7B2F4
:10EEF00020462FF086FD08A807F084FA9DF83430EC
:10EF0000434E444943F01203002520468DF8343027
:10EF10000F9513F0AFFA96F8B43100934FF004094F
:10EF200009F1FF3927FA09F2D20716D554F829203A
:10EF30005AF8291001925846F1F7E4FF009B019A14
:10EF4000014623FA09F010F0010F05F10105104602
:10EF50004ED0F1F7CFFE44F82900B9F1000FDFD110
:10EF60002846F1F777FF766C2B4D36F023FA0146F1
:10EF70003046F1F7C7FF294B08905B7F8DF836309C
:10EF800008A92046264C06F04DFF0423A37284F8FE
:10EF90000B8011F0F7F810F0CFFD11F0F3F8A36B30
:10EFA00013F0640F30D0A66B1E4D16F0200F03D067
:10EFB000AB6C1D4806219847730603D5AB6C1A4805
:10EFC000072198476B6E9847ADF80C0040EA102077
:10EFD000384203D0AB6C144808219847E66B56B111
:10EFE00002F0F2FF07F074FF002013B0BDE8F08FCD
:10EFF000F1F77EFEAFE76B6C0C480421984710F0E8
:10F0000097FFA6720120F0E7EB6D04209847C4E754
:10F01000489D0020DC9900200C9C00204098002096
:10F0200040990020F09900207C99002078990020D8
:10F0300010B50C4C94F8B32112F0020309D0C0B201
:10F0400090FAA0F20028B2FA82F214BF13464FF0F1
:10F05000FF33242202FB034301290CBF986C586C38
:10F0600010BD00BF489D00202DE9F04F8A4B85B0B0
:10F0700093F84430009304460D461646002B00F0EA
:10F080009980002963D003F00703072B5FD14FF06D
:10F0900000080327DFF8089201E04FF00108013F64
:10F0A00055F8271054F82700F1F722FE494620F0C2
:10F0B0000040F2F7E3F8002800F0EA8008F10108C8
:10F0C000002F41D0B8F1020FE7D12368D5F800B086
:10F0D000039359461846F1F70BFE6B6801931946E6
:10F0E00081466068F1F704FEAB6802931946074653
:10F0F000A068F1F7FDFD039BD6F800A080465146BD
:10F100001846F2F79DF8039B002856D05946504602
:10F11000F1F7EEFD494683463846F1F7A7FF594619
:10F12000F1F7F0FE0199F1F7E5FD494660604046D0
:10F13000F1F79CFF5946F1F7E5FE0299F1F7DAFD88
:10F14000C4F800A0A06040E0B8F1020FBDD04FF0BD
:10F15000040B4FF024084FF0000A009B0BF1FF3B1B
:10F1600023FA0BF3DB0722D54C4B08FB0B3351463C
:10F17000D86BF2F765F8D0B106EB8B0354F82B503F
:10F180001F6928463946F2F75BF800287CD13946DA
:10F1900056F82B904846F2F753F830B139462846D6
:10F1A000F2F74EF8002871D1B94644F82B90BBF124
:10F1B000000FD2D105B0BDE8F08FD6F810A01846E8
:10F1C0005146F2F75BF80028A0D1D4F804A0D6F895
:10F1D00004B050465946F2F733F8E8B1696858462A
:10F1E000F1F786FD394682464846F1F73FFF514622
:10F1F000F1F788FE2968F1F77DFD39462060404629
:10F20000F1F734FF5146F1F77DFEA968F1F772FD81
:10F21000C4F804B0A06007E0D6F814B050465946D0
:10F22000F2F72CF80028D9D1D4F808A0D6F808B005
:10F2300050465946F2F704F8E8B1A9685846F1F784
:10F2400057FD414682464846F1F710FF5146F1F717
:10F2500059FE2968F1F74EFD414620603846F1F726
:10F2600005FF5146F1F74EFE6968F1F743FDC4F81A
:10F2700008B060606BE7D6F818B050465946F1F711
:10F28000FDFF0028D9D162E7294681E7A9468CE72E
:10F29000002F7FF404AF5AE740990020489D0020DA
:10F2A0006F12833A40EA104343EA102303F0FF034E
:10F2B00082B043EA106002B07047000013B5104CF2
:10F2C0000190FFF7EFFF94F8AC30034215D0019B9B
:10F2D000C4F896300FF020FF40F2011318420CD111
:10F2E000E36B53B902F070FE064B9B6C012104F1F5
:10F2F0003C0002B0BDE81040184702B010BD00BF8E
:10F3000040990020F09900202DE9F04F264E274C1F
:10F3100096F8B29194F8443096F8B4B194F80CA0F1
:10F3200085B009F00802009396F84A310192204A0C
:10F3300003F001036434042500274FF024090099E9
:10F34000013DE940C9072BD513B32AFA05F1C807D7
:10F350001ED552F8258009FB05614046C96BCDE9F1
:10F360000232F1F7C7FCDDE90113039A91B12BFAE0
:10F3700005F1C9074DBF00F10040206027612760FB
:10F3800048BF2061043C002DD9D105B0BDE8F08F05
:10F39000B846E0E708F100482060C4F81080F1E7C3
:10F3A00027612760EEE700BF489D002040990020BC
:10F3B0001C2300202DE9F84F294D95F8B2318846DD
:10F3C0001907C7B211D52749042300200024013BA7
:10F3D00027FA03F2D20742BF01EB8302C2F89C0076
:10F3E0009464002BF3D1BDE8F88FDFF87890042403
:10F3F0004FF0000A4FF0004B013C27FA04F3DB0703
:10F400001ED595F8B431E34013F0010F4FEA84069E
:10F410001BD0242303FB0453D86BB8F1000F12D088
:10F42000114B9959F1F766FC242303FB04534E4416
:10F43000196BB064F1F766FD35F0C8FBC6F89C00A7
:10F44000002CD9D1CFE75946ECE7B8F1000F04D032
:10F45000054B985900F10040E6E75046E4E700BF4D
:10F46000489D0020409900201C2300202DE9F04FEA
:10F47000AA4B1D88A9B01DB1002029B0BDE8F08FAE
:10F48000A74CDFF8BC92C3B202931EA894F8B53122
:10F4900000935FFA81FB06F0B5FF9DF88C3025954F
:10F4A00043F012038DF88C309E4B01955B7F8DF8F5
:10F4B0008E304FF000084FF0040A46460AF1FF3A3A
:10F4C0000EAA0125029B05FA0AF542F82A5023FAF2
:10F4D0000AF2D00741D594F82D11242202FB0A42EA
:10F4E00021FA0AF111F0010FD26B12AF06D01046CB
:10F4F00000210392F1F7A4FE039A20B14946104679
:10F50000F1F700FD00E08848884A47F82A00926E2B
:10F510000021284690471AAA002142F82A000546F1
:10F52000F1F784FE0028A7D129462846F1F7EAFC26
:10F5300001464046F1F7DEFB57F82A508046314637
:10F540002846F1F77DFE00B92E462BFA0AF212F09A
:10F55000010F019B18BF53460193BAF1000FADD1C3
:10F5600000213046F1F762FE002840F03A82BBF1FC
:10F57000000F61D0D4F8A4016D4900F10040F1F70B
:10F5800075FD019A242303FB0243D96BF1F7BAFC02
:10F59000D4F8A851064601462846F1F76FFE00B19F
:10F5A0003546D4F8AC6129463046F1F749FE00B142
:10F5B0002E46019A242303FB02433046196BF1F7D0
:10F5C000A1FCF1F77BFE079094F83D31009A13F00F
:10F5D000100F14BF6523642309930123002503EB57
:10F5E0004203049300950395069516AF514938469A
:10F5F00012F040FF4A4B002693F8B43108934FF0C5
:10F60000000A0424324612AB0299013CE140059104
:10F61000C90733D54149089801EB8401E04010F057
:10F62000010FC1F89C20009853F824100AD002283A
:10F630000AD001F1004107E0CDF81CB0C4E7029602
:10F640000493D2E70228F4D047F82410CDE90A2326
:10F6500057F824001AAB20F0004053F82410F1F7BB
:10F6600005FD51468146F1F7EBFDDDE90A2300B1C6
:10F67000D1460EA9CA4611F824100E43002CC3D15E
:10F680002D4BD3F8B43023B1009A9DF808001AA985
:10F690009847009B022B24D1404635F08BFE28A9C9
:10F6A0001E4C41F8280D16A8E67206F0BBFB042399
:10F6B000A37210F067FD10F03FFA1C4C1F4F009B27
:10F6C000022B00F09D80636E9847012DADF830004D
:10F6D000C3B2C0F3072035D0022D00F08B80024664
:10F6E0008AE004241AAA16AF059B013CE340DB071D
:10F6F00011D552F8241008925046F1F703FC00216E
:10F70000814657F82400F1F7AFFD089A08B909F1CE
:10F71000004947F82490002CE6D1BDE7409900202D
:10F72000489D00204098002000000744F0990020E8
:10F730000000C842DC9900200C9C00207899002031
:10F740000000C0BF23EA0B09024649EA02091BEA8E
:10F75000090F19D0C5B958401BEA000F4ED00199C6
:10F76000A44A1BEA030F02EB81020CBF022501250C
:10F77000D2F89C20D4F890300692294658469847F3
:10F78000012329EA0B0903934FF004080EAB012172
:10F7900008F1FF3853F8282016420DD029FA08F254
:10F7A000D00709D501FA08F226EA02060198039A61
:10F7B000404508BF00220392B8F1000FE8D18D4BFD
:10F7C000039ADE72E2B1019A03EB8203069AD3F840
:10F7D0009C30D31A002B079AB8BF5B4293420FDDCF
:10F7E000854B86489B6C0F21984702F0EDFB07F094
:10F7F0006FFB41E620EA0B029946A6E70395C3E7B3
:10F8000010F0C0FC7B4B099A9B6B13EA02080BD0EB
:10F81000B8F1010F10D14146636C384698477849DA
:10F82000D4F8C4000BF052F9764B0420DB6D9847F6
:10F8300032077FF444AF2DE018F0200F03D0A36C03
:10F840006E480621984718F0400F03D0A36C6B4810
:10F8500007219847E36B002102209847009B022B69
:10F8600040F0C180636E9847029BADF8340040EAD7
:10F87000102000F0FF00034203D0A36C08215F4872
:10F8800098475C4BDB6B002BAFD15B4B5E485B6CEE
:10F890000421984710F04CFB5C4A574BB2F8B0017A
:10F8A000DB6BDFF8549100219847009B029E022BEE
:10F8B00009BF01230223564F00931CBF00934FF052
:10F8C0007E5704244FF00008013C26FA04F3DB07BE
:10F8D00028D5504B394653F82400F1F713FB4FF06D
:10F8E000010A12AB0AFA04FA5FFA8AFA43F8240012
:10F8F0000099D9F86830504698471AAB002143F870
:10F9000024000590F1F792FC059A10B126EA0A0648
:10F91000F6B211461046F1F7F5FA01464046F1F706
:10F92000E9F98046002CCFD1BBF1000F07D0324B54
:10F930002146D3F89030204698472546039400216D
:10F940004046F1F79BFC30B12EB1049B049A013B79
:10F95000002A7FF474AEBBF1000F32D02B4B019A1A
:10F960004FF0240808FB02380021D8F84040204618
:10F97000F1F75CFC054620BB00212046F1F760FC56
:10F980001D4F002814BF022101215846D7F890903E
:10F99000C847019B28AA02EB8302D8F8403023F025
:10F9A000004342F8583C12A94FF07E525846FFF7E8
:10F9B00095FA00283FF460ADD7F8903029462846E4
:10F9C000984701213046FFF7F5FC304601F09CF9DD
:10F9D000084B002293F844009A72029A024383F87B
:10F9E0004420012049E518F0040F3FF44AAFA36C0E
:10F9F000092144E740990020F09900207C990020DB
:10FA0000FC9A00200C9C002078990020489D002042
:10FA1000000020411C23002030B558B1064C03469D
:10FA200000F1100518685968224603C20833AB423A
:10FA30001446F7D1004830BD1C2300202DE9F04FBB
:10FA4000444C94F8B331990785B08046C6B24FF064
:10FA5000000704D5304605F083FC01283FD894F810
:10FA60004A013D4D4146AB6D00F001009847D5F885
:10FA7000A04014B10120A047C4B2344048D1374B54
:10FA80003946D3F810314046984780F00100404293
:10FA9000C0B23AE0EA0717D5B9F1FF0F13D00BFB5C
:10FAA0000A420BFB0943916C986C01920093F1F7A9
:10FAB000BDFB30B1019A009B516C586CF1F7B6FB5D
:10FAC00010B9054609E0D1460AF1010AC5F3470518
:10FAD000002DDFD1B9F1FE0FC1D101240BE0354675
:10FAE0004FF0FF094FF0000A4FF0240BF0E7F30747
:10FAF00005D401357608002EF9D1304605E004FA28
:10FB000005F0FFF79BFF0028F3D005B0BDE8F08FAC
:10FB1000D5F890300BB93720F7E74FF001070123F4
:10FB200000221C4212D002B11F469C42F3D16B6EE0
:10FB3000984740EA10202042A1D0094A0949384696
:10FB4000FFF7CCF900289AD12D20DEE75B00DBB26D
:10FB50000122E6E7489D0020F09900200C9C00203F
:10FB6000000020411C230020C1F3072138B54B07BA
:10FB700024D581F00201C1F3400169B3174C184D3F
:10FB8000238943F0040323810FF0C6FA08280146B5
:10FB90000AD12B6C04F13800984707F099F9D8B1D5
:10FBA0000FF0BAFA0028F8D102F00EFAAB6C0D484B
:10FBB00002219847BDE8384007F08AB907490A4B47
:10FBC0000122D3F8144101F1580391F8AD10A04778
:10FBD00080F00101C9B2D0E738BD00BF40990020D4
:10FBE000F09900207C9900200C9C0020094A92F892
:10FBF000B81192F8B9310B4392F8B71192F8B621C7
:10FC00000B431343044A92F8441013730B4082F8D9
:10FC100044307047489D0020409900200C4B93F8D9
:10FC2000B22102F00503052B0FD10A4B93F88E0089
:10FC300008B952060AD4187B40B193F8443030EA30
:10FC4000030314BF0120002070470020704700BF4D
:10FC5000489D002040990020084B094A9A66094BAC
:10FC6000094AC3F81421094AC3F81821084AC3F8FD
:10FC70001C21084AC3F81021704700BFF0990020EA
:10FC800031F000080C9C0020A5EA000801EB0008F8
:10FC900069F000086DF4000810B5074B002213F856
:10FCA000324084424FEAC20101D1581810BD0132DE
:10FCB000182AF4D10020F9E7209C0408034B044AD9
:10FCC0001B6850700BB11046184770476C2300201A
:10FCD000602300200348FF234370034B1B6803B1DC
:10FCE00018477047602300206C23002070B490F9FF
:10FCF0000730002B5ADB017A2D4B1029197052D88E
:10FD00004E002C4A7418145D002C4CD04C1E072C4D
:10FD100022D8DFE804F0121221212121040F012250
:10FD20009A70427A9A80244B1B68002B3ED0204860
:10FD300070BC184700229A70F5E7417A032928BF62
:10FD40000321997000228A42EDD2851803EB420408
:10FD5000AD7AA5800132F6E774181444A578F5B998
:10FD60006478E4B9447A6408032C28BF03249C70A7
:10FD7000BDB931440A445278002A14BF022203223A
:10FD800010440022A24200F10200CCD246798179CF
:10FD900003EB420541EA0621A9800132F2E7022481
:10FDA000E2E70222ECE7FF225A70BCE770BC704722
:10FDB000602300201C9F04086C2300202DE9F341E0
:10FDC0001D4B1D680024ADF8004085B31B4B182661
:10FDD00006FB05362746A04656F8143C013D9847D9
:10FDE00038B116F8183C012B1FD01BD3022B08BFCB
:10FDF0000124183E002DEFD19DF8003068F3000378
:10FE000067F3410364F382038DF80030BDF80030DE
:10FE10000020DAB262F307001B0A63F30F2002B07E
:10FE2000BDE8F0814FF00108E3E71F46E1E72C460B
:10FE30002F46A846E0E700BF5C2300202C230020CB
:10FE400038B50E4B1C68BCB10D4B182505FB0435AD
:10FE500055F8043C013C6BB115F8182C012A04D06C
:10FE600003D3022A01D0002000E098472CB120B92A
:10FE7000183DEDE7002CFBD1002038BD5C230020AD
:10FE80002C230020024B1868003018BF0120704757
:10FE90005C23002038B5074B1C6854B1064B18256D
:10FEA00005FB043555F8103C013C9847183D002CE3
:10FEB000F8D138BD5C2300202C230020054B1B68A3
:10FEC000022B05D0044A182101FB0323DB681847E5
:10FED000704700BFF00300202C230020F8B5124B20
:10FEE0001B68022B04460D46164607D10F4B1B68B4
:10FEF000022B0ED1002000F00100F8BD0C4F4FF096
:10FF0000180C0CFB03731B6998470028EED00120E6
:10FF1000F1E7074A182101FB032320461B693246FB
:10FF200029469847E7E700BFF4030020F0030020CC
:10FF30002C230020F0B5134F3B68012B064694BFDD
:10FF40004FF0010C4FF0000C15D80F491824024651
:10FF500004FB031400F1180E10685168254603C510
:10FF6000083272452C46F7D13278022A05D1074A69
:10FF7000136001333B606046F0BD002AF9D1044AAA
:10FF8000F6E700BF5C2300202C230020F4030020B0
:10FF9000F0030020102809D800EB4000044A131891
:10FFA000125C002A14BF18460020704700207047DA
:10FFB0001C9F04082DE9F04387B0102981460D46A7
:10FFC00090461E469DF838407DD8404A01EB4103DB
:10FFD000D718D35C002B76D01022002102A82EF077
:10FFE00010FD3B4A8DF80B9013780193591C0123A7
:10FFF0008DF808304FEA18238DF80D30354B11700D
:020000040801F1
:100000000F9A1A60344B8DF80C500022072D8DF892
:100010000E801A605A601A8111D104238DF80930BC
:1000200005238DF80A3001222C4901A8FFF756FF5D
:10003000002814BF00204E2007B0BDE8F083E11C6B
:1000400049007B78C9B28DF8091083B3B8780823CA
:1000500090B18DF80A308DF809300DF10F039442FC
:1000600003F10203DFD936F8121003F8011C080A65
:1000700003F8020C0132F2E703318DF80A30630015
:100080008DF809108DF810408DF81130002CCAD071
:1000900033888DF813301A0A012C8DF81220C2D93A
:1000A00073888DF815301A0A8DF81420BBE7013DCE
:1000B000012D8DF810409ABF0734E4106400053418
:1000C0008DF80A40AFE70320B6E700BF1C9F040885
:1000D0006A2300206C230020602300200C9F04086A
:1000E00070B50C4CA36805460BB1012098470A4B2C
:1000F0001D600A4B02221A70094B5A68094B1A609C
:10010000236A98476369697A05F10B00BDE870407E
:10011000184700BF30250020902300200D25002027
:1001200080230020F4240020B0F5E13F11D0B0F589
:10013000164F10D0B0F5964F0FD0B0F5165F0ED019
:10014000B0F5965F0DD0B0F5166F14BF03200020F8
:100150007047052070470420704703207047022035
:10016000704701207047000008B5094B83F8CA109A
:10017000C9B2084B53F82100074B1860074B33F8FE
:100180001120074B1A60074B1B689847002008BDD9
:10019000489D0020689F040880230020F824002048
:1001A0000425002030250020014B1868FFF7BCBF54
:1001B00080230020024B93F8C801C0F3021070475F
:1001C000489D0020024B5868003018BF012070473E
:1001D00030250020054B06480649006810B4D3F8C6
:1001E000D0410822A446012310BC6047F0990020AA
:1001F0008823002080230020084909484FF49643B3
:10020000322210B4C1E90032064B0068D3F8D04165
:100210000822A446012310BC604700BF80230020B1
:1002200088230020F099002070B5174B174C18490F
:10023000D3F8D4510968012308222046A84740B1C9
:1002400023681846FFF770FF124A52F820209342A5
:1002500001D0FFF7D1FF104B01221A7023680F4C19
:100260001846FFF761FF0E4A32F810100D4A184683
:1002700011602268904763682BB10B4ABDE870405B
:1002800092F8C801184770BDF09900208023002023
:1002900088230020689F04087D230020302500204B
:1002A000F824002004250020489D0020014B1878E8
:1002B000704700BF7D230020024B1878003018BF24
:1002C000012070470D250020044A1378002BFCD133
:1002D000034B1A68034B1A60704700BF0C250020BF
:1002E000782300208025002038B5037823B100242E
:1002F000201C18BF012038BD2B4B93F90020002A89
:100300004DDB4378D2B2934214BF00230123002B6C
:10031000EDD043684FF49640984704460028E6D055
:10032000436C002BE3D0C36B002BE0D0836B002B1E
:10033000DDD0036B002BDAD0C369002BD7D0036C60
:10034000002BD4D0036A002BD1D0836A002BCED0EF
:100350001648174D9847174B626C1A60A26C5A608A
:10036000E26BDA60A26B1A61226B5A61E2699A61F0
:10037000226CDA61226A1A62E26C9A60D5F8AC31BA
:10038000002BB5D061780C4A1131D22098476178A2
:10039000D5F8AC31084A1131D1209847A8E78378C5
:1003A00003F01203102BAFE740040020410D0208B8
:1003B000F099002030250020809F040870B51C4A69
:1003C000137803F0FF06002BFAD11A4B1A4C1B7856
:1003D000DBB11A4D286828B11022314618302EF0B2
:1003E00010FB2E60164B174D1A68174B1A60174BEF
:1003F000D3F8E8319847164B00F5FA7018600123DE
:100400002370EB6998472B6A98472378072B09D10B
:100410000E4BD3F8E83198470D4B00F5FA70186091
:10042000012323700B4BBDE870401B68184700BFC9
:100430000C250020409900200D250020902300204D
:10044000782300203025002080250020F09900200E
:100450000825002070230020024B01461878FEF783
:10046000D9B800BF0804002008B50C4B70B1026871
:100470001A6042685A6082689A60094A1068FFF7F9
:1004800053FE33F81020074B1A6008BD06490A686E
:100490001A604A685A608A68EEE700BFF8240020B4
:1004A0008023002004250020989F040810B5094CE3
:1004B00062684AB1084B93F8C80161F3061083F8EB
:1004C000C80190470BF024FB6368002B0CBF35205C
:1004D000002010BD30250020489D002010B50C4C98
:1004E0002368A3B11B7E93B10A4B07221A700A4BF3
:1004F000D3F8E831984723685A8B084B1B6813449C
:100500001844074A074B186093680133936010BD85
:10051000902300200D250020F099002004250020C4
:100520001025002008250020064B10B51B68044646
:1005300098472CB904490548BDE8104008F0F6BDBD
:1005400010BD00BF8C23002064A0040869A004082B
:100550002DE9F74F8B4F3B78002B68D101238A4C54
:100560003B702378042B17D8DFE813F0050019003F
:1005700026003600F300854C854B20681B689842A6
:100580000AD0844B1B683BB9834B1B7823B9FFF718
:10059000A7FD23689B6A236000233B7047E07F4BE5
:1005A0007F4ED3F8E83135689847281A0028F3DCE5
:1005B000002333602370EFE77A4DEB6898470646D7
:1005C0000028E9D12B6A984703232370AB68002BDE
:1005D000E2D030469847DFE7734B6E4D18689A4675
:1005E000002845D001381860002841D1DFF8C481C7
:1005F000D8F80C300133C8F80C302B681A78CAB11F
:10060000012222705A6A12B15A6A5968904700232F
:100610002B6000233B702378032B08D05F4BD3F86B
:10062000E8319847614B1B6818445D4B186003B074
:10063000BDE8F08F5B4EB36998472B68DB7A984230
:1006400013D1B369984703060FD5B3699847584B40
:10065000B0F1FF3F08BFFC20187006232370D8F8C4
:1006600014300133C8F81430D3E704232370D0E7E3
:100670004C4E336998472B689A7A9042B0468BD398
:100680004C4E93F80AB0DAF8002003F10B093368F6
:1006900001333360484B5B689B1AB26993422CBFAD
:1006A000B361B2615FFA8BFBD8F81830984709F84C
:1006B000010B2868837A013BDBB28372002BF3D1F4
:1006C000037ADFF8DC80DFF8D4A0DFF8E09083B3B2
:1006D000ABF1020211460B300192F6F774FF2B6862
:1006E000019A1A44D17AC2B2914206D10BF1FF327B
:1006F0001A44D27AB2EB102F1BD032690132326128
:100700001A7832B1012222701A6A6AB900232B606A
:1007100001E006232370DAF8E8319847D9F8003071
:100720001844C8F8000037E71A6A5968FE20904755
:10073000ECE7286803780BB90523EBE70123237066
:10074000C369002BE2D080F80AB0C369043098472F
:10075000DCE7104B1B681B780BB101232370114B96
:100760001B699847134BB0FA80F0400918770B4B80
:10077000D3F8E83198470D4B1B681844084B1860B4
:100780000AE700BF0C2500200D2500208025002051
:1007900078230020902300207C230020F099002063
:1007A0000825002030250020F42400200425002006
:1007B00074230020102500208023002070B5174DE1
:1007C0000446686801306860201D01F1140551F885
:1007D000046B40F8046BA942F9D1204600F8182BAD
:1007E000BBB10F490979A1B9194603F1100551F8B8
:1007F000046B40F8046BA942F9D1DB680BB9236A9A
:10080000636222B9237E13B1064BC4E90833204644
:1008100070BD102200212EF0F4F8F8E7102500201A
:1008200040990020DD0401082DE9F84F0F46417979
:100830000C290546144602D883790C2B08D9BB68CD
:1008400013B90020BDE8F88F2968FD209847F8E724
:1008500002390730F6F7B7FE6B792B44020A9A711A
:10086000664A58711378002BFCD1654B587980F09B
:100870000100044000F0A380624E3378002BE0D1E9
:10088000DFF8A491DFF8A4A101233370C84699F8DA
:10089000003003F0FF02EBB93B4629465A48DFF827
:1008A0008CB1DFF86C91FFF789FFFFF719FC327804
:1008B00002F0FF03A2B9554A33701360524A137312
:1008C000534B1B68003318BF012388F8003084F0B5
:1008D0000100B7E7DAF85CB00EF01EFCD847D6E7A7
:1008E000DBF85CA00EF018FCD04798F80030043B11
:1008F000032BDCD8DFE803F002311E3CDFF80CA14B
:10090000DAF800305A6A1AB15A6A5968FF209047DB
:10091000DAF800301B7E002B14BF01230023337054
:10092000C5D13C4B1B6998473B4BB0FA80F040095E
:100930001877BCE7DFF8D4A0DAF800301A6A22B1E1
:100940001A6A5968354B18789047DAF800301B7EE0
:10095000003318BF01233370A9E72C4B1868C36913
:1009600013B1C369043098470020307004469EE7F5
:100970002B4BD9F800A0D3F8E8319847AAEB000038
:10098000002894DCDFF884A00023C9F80030DAF8EE
:1009900000301A7E013AD2B21A762AB9BA681A62BF
:1009A000FA6802B9BA685A62183300222946164812
:1009B000FFF704FFCAF80000FFF792FB77E7134B3D
:1009C0001A683AB1104B197B21B1D27ADB7A934283
:1009D0003FF47DAFDFF85880124BD8F800601B68F9
:1009E000B26A9A423FF473AF3B4601222946304631
:1009F000FFF7E4FEB36AC8F8003068E70C25002072
:100A0000409900207C2300205425002090230020C2
:100A10000825002030250020102500207423002008
:100A2000F0990020802500200D2500200C9C00203E
:100A30007823002030B5184C237FA3B00D464BB16E
:100A40002068164A164B0221002814BF104618468B
:100A500008F010FBA369049323690393636902936D
:100A6000E3680193A36800936D2163680D4A06A8AB
:100A70002FF06EFC012106A808F0FCFA4DB12B788E
:100A800003F0DF03522B04D12022002102482DF075
:100A9000B8FF002023B030BD1025002070A004084E
:100AA00096A00408B6A0040870B5514B514C1870BC
:100AB00088B00D465048002110F0B0F890B994F875
:100AC00007326FF3451384F8073294F807329B0618
:100AD00006D44A494A48FBF775FF102011F020FD63
:100AE00008B070BD082004F0FBFD464B18600028DC
:100AF00094F8073214BF0122002262F3451384F8F0
:100B00000732E2D0404EB36833BBA81C24D0012288
:100B1000114601A8FDF708FD691C08BF9DF80850A3
:100B20003A4908BF05F1FF35EDB200230D701A46B2
:100B300001A8079DA84728B1354BB3600022D421F6
:100B4000FDF754FBB36894F80722003318BF012364
:100B500063F3451284F8072294F807329A06AED55B
:100B600000212C48FBF764FE94F8073260F345132C
:100B700084F807320028A8D0274BD4F8B0211A6097
:100B8000264BC4F8B031264B264A996E1160264890
:100B9000264A9A660CF008F9254A264B1360264A25
:100BA000C3F85C31136003F12C029A6203F158021E
:100BB0005A6503F18402C3F8802003F1B002C3F840
:100BC000AC2003F1DC02C3F8D82003F58472C3F82B
:100BD000042103F59A72C3F830211848FFF7AAF9E7
:100BE000174811F0F3FA0020FFF768F96DE700BF2E
:100BF00040040020F0990020E9020108B09F040899
:100C000027910108882300203025002008040020B7
:100C1000590401085105010870230020BD03010893
:100C20000C9C00208C2300200C04002029050108C6
:100C3000802500209423002078230020509F040862
:100C4000F80300202DE9F8430E46804608994FF03E
:100C50007E5017469946F0F74BF804460146304659
:100C6000F0F750F9394605460898F0F74BF9014678
:100C70002846F0F73FF8214605463846F0F742F996
:100C8000494607460898F0F73DF901463846F0F71F
:100C900031F80899F0F736F9214607462846F0F76B
:100CA00031F901463846F0F725F80899F0F72AF9A6
:100CB000214607464046F0F725F908998046304618
:100CC000F0F720F901464046F0F714F82146F0F716
:100CD00019F9294606460898F0F714F901463046F6
:100CE000F0F708F82146F0F70DF901463846F0F71D
:100CF00001F8BDE8F88300000149024811F0BABBD1
:100D0000DC990020982500202DE9F8431D4C1E4F4A
:100D10001E4D06464FF0040808F1FF38F3B223FADF
:100D200008F3DB0727D54FF0240909FB0849D9F858
:100D30003010D9F85000F0F7E5F833F047FFD0B1A4
:100D4000F0F788F8D9F83010F0F790F901232A78F5
:100D50000F4947F8280003FA08F3DBB294F8B4010E
:100D60001A432A7020FA08F00A78C00754BF1343C8
:100D700022EA03030B70B8F1000FCDD1BDE8F843B0
:100D8000FFF7BABF489D002084250020942500204D
:100D9000952500202DE9F04F4B7D03F00603062B2F
:100DA0008FB080460C4602D04969FEF7DDFE0EF09A
:100DB000B3F9022800F09C8006F08AF883460028E8
:100DC00000F09680504B1B780093002B56D04F4A72
:100DD00001921578082604270023009A324207F171
:100DE000FF371ED003934A4B58F8272053F827A00B
:100DF000029210465146F0F741FA4FEA8709DDE9C1
:100E00000223002843D035420BD0424A514659F8BC
:100E1000020025EA0605EFF76DFF3D4B43F8090098
:100E20005B467608002FD8D1E3B1019B04A81D7062
:100E300005F0E8FA23680493E3690B93E3680793EA
:100E4000227D9DF82430C2F3000243F0080362F3D0
:100E500000038DF8243004F059FF58BB04A92C4836
:100E600004F0E0FF2A4D434608F11006186859685F
:100E70002A4603C20833B3421546F7D106F028F8D4
:100E8000F0B104F043FFF0B105F09AFDF6E75146EA
:100E900010460293F0F7D4F9029B0028C1D03542E6
:100EA000BFD11C4B354359F803105046EDB2EFF754
:100EB0001FFFB2E705F084FD06F00AF80028CAD14A
:100EC0000FB0BDE8F08F2146404604F0ABFF78B983
:100ED00023699B7A1B070BD5237903F00303012BAE
:100EE00006D106F0BDFA2069E268436A2179984785
:100EF000094B1A782AB9587880F0010000F00100F7
:100F0000DEE70020FAE700BF9425002095250020A9
:100F10009825002084250020409900200000000032
:100F20002DE9F04FA7B014460C939DF8C4300993F7
:100F30009DF8C530BDF924A008939DF8C6301493E0
:100F40000C9B05904FEA8A094B4415930C9B53F870
:100F50002A008B46EFF728FBBDF92050069001F1DF
:100F600000430A930C9BAF003B4416930C9B53F831
:100F700025008846EFF718FB01F1004307900B931B
:100F800054F82A0004EB09030E461793EFF70CFB05
:100F9000069A4346EFF7AAF9E319CDE90E0154F892
:100FA00025001893EFF700FB079A3346EFF79EF9F9
:100FB000059BCDE9100153F82A00EFF7F5FADDE9BA
:100FC0000E23EFF791F9059BCDE9120153F82500A7
:100FD000EFF7EAFADDE91023EFF786F9DDE91223EE
:100FE00006460F4606980A99EFF736FB32468046CA
:100FF00089463B4607980B99EFF72EFB02460B46B6
:1010000040464946EFF772F9324680463B468946EC
:1010100006980A99EFF720FBDDE9122306460F46F2
:1010200007980B99EFF718FB02460B4630463946F6
:10103000EFF75AF942464B4634F0BEF8EFF704FE9C
:10104000329B002B804640F38581BD49F0F702F9C1
:1010500050B14046EFF7A8FAB5A3D3E90023EFF764
:1010600045F9EFF7F1FD80469BF815305A0728D473
:10107000B44AD2F8186126B343F004038BF8153054
:10108000DDE90E01EFF7E0FD1C90DDE91001EFF75F
:10109000DBFDAD4B0393329B0293319BADF80430E3
:1010A0001B0C8DF80630309B1D9000931CAB0CCBB5
:1010B00021460598B0479BF8153060F341038BF843
:1010C0001530329B002BB8BF5B42012B40F3AC8044
:1010D00003F1FF394846EFF7BDFEEFF765FA94A339
:1010E000D3E90023EFF7B8FA329B002B06460F46F0
:1010F000D4BF08F100404046EFF756FA32463B466F
:10110000EFF7F4F8EFF7A0FD04260746099B013E30
:10111000B3421BD0089BB34218D0059B54F826104D
:1011200053F82600EFF7E4FD3946EFF79FFF01463D
:10113000EFF7E0FDEFF738FA7FA3D3E90023EFF7ED
:101140008BFAEFF781FD22AB43F82600002EDDD1AC
:10115000059B1EAE03F1100718685968324603C29A
:101160000833BB421646F7D1099B26AA02EB83033C
:1011700054F82A2043F8202C089B26AA02EB83036C
:1011800054F8252043F8202C149B26A954F823203A
:1011900001EB83031EAD43F8202C329B002BCCBF08
:1011A00001274FF0FF3722AE4FF0040A099B0AF1E6
:1011B000FF3A53450AD0089B534507D055F82A00FB
:1011C00056F82A10EFF796FD45F82A00BAF1000FFD
:1011D000ECD19DF824308DF8C4309DF820308DF886
:1011E000C5309DF850308DF8C630319BADF80430D5
:1011F0001B0C8DF80630309B0093224602970C9B07
:1012000059462846FFF78CFE09F1FF39AC462246C5
:10121000634603CBB342106051609C4602F1080262
:10122000F6D1B9F1000FBFD130990846EFF762FD52
:10123000464B9D6829460646F0F720F800286FD0F7
:1012400029463046EFF754FD2946EFF75BFE34F0B0
:10125000B1F84FF07C5105464046EFF753FE309908
:10126000EFF750FE294620F00040EFF7FFFE33F085
:101270009DFBF0F749F81490002851D0EFF7EAFDF4
:101280009BF81450AB0606460AD50146DBF8000071
:10129000EFF738FE6FF34515CBF800008BF81450CC
:1012A00031464046EFF7E2FE0425814622AF099B16
:1012B000013DAB420ED0089BAB420BD0059B54F8CE
:1012C000251053F82500EFF713FD3146EFF7CEFE5A
:1012D00047F82500002DEAD149464846EFF712FEAF
:1012E00001464FF08040EFF703FD19490646484696
:1012F000EFF708FE4FF0814107463046EFF7FAFC62
:1013000001463846EFF7FEFD4FF07C511290304613
:10131000EFF7F8FD4FF0010A1990149B9A4528D178
:1013200059460598FFF736FD27B0BDE8F08F00BF9E
:10133000182D4454FB211940182D4454FB21094019
:10134000BD3706350C9C002098990020489D002050
:10135000ABAA2A3E5E49EFF787FF00283FF484AE30
:101360004046EFF721F958A3D3E90023EEF7BCFF7D
:1013700077E60B2D6DD81298EFF716F9CDE90C0131
:101380001998EFF711F9069A0A9B06460F46DDE910
:101390000C01EFF761F9079A0B9BCDE91A01304672
:1013A0003946EFF759F902460B46DDE91A01EEF727
:1013B0009DFFEFF749FC069A0A9B80463946304666
:1013C000EFF74AF9079A0B9B06460F46DDE90C0139
:1013D000EFF742F902460B4630463946EEF784FFF6
:1013E000069040460A91EFF7DFF8013507900B9120
:1013F000069A0A9BDDE90E01EEF778FFEFF724FC71
:10140000179B079A18600B9BDDE91001EEF76EFF42
:10141000EFF71AFC189B04261860099B013EB342A3
:101420000BD0089BB34208D022AB54F8260053F8E7
:101430002610EFF75FFC44F82600002EEDD1594648
:101440002046FFF7A7FC00283FF46EAF0AF1010A1F
:1014500063E75046EFF7FEFC4946EFF753FD0546BC
:1014600033F0B4F90646284633F02EFE159B1B6870
:1014700003F10048169B0746314640461D68EFF7CA
:1014800041FD394606902846EFF73CFD069B014694
:101490001846EFF72FFCEFF787F806900A914046C1
:1014A0003946EFF72FFD314607462846EFF72AFD6C
:1014B00001463846EFF71CFCEFF776F80025079059
:1014C0000B9195E7AFF30080182D4454FB21194090
:1014D000BD3706B52DE9F04F97B012AC0F930E90C3
:1014E00010910292134602F11005186859682246BD
:1014F00003C20833AB421446F7D1DFF8E881002578
:101500004FF07C5941462846EFF7F4FB4FF07E51EF
:101510000446EFF7B3FE08B14FF07E54029B1B6800
:1015200003930F9B03981B680493209B04991B68EB
:1015300005930E9B059A1B6800940693FFF782FBA8
:10154000029B5B6807930F9B5B680893209B08993D
:101550005B6809930E9B099A5B680094074607989D
:101560000A93FFF76FFB129B0B93139B0C9306469A
:101570000023294620460D93EFF7BAFB5849EFF7B1
:1015800073FE10BB0D9B4BB929462046EFF7B0FB0D
:1015900054498046EFF75EFE002858D12946204680
:1015A000EFF7A6FB10991297804612A81396FFF743
:1015B000F1FB38B14FF07E5120462546EFF740FE53
:1015C00000289FD117B0BDE8F08F29462046EFF7DD
:1015D00091FB4946EFF796FC069B00908046059AE2
:1015E00004990398FFF72EFB099A0A9B0899CDF8F6
:1015F000008082460798FFF725FB314683460C980A
:10160000EFF778FB4946EFF77DFC01465846EFF7C8
:101610006FFB394620F000430B981193EFF76AFBFC
:101620004946EFF76FFC01465046EFF761FB119B0F
:1016300020F000411846EFF75DFB2A49EFF70AFE5C
:1016400000289FD15E4657464446012391E7414614
:101650004046EFF74FFB2946EFF74CFB4FF07E512A
:101660008046EFF701FE002898D1069B059A049961
:10167000CDF800800398FFF7E5FA099A0A9B0899CC
:10168000CDF8008082460798FFF7DCFA5146834682
:101690000B98EFF72FFB4946EFF734FC014638462D
:1016A000EFF726FB594620F000430C980D93EFF717
:1016B00021FB4946EFF726FC01463046EFF718FBC1
:1016C0000D9B20F000411846EFF714FB0549EFF79A
:1016D000D5FD00287FF462AF5E465746444653E787
:1016E0006F12033BCDCCCC3D2DE9F04F8BB01446AF
:1016F000894605465169D66805934FF07E50EFF74D
:10170000B5FC94F82C300390D80748BFE769206AED
:1017100058BF00279907AB494CBFD4F81C804FF045
:101720000008EFF7EFFB33F00DFD21690090EFF7B4
:10173000E9FBD9F80810EFF7DDFA4B4604900DF1FC
:10174000180C09F1100E18685968624603C2083374
:1017500073459446F7D14FF0000A0AF1010B584641
:10176000EFF778FB039933F05FFA01463046EFF765
:10177000C9FB01462069EFF781FD002840F09B80FE
:10178000A36AD9F808106068023353440193EFF755
:10179000AFFA00218246EFF771FD48B194F82C3082
:1017A000DA0748BF07F10047980748BF08F100482B
:1017B00041463846EFF79EFA51468346EFF79AFACC
:1017C000A3690293824600211846EFF72FFD78B9EE
:1017D000029B51461846EFF795FB5946029050463A
:1017E000EFF786FA029B01461846EFF73FFCA0612F
:1017F0002B7D009843F001032B750021EFF716FDB8
:1018000000285AD001230293019B013B019363D02E
:10181000A168D9F800B03046EFF76CFA94F82C3094
:10182000666AD90702D52169EFF762FA3146EFF708
:1018300069FB5946EFF75EFA2946069006A8FFF7BE
:10184000A9FA002848D005F00BFE002847D02B7DD0
:101850006FF300032B752B7943F080032B716B7EA4
:1018600043F002036B7694F82C30DA073CD45146EF
:101870000898EFF73FFA2946089006A8FFF78AFA7A
:1018800050B394F82C309B0743D405F0E9FD10B910
:101890000DF042FC00BB2B7D43F001032B752B792F
:1018A0006FF3C7132B71019B012B47D1D9F800307F
:1018B000266906937EE0DA464FE700993046EFF757
:1018C00021FB01460498EFF713FA2946089006A871
:1018D000FFF760FA002895D10BB0BDE8F08F0DF04E
:1018E0001BFC0028B3D0F7E7616A2069EFF70AFB19
:1018F00001460698EFF7FEF9394606900898EFF78B
:10190000F7F92946089006A8FFF744FA0028AED157
:10191000E2E7616A2069EFF7F5FA01460698EFF70A
:10192000E7F9414606900898EFF7E2F92946089052
:1019300006A8FFF72FFA0028A7D1CDE7029BE6689B
:10194000013318460293EFF785FA039933F06CF9E7
:1019500001463046EFF7D6FAD4F810B006460146F5
:101960005846EFF78BFC00B95E4659463046EFF714
:10197000BFF9616AEFF7C6FAD9F80010EFF7BAF9C4
:101980002946069006A8FFF705FA0028A4D06B7E2A
:10199000059A009862F341036B760021EFF746FC4D
:1019A00090B900993046EFF7ADFA01460498EFF789
:1019B0009FF90890294606A8FFF7ECF900287FF464
:1019C00023AF89E735FA8E3C0021EFE770B50C466E
:1019D0000546E36E0360437D43F006034375037DD4
:1019E00043F014030375D4F8C430C3611A4B93F861
:1019F0004A315B07114604F1B00410D5174B184A61
:101A0000D3F81C312046984729462046FFF7C2F9F3
:101A10000DF082FB30F4007411D000200EE0114B69
:101A200093F8AD100029EFD00C4A5833D2F8146166
:101A300020460122B0470028E6D10F2070BD04F0F7
:101A40004FF90028E9D020200DF0A6FB0EF09AFBFC
:101A50000EF072F82046F1E7489D00200C9C002013
:101A6000989900204099002010B504460DF054FBD1
:101A7000022807D005F0F4FC20460021BDE8104004
:101A800003F046BB10BD00002DE9F04F89B01D46A4
:101A90009DF8483005939DF84930149E06939DF8B3
:101AA0004A300793137DBDF91C90D6F814B043F06B
:101AB0000103824688461375594655F82900144695
:101AC00005EB8907EFF7BCFB002854D1B37E55F82E
:101AD0002920012B5BD001924346294608F11000D2
:101AE00053F804CB41F804CB8342F9D145F82920BF
:101AF00021462846FFF74EF9002844D0059B05EB08
:101B000083030393069B05EB83030493139BFBB1B1
:101B1000D6F8149038684946EFF7B0FB002839D161
:101B2000079BD7F8009006EB83030293029BD3F840
:101B300000B049465846EFF783FB002833D1237D98
:101B400043F001032375139B013B139340F0A580E1
:101B500005F1100355F8042B48F8042B9D42F9D1E8
:101B60005E4B1A78002A40F0B780587880F0010068
:101B700000F0010008E045F829B021462846FFF7AB
:101B800009F90028A2D1002009B0BDE8F08F7369DF
:101B90000193A1E7C7F8009021462846FFF7FAF81D
:101BA0000028BDD1EFE7F1684846EFF7A1F881467C
:101BB00001465846EFF762FB00B1D946237D6FF32B
:101BC000000323752146C7F800902846FFF7E2F886
:101BD0000028D8D0BAF1540F1CD1637920690022B3
:101BE0004FF000010CF008FF0028CCD021792069CB
:101BF000E26881F00203C3F3400363F34101217102
:101C0000436A9847237983F00202C2F3400262F3E9
